:100000000C94E6160C9417170C9417170C941717EA
:100010000C9417170C9417170C9417170C941717A8
:100020000C9417170C9417170C9417170C94171798
:100030000C9417170C9417170C9417170C94171788
:100040000C9417170C9457240C9417170C9417172B
:100050000C9417170C9417170C94C5340C94A6B471
:100060000C9417170C9417170C9417170C94171758
:100070000C9417170C9417170C9417170C94171748
:100080000C9417170C9417170C9417170C94171738
:100090000C9441460C9417170C9417170C94AAAAA9
:1000A0000C9417170C9417170C9417170C94171718
:1000B0000C9417170C9417170C9417170C94062010
:1000C0000C9417170C9417170C9417170C94093EDF
:1000D0000C9417170C9417170C9417170C941717E8
:1000E0000C941717084AD73B3BCE016E84BCBFFD6A
:1000F000C12F3D6C74319ABD56833DDA3D00C77FF8
:1001000011BED9E4BB4C3E916BAAAABE0000008090
:100110003F05A84CCDB2D44EB93836A9020C50B91F
:10012000918688083CA6AAAA2ABE000000803F004B
:100130000C94D3390C9409AA0C947D390C9415FCB9
:100140000C9431C00D949B050C9482BF0C94E7FC79
:100150000C941DAC0C944FAC0C9418B40C9458FE39
:100160000C94E2380C9419AA0C9463B40C94DEEC51
:100170000C94F8F20D949E050C94A4390C940AAAE0
:100180000D9493050C9430390C949CFE0C94C33957
:100190000C94C5390C94BBFC0C9459B40D944306D3
:1001A0000C94C4FF0C94A7F40C9454AC0C9445FF2D
:1001B0000C944AAC0C940FAC0C942AAC0D942F0008
:1001C0000C94F2FE0C940EB40C9457390C94CEFEA1
:1001D0000C9445B40C94F9390C9497390C944FB4A1
:1001E0000C9419AC0C9424AC0C9417F60C9442ACFF
:1001F0000C94FCB30C940DFF0C9431B40C94BAEC39
:100200000C943CAC0D9472050C940EED0C9411FE04
:100210000C9446FC0C9417FC0C94EAB30C942BC180
:100220000C94641B0C9411FD0C944A390C9498F6B0
:100230000C94F4B30C940CEE0C94ABB90C9422B463
:100240000C94A3F80C94A0FE0C9475FC0C94B0FED6
:100250000C9434AC0C942CAA0C94C9EC0C945FFD57
:100260000C9423390C94ECEC0D94B1050C94673785
:100270000C94FEBA0C942FC00C9421AC0C945DF934
:100280000C94D6B30C945DF20C9409390D948E0540
:100290000C9446AC0C94A7F80C9471390C94D1EDE5
:1002A0000C943BB40C94ED390C94C7390C94371B67
:1002B0000C9419170C9469F70D9496050C945CFC3A
:1002C0000C9465F60C9444FD0C9415AC0C9449BB4D
:1002D0000C9438AC0C942CF90C9409BF0C94FC3899
:1002E0000C942EAC0C940BFA0D9434000C94C9B3FE
:1002F0000C94D1B30C9407BF0C9404B40C9435F354
:100300000C9494F90C9450AC0C9407F70C94E0B353
:100310000D942B004E414E494E495459494E46CDFD
:10032000CCCC3D0AD7233C17B7D13877CC2B3295AC
:1003300095E6241FB14F0A000020410000C842008A
:10034000401C4620BCBE4CCA1B0E5AAEC59D745301
:10035000746F7265642073657474696E677320725C
:100360006574726965766564006C6576656C696E46
:10037000675F6163746976653A0048617264636FB0
:100380006465642044656661756C7420536574749B
:10039000696E6773204C6F6164656400434D443A35
:1003A000303100434D443A0066616E5F793A200077
:1003B00066616E5F783A2000656E642073657475BF
:1003C00070006F6B206572723336365F73776974B5
:1003D00063683A0073745F696E6974004932435F01
:1003E000696E6974002020506C616E6E6572427592
:1003F0006666657242797465733A200020467265BC
:1004000065204D656D6F72793A200050524F20364D
:10041000313048545F56312E312E352E3800465734
:100420003A0020536F667477617265205265736578
:100430007400205761746368646F67205265736548
:1004400074002042726F776E206F7574205265734E
:100450006574002045787465726E616C2052657316
:10046000657400506F7765725570007374617274B3
:10047000002C20002C2000203A2073796E635F70DE
:100480006C616E5F706F736974696F6E0A00202013
:1004900063757272656E745F706F736974696F6E85
:1004A0003D004E6F7A7A6C65206175746F2D636CB8
:1004B00065616E656400416E6F746865722066697F
:1004C0006C616D656E7420697320746F6F20736842
:1004D0006F72740054776F2073656E736F7220644F
:1004E00065746563742066696C616D656E745F72B6
:1004F000756E6F757400416E6F7468657220666901
:100500006C616D656E7420697320656D707479001F
:10051000416E6F746865722066696C616D656E749A
:10052000206175746F2D6C6F6164696E67207374E0
:1005300061727400756E6C6F61645F74656D706577
:100540007261747572655B315D203D2000416E6F94
:10055000746865722066696C616D656E742069737C
:1005600020746F6F2073686F72740054776F2073FC
:10057000656E736F72206465746563742066696C60
:10058000616D656E745F72756E6F757400416E6F2C
:10059000746865722066696C616D656E742069733C
:1005A00020656D70747900416E6F746865722066A5
:1005B000696C616D656E74206175746F2D6C6F610F
:1005C00064696E6720737461727400756E6C6F611C
:1005D000645F74656D70657261747572655B305DC2
:1005E000203D20005072696E7465722073746F70C4
:1005F0007065642064756520746F206572726F7217
:10060000732E2046697820746865206572726F7257
:1006100020616E6420757365204D39393920746FFF
:1006200020726573746172742E202854656D706534
:100630007261747572652069732072657365742EBA
:100640002053657420697420616674657220726538
:100650007374617274696E67290041626F727420ED
:10066000434D44207768656E204175746F2D6C6F23
:100670006164696E672E0053746F70006F6B004E7B
:10068000006F6B004E6F204C696E65204E756D6279
:100690006572207769746820636865636B73756D34
:1006A0002C204C617374204C696E653A20004E6FAB
:1006B00020436865636B73756D2077697468206C7F
:1006C000696E65206E756D6265722C204C61737465
:1006D000204C696E653A2000636865636B73756DC5
:1006E000206D69736D617463682C204C6173742094
:1006F0004C696E653A2000636865636B73756D20A5
:100700006D69736D617463682C204C617374204C47
:10071000696E653A2000636865636B73756D3A00B6
:10072000636865636B73756D206D69736D61746368
:10073000682C204C617374204C696E653A2000521D
:10074000656365697665642067636F6465206C69BD
:100750006E653A004C696E65204E756D626572205B
:100760006973206E6F74204C617374204C696E65E0
:10077000204E756D6265722B312C204C6173742094
:100780004C696E653A20004D3131300073746570EC
:100790004C3A007374617274206368616E6765001F
:1007A000737465704C3A007374617274206368618D
:1007B0006E6765005400000025440000FE43000001
:1007C000FF4300000000000000000000A0C0000087
:1007D000000000000000000000003C3C3C20646F72
:1007E0005F626C6F636B696E675F6D6F76655F7478
:1007F0006F003E3E3E20646F5F626C6F636B696E9C
:10080000675F6D6F76655F746F00646F5F70726FA6
:1008100062655F726169736528006465706C6F79E9
:100820003A2000203A207365745F70726F62655FD2
:100830006465706C6F7965640A002020637572725C
:10084000656E745F706F736974696F6E3D00726579
:100850007365745F6265645F6C6576656C00202803
:10086000646F6E6529004578747261706F6C617495
:1008700065205B0042696C696E656172204C65762B
:10088000656C696E6720477269643A002028646964
:100890007361626C6564290041424C2041646A7551
:1008A00073746D656E74205A002028656E61626CE9
:1008B0006564290042494C494E45415200417574D6
:1008C0006F20426564204C6576656C696E673A20DE
:1008D0000020262053616D65205A20617300204E50
:1008E0006F7A7A6C65290020262041626F76650058
:1008F00020262042656C6F77002028416C69676E66
:100900006564205769746800205A3A0020593A00FB
:1009100050726F6265204F666673657420583A00A6
:100920004649585F4D4F554E5445445F50524F42D3
:10093000450050726F62653A2000436172746573BE
:1009400069616E004D616368696E652054797065F8
:100950003A2000203A2073657475705F666F725F8D
:10096000656E6473746F705F6F725F70726F6265D3
:100970005F6D6F76650A00202063757272656E7414
:100980005F706F736974696F6E3D00203A20636C0D
:1009900065616E5F75705F61667465725F656E64D8
:1009A00073746F705F6F725F70726F62655F6D6F8F
:1009B00076650A00202063757272656E745F706FD1
:1009C000736974696F6E3D003C3C3C2047323900CE
:1009D0006F6B20524520473239205331006F6B2016
:1009E000524520553520530020636F727265637441
:1009F0006564205A3A0047323920756E636F72720F
:100A00006563746564205A3A00203A203E20707273
:100A10006F62696E6720636F6D706C6574650A0044
:100A2000202063757272656E745F706F736974698C
:100A30006F6E3D00205A0047323920500020284474
:100A4000525952554E2900473239204175746F2052
:100A5000426564204C6576656C696E67006261630F
:100A60006B0066726F6E74007269676874006C6503
:100A70006674003F2856296572626F7365206C6545
:100A800076656C20697320696D706C61757369623D
:100A90006C652028302D34292E00426164205A20B4
:100AA00076616C7565004E6F2062696C696E656178
:100AB00072206772696400203A203E3E3E20473231
:100AC000390A00202063757272656E745F706F73EF
:100AD0006974696F6E3D0054726967657265642060
:100AE000706F736974696F6E206F7574206F662004
:100AF00072616E6765006F6B20524520473331206D
:100B00005330005072696E742061626F7274656454
:100B10002E006F6B205245204D3131322053310071
:100B20000052552066696C616D656E742069732092
:100B300072756E6F75740046696C616D656E7420B8
:100B4000646F6F72207374617475733A005255202C
:100B500066696C616D656E74206973206F6B0052FD
:100B6000442066696C616D656E74206973207275CE
:100B70006E6F7574200052442066696C616D656EFD
:100B800074206973206F6B20004C552066696C617E
:100B90006D656E742069732072756E6F75742000B8
:100BA0004C552066696C616D656E74206973206FA9
:100BB0006B20004C442066696C616D656E74206921
:100BC000732072756E6F757420004C442066696CDA
:100BD000616D656E74206973206F6B20006F6B20F0
:100BE0004D35383220005072696E74207061757313
:100BF00065642E006F6B205245204D3630322053F5
:100C000031006572725F70617573655F6275666CE5
:100C1000656E203D2000517569636B5F73746F7062
:100C20005F706C616E65645F6D6F766573203D20EB
:100C300000517569636B5F53746F705F67636F64B6
:100C4000655F4C6173744E203D20006F6B205245F0
:100C5000204D3630312053310053746F707065640D
:100C60005F67636F64655F4C6173744E203D200065
:100C70004D36303120427265616B004D36303100A7
:100C80004D313132006F6B205245205531302053A9
:100C900030006F6B205245205531302053310045D4
:100CA0006E636F6465725F636F756E745B315D2038
:100CB0003D2000456E636F6465725F636F756E748F
:100CC0005B305D203D20006F6B2052452055323750
:100CD000205330006F6B205245205532372053315E
:100CE00000456E636F6465725F636F756E745B3130
:100CF0005D203D2000456E636F6465725F636F75B4
:100D00006E745B305D203D20002057493A0020572B
:100D1000543A003A0020570000202F003A002048A3
:100D200000202F003A00204600202F0020423A00E9
:100D3000202F0020433A00202F002054313A002079
:100D40002F0054303A0041626F727420434D443A90
:100D500020006F6B205245204D363031205331003A
:100D600053746F707065645F67636F64655F4C6137
:100D700073744E203D20004D363031204272656143
:100D80006B004D363031004D313132006F6B4E000B
:100D9000526573656E643A200053746F70004E00A4
:100DA0006F6B006F6B0063757272656E745F706F4E
:100DB000736974696F6E5B455D3D00546172676570
:100DC000745F706F736974696F6E5B455D3D00524F
:100DD0006573656E643A200063757272656E745F48
:100DE000706F736974696F6E5B5A5D3D0054617218
:100DF0006765745F706F736974696F6E5B5A5D3D90
:100E0000005461726765745F706F736974696F6EA7
:100E10005B5A5D206973206D756368206C65737320
:100E2000207468616E2063757272656E745F706F96
:100E3000736974696F6E5B5A5D207768656E2070A8
:100E400072696E74696E672E0054617267657420F2
:100E5000706F736974696F6E5B5A5F415849535D77
:100E60002063616E2774206265206C657373207443
:100E700068616E20300020746F6F206C6F6E672089
:100E8000657874727573696F6E2070726576656EC1
:100E9000746564005072696E7465722068616C7468
:100EA00065642E206B696C6C28292063616C6C650D
:100EB0006421004552523A3130004552523A3100D5
:100EC0004C494E45004C494E45004C494E45004565
:100ED00052523A32004C494E45004C494E4500456D
:100EE00052523A3330004552523A33003000657264
:100EF000725F6C617374204552523A0020453A008B
:100F0000205A3A0020593A00583A0066696C616DDF
:100F1000656E745F626F785F3420697320656D70F1
:100F20007479207768656E20706F776572206F6EB8
:100F30002E0066696C616D656E745F626F785F33F9
:100F400020697320656D707479207768656E2070F4
:100F50006F776572206F6E2E0066696C616D656ECD
:100F6000745F626F785F3220697320656D70747989
:100F7000207768656E20706F776572206F6E2E0027
:100F800066696C616D656E745F626F785F31206950
:100F90007320656D707479207768656E20706F7747
:100FA0006572206F6E2E004368616E676520746FF6
:100FB0002066696C616D656E7420626F783A2000FE
:100FC00066696C616D656E745F626F785F6578638A
:100FD00068616E6765206661696C20004368616EB8
:100FE000676520746F2066696C616D656E74206240
:100FF0006F783A20006175746F20756E6C6F616454
:10100000206661696C2064756520746F2073656E5D
:10101000736F7220747269676765642E00617574FE
:101020006F2D756E6C6F6164206661696C206475EC
:101030006520746F2074696D656F75742E00466944
:101040006C616D656E742069732072756E6F757456
:1010500020616E6420737461727420746F206175F6
:10106000746F2D756E6C6F6164696E672E00496ECA
:1010700076616C69642066696C616D656E7420636D
:1010800068616D62657200416E6F7468657220669A
:10109000696C616D656E7420697320746F6F207365
:1010A000686F72742E00416E6F7468657220666995
:1010B0006C616D656E74206973206175746F2D6C41
:1010C0006F61646564207375636365737366756CC3
:1010D0006C79004175746F2D6C6F6164696E672067
:1010E0006C656E746820697320746F6F206C6F6E0E
:1010F000672E00203A203C3C3C20646F5F70726F8A
:1011000062655F6D6F76650A002020637572726597
:101110006E745F706F736974696F6E3D0071737781
:101120002070726F62655F73746174757332203DF5
:1011300020007173772070726F62655F73746174E1
:10114000757331203D20004C657373207468616EA7
:1011500020746865206D696E5F706F735B7A5D00E7
:1011600063757272656E745F706F736974696F6EA8
:101170005B5A5D00203A203E3E3E20646F5F7072F5
:101180006F62655F6D6F76650A002020637572720D
:10119000656E745F706F736974696F6E3D00337252
:1011A00064205A686F6D653A00326E64205A726529
:1011B00074726163743A007365636F6E6420686F64
:1011C0006D653A00726574726163743A00317374CC
:1011D00020686F6D653A0020563A006F6B205531DC
:1011E000330020563A006F6B205531330020413ACE
:1011F000006F6B20553133006F6B20553133204425
:101200003A006F6B2055313320443A0020746F6FE1
:10121000206C6F6E6720657874727573696F6E20CD
:1012200070726576656E746564006563686F3A0018
:10123000706C657465640074696D005A00590058DB
:1012400000450070756C5F636E7400796573004EC5
:10125000554C4C004C4E37373000000096C2000011
:1012600034420000254300808E430080CA43004082
:1012700003440040214400000000000082C200003E
:101280005C4200002F43008093430080CF4300C0A6
:1012900005440000000000000000205A3A002059D8
:1012A0003A0020583A00656E6473746F707320685A
:1012B00069743A20006563686F3A0024F4D43050B2
:1012C000C38E20C2A24017828B7011127A910D81B9
:1012D0006CD90AA861E108C7586607615143061E28
:1012E0004B5D05C145A7041A411104093D980371DE
:1012F0003931034036DB0265339102D43054028029
:101300002E1D02632CEE01752AC501B028A0011024
:101310002781018F2564012B244B01E0223401AC8D
:10132000211F018D200D01801FFC00841EED009700
:101330001DDF00B81CD200E61BC600201BBC0064E9
:101340001AB200B219A8000A19A0006A189900D1AF
:1013500017910040178B00B516840031167E00B33C
:101360001579003A157300C7146F0058146A00EE1F
:101370001366008813630025135E00C7125B006CC0
:1013800012570015125400C111510070114F002165
:10139000114B00D61049008D104700461044000242
:1013A000104200C00F4000800F3E00420F3C00067C
:1013B0000F3B00CB0E3800930E37005C0E35002734
:1013C0000E3400F30D3200C10D3100900D3000607D
:1013D0000D2E00320D2D00050D2C00D90C2B00AE6A
:1013E0000C2900850C29005C0C2700350C27000E09
:1013F0000C2600E80B2400C40B2400A00B23007D66
:101400000B23005A0B2100390B2100180B2000F888
:101410000A1F00D90A1E00BB0A1E009D0A1D00807B
:101420000A1D00630A1C00470A1B002C0A1B00113E
:101430000A1A00F7091A00DD091900C4091900ABDE
:10144000091900920917007B091800630917004C5D
:1014500009160036091600200916000A091500F5BC
:10146000081500E0081400CC081400B8081400A403
:10147000081400900813007D0812006B0813005830
:101480000812004608120034081100230811001247
:1014900008110001081100F0071000E0071000D04B
:1014A000071000C0071000B0070F00A1071000913F
:1014B000070E0083070F0074070F0065070E005723
:1014C000070E0049070E003B070D002E070E0020F7
:1014D000070D0013070D0006070D00F9060C00EDBF
:1014E000060D00E0060C00D4060C00C8060C00BC7B
:1014F000060C00B0060C00A4060B0099060C008D2B
:10150000060B0082060B0077060B006C060B0061D1
:10151000060A0057060B004C060A0042060A00386D
:10152000060A002E060A0024060A001A060A0010FF
:1015300006090007060A00FD050900F4050900EB8D
:10154000050900E2050900D9050900D0050900C711
:10155000050900BE050900B5050800AD050800A590
:101560000509009C050800940508008C0508008406
:101570000508007C050800740508006C0507006577
:101580000508005D050700560508004E05070047E1
:101590000507004005080038050700310507002A47
:1015A000050700230507001C050600160507000FA8
:1015B0000507000805060002050700FB040600F504
:1015C000040700EE040600E8040600E2040700DB5E
:1015D000040600D5040600CF040600C9040600C3B3
:1015E000040600BD040600B7040600B1040500AC03
:1015F000040600A6040600A00405009B040600954E
:10160000040500900406008A040500850405008096
:101610000406007A04050075040500700405006BDB
:1016200004050066040500610405005C040500571C
:10163000040500520405004D04050048040500435C
:101640000405003E0404003A04050035040500309A
:101650000404002C04050027040400230405001ED4
:101660000404001A04040016040500110404000D0B
:10167000040400090405000404040000040400FC40
:10168000030400F8030400F4030400F0030400EC76
:10169000030400E8030400E4030400E0030400DCA6
:1016A000030400D8030400D4030400D0030400CCD6
:1016B000030400C8030300C503030024F404D92075
:1016C0001BC40C5C0E9804C4095F0265077101F429
:1016D00005F900FB04B30048048700C10369005802
:1016E00003550003034500BE023A00840231005353
:1016F000022A002902250004022000E4011C00C87F
:10170000011900AF01170098011400840113007142
:101710000110006101100051010E0043010D00365F
:10172000010B002B010B0020010B00150109000C1F
:1017300001090003010800FB000800F3000800EBAA
:10174000000700E4000600DE000600D8000600D214
:10175000000600CC000500C7000500C2000500BD62
:10176000000400B9000400B5000400B1000400AD9D
:10177000000400A9000400A5000300A20003009FCC
:101780000004009B000300980003009500020093F2
:10179000000300900003008D0002008B000300880E
:1017A0000002008600020084000300810002007F26
:1017B0000002007D0002007B000200790002007739
:1017C0000001007600020074000200720001007146
:1017D0000002006F0002006D0001006C0002006A50
:1017E0000001006900020067000100660001006559
:1017F000000100640002006200010061000100605D
:101800000001005F0002005D0001005C0001005B60
:101810000001005A00010059000100580001005762
:101820000001005600010055000100540001005362
:10183000000000530001005200010051000100505F
:101840000001004F0001004E0000004E0001004D5D
:101850000001004C0001004B0000004B0001004A59
:101860000001004900010048000000480001004755
:101870000001004600000046000100450000004550
:101880000001004400010043000000430001004249
:101890000000004200010041000000410001004042
:1018A0000001003F0000003F0001003E0000003E3C
:1018B0000001003D0000003D0001003C0000003C34
:1018C0000000003C0001003B0000003B0001003A2A
:1018D0000000003A00010039000000390001003822
:1018E0000000003800000038000100370000003719
:1018F000000100360000003600000036000100350F
:101900000000003500000035000100340000003404
:1019100000000034000100330000003300000033F9
:1019200000010032000000320000003200010031EE
:1019300000000031000000310001003000000030E4
:10194000000000300001002F0000002F0000002FD9
:101950000000002F0001002E0000002E0000002ECD
:101960000001002D0000002D0000002D0000002DC2
:101970000001002C0000002C0000002C0000002CB6
:101980000001002B0000002B0000002B0000002BAA
:101990000001002A0000002A0000002A0000002A9E
:1019A0000001002900000029000000290000002992
:1019B0000000002900010028000000280000002885
:1019C0000000002800000028000100270000002778
:1019D000000000270000002700000027000100266B
:1019E000000000260000002600000026000000265F
:1019F0000001002500000025000000250000002552
:101A00000000002500000025000100240000002443
:101A10000000002400000024000000240001002336
:101A2000000000230000002300000023000000232A
:101A3000000000230000002300010022000000221B
:101A4000000000220000002200000022000000220E
:101A50000001002100000021000000210000002101
:101A600000000021000000210000002100010020F2
:101A700000000020000000200000002000000020E6
:101A80000000002000000020000000200001001FD6
:101A90000000001F0000001F0000001F0000001FCA
:101AA0000000001F0000001F0001001E0000001EBB
:101AB0000000001E0000001E00000073745F7379B8
:101AC0006E6368726F6E697A6500517569636B5FEA
:101AD00073746F705F636F64656C696E653D005110
:101AE0007569636B5F73746F705F63757272656E37
:101AF000745F706F736974696F6E5B5A5F415849A8
:101B0000535D3D00517569636B5F73746F705F6304
:101B1000757272656E745F706F736974696F6E5BF6
:101B2000595F415849535D3D00517569636B5F735F
:101B3000746F705F63757272656E745F706F7369D6
:101B400074696F6E5B585F415849535D3D00517534
:101B500069636B5F73746F705F63757272656E74C7
:101B60005F706F736974696F6E5B455F415849536D
:101B70005D3D0063757272656E745F74656D70654E
:101B80007261747572655F66696C616D656E7420F3
:101B9000697320746F6F206C6F772E4600637572C7
:101BA00072656E745F74656D70657261747572656F
:101BB0005F66696C616D656E7420697320746F6F08
:101BC00020686967682E46006C6173745F63757284
:101BD00072656E745F74656D70657261747572653F
:101BE0003A0063757272656E745F74656D706572CC
:101BF00061747572653A006F6B4E006D616E61675E
:101C0000655F6865617465722073657269616C5F98
:101C1000666C75736800202D20496E76616C69646E
:101C2000206578747275646572206E756D62657278
:101C30002021004572726F723A0070012C019001F0
:101C40002701B0012201C0011D01F001180110029D
:101C5000130130020E016002090190020401C0026A
:101C6000FF000003FA004003F5008003F000D003FA
:101C7000EB002004E6007004E100E004DC00400515
:101C8000D700C005D2004006CD00D006C8008007AE
:101C9000C3003008BE00F008B900C009B400B00AA3
:101CA000AF00B00BAA00D00CA500000EA000500F92
:101CB0009B00C01096005012910000148C00C015BB
:101CC0008700B0178200B0197D00D01B7800001E7D
:101CD000730040206E0090226900F02464004027C9
:101CE0005F0090295A00E02B5500102E5000203044
:101CF0004B0010324600E033410090353C00103775
:101D0000370070383200A0392D00B03A2800A03BCF
:101D10002300603C1E00103D1900903D1400103E51
:101D20000F00703E0A00C03E0500003F00000000AA
:101D30000000300E0100C00E0A00500F1400D00F3A
:101D40001E0060102800E010320070113C00F011FD
:101D500046007012500000135A00801364000014F3
:101D60006E00901478001015820090158C001016EB
:101D700096009016A0001017AA009017B400101833
:101D8000BE009018C8001019D2009019DC00101A7B
:101D9000E600801AF000001BFA00801B0401F01B13
:101DA0000E01701C1801F01C2201601D2C01E01DA9
:101DB0003601501E4001D01E4A01401F5401B01F81
:101DC0005E0130206801A020720110217C01902169
:101DD00086010022900170229A01E022A401502382
:101DE000AE01C023B8013024C201A024CC011025CB
:101DF000D6018025E001F025EA016026F401902A51
:101E00005802802EBC0250322003E0358403503942
:101E1000E803803C4C046003C800B003C300100416
:101E2000BE008004B900F004B4008005AF001006C5
:101E3000AA00B006A5007007A00040089B0020097A
:101E40009600200A9100500B8C00900C8700100E19
:101E50008200A00F7D004011780010137300001560
:101E60006E001017690050196400B01B5F00301E2F
:101E70005A00C020550050235000F0254B00802808
:101E80004600002B4100702D3C00C02F3700F03180
:101E90003200F0332D00C035280070372300E038C1
:101EA0001E00203A1900303B1400203C0F00E03C9B
:101EB0000A00803D0500003E00003A20456E635F49
:101EC0005370656564203D2000455F61626E6F72EE
:101ED0006D616C20004552523A3430004552523AFE
:101EE00034006F6B4E00526573656E643A004D317D
:101EF00030392048656174696E6720656E64004DF5
:101F00003130392048656174696E6720737461727D
:101F1000740053746F7000504944204175746F749D
:101F2000756E652066696E697368656421205075F9
:101F30007420746865204B702C204B6920616E649E
:101F4000204B6420636F6E7374616E747320696ECE
:101F5000746F20436F6E66696775726174696F6E26
:101F60002E6800504944204175746F74756E652069
:101F70006661696C6564212074696D656F757400B4
:101F800020403A006F6B20543A006F6B20423A00B9
:101F9000504944204175746F74756E65206661699F
:101FA0006C6564212054656D70657261747572652D
:101FB00020746F6F206869676800204B643A2000C6
:101FC000204B693A2000204B703A200020436C617E
:101FD0007369632050494420002054753A20002042
:101FE0004B753A2000206D61783A2000206D696EB3
:101FF0003A200020643A200020626961733A200090
:102000002044002049002020204D33303120500052
:102010005049442073657474696E67733A00205A9E
:102020000020590020204D323036205800486F6D76
:1020300065206F666673657420286D6D293A0020EF
:102040004500205A00205800204200205400202043
:102050004D323035205300416476616E63656420F3
:102060007661726961626C65733A20533D4D696EA9
:1020700020666565647261746520286D6D2F732913
:102080002C20543D4D696E2074726176656C20661B
:102090006565647261746520286D6D2F73292C202D
:1020A000423D6D696E696D756D207365676D656E16
:1020B000742074696D6520286D73292C20583D6D3E
:1020C0006178696D756D205859206A65726B20289A
:1020D0006D6D2F73292C20205A3D6D6178696D75C7
:1020E0006D205A206A65726B20286D6D2F73292C24
:1020F0002020453D6D6178696D756D2045206A65CC
:10210000726B20286D6D2F73290020540020204D04
:10211000323034205300416363656C6572617469C9
:102120006F6E3A20533D616363656C6572617469DB
:102130006F6E2C20543D726574726163742061630C
:1021400063656C65726174696F6E00204500205A8A
:102150000020590020204D3230312058004D617848
:10216000696D756D20416363656C65726174696F3B
:102170006E20286D6D2F7332293A00204500205AB9
:102180000020590020204D3230332058004D617816
:10219000696D756D2066656564726174657320286C
:1021A0006D6D2F73293A00204500205A00205900F8
:1021B00020204D39322058005374657073207065AB
:1021C0007220756E69743A006563686F3A007072C8
:1021D0006F62655F6F66667365743A200020413AEE
:1021E000006F6B20553133000000E0400000E040FC
:1021F00000007041FFFFFF000025440000FE430087
:10220000C00044556E6B6E6F776E20636F6D6D61AD
:102210006E643A200020434E54335F636F6D7061EB
:10222000726500206A756467656D7574696C790004
:1022300020434E54325F636F6D70617265002043BE
:102240004E54315F636F6D7061726500656E64201E
:102250004931006F6B2052452055333920533000EF
:102260006F6B2052452055333920533100456E6342
:102270006F6465725F636F756E745B315D203D20C6
:1022800000456E636F6465725F636F756E745B307B
:102290005D203D20006F6B20524520553336205382
:1022A0003100756E6C6F61645F74656D706572612D
:1022B00074757265203D2000456E636F6465725FC2
:1022C00053706565643A002045313A006F6B2052C7
:1022D00045205533342045303A30002045313A30DE
:1022E000006F6B205245205533342045303A00456D
:1022F0006E635F616C61726D5F656E61626C653AA1
:10230000006F6B20524520553333205300576172C4
:102310006E696E675F64656C61795F6D73203D20E7
:10232000004265645F6368616D6265725F666163E8
:10233000746F723A00204500204D006F6B205245AB
:10234000205533302053006F6B20524520553239D1
:102350002053006F6B2052452055323420533000FB
:102360006F6B2052452055323420533100706F7707
:1023700065725F6F66665F73746F7070696E6720F9
:102380003D20007072696E74696E675F6578747263
:1023900075646572735F6E756D203D2000436F6FCD
:1023A0006C696E67206C6576656C20616C61726D1E
:1023B00020656E61626C653A00544553545F4D4F21
:1023C00044453A0020523A00204C3A006F6B2052AC
:1023D000452055313800200020413A0020563A006F
:1023E000204C3A00204D3A0020433A0020443A0065
:1023F0006F6B20553133006F6B20524520553132C1
:10240000205331002046533A002050533A00204CCC
:102410003A00205A3A0020593A0020436F756E74F2
:1024200020583A200020453A00205A3A0020593AD4
:10243000006F6B20583A00506C65617365207075B1
:10244000736820746865206578747275646572209D
:102450006D6F746F7220746F20636C616D70207487
:102460006865207374616E6461726420737465655D
:102470006C2077697265206669727374004C494EEE
:1024800045004C494E4500456E636F6465725F635D
:102490006F756E745B315D203D2000456E636F6427
:1024A00065725F636F756E745B305D203D20004424
:1024B000617465526573756D65643A0020005F6FE5
:1024C00066667365743A0077656967687400200012
:1024D000203D20007765696768745F6761696E00F9
:1024E0006F6B20524520553520530020503000207E
:1024F0005031006F6B205245205534205330006F0F
:102500006B205245205534205331006F6B205245CB
:10251000205532205331006F6B2052452055322018
:102520005330006F6B205245205531205330006FDF
:102530006B205245205531205331004552523A000C
:102540006F6B205245205534362054312059006F8E
:102550006B205245205534362054302059006F6B83
:10256000205245205534362054312058006F6B20BE
:10257000524520553436205430205800205A6F667A
:1025800066736574006F6B205245205534362054B5
:1025900031205A006F6B205245205534362054307C
:1025A000205A0054726967676572696E6720626FAE
:1025B0006F746C6F61646572207669612055353087
:1025C000006F6B20524520553435205A00205A6F39
:1025D0006666736574006F6B205245205534342055
:1025E0005331205A006F6B2052452055343320530D
:1025F0000053746F707065645F67636F64655F4CF0
:102600006173744E203D20004552523A3030300004
:102610006F6B205245204D363031205331006472AB
:10262000697665725F616C61726D3A00452D7374F5
:102630006F70207374617475733A0044502E4F4E5E
:10264000207374617475733A005072696E746572A8
:10265000206D6F64653A007761746572206C6576F1
:10266000656C206973206F6B007761746572206CF4
:102670006576656C206973206C6F7700457874729D
:102680007564657220636F766572206973206F6B65
:1026900000457874727564657220636F7665722088
:1026A0006973206D69737300506F776572206F6670
:1026B0006620627574746F6E20697320646973613B
:1026C000637469766500506F776572206F66662067
:1026D000627574746F6E20697320616374697665C6
:1026E000004265642074656D702073776974636857
:1026F000206973206E6F726D616C00426564207496
:10270000656D7020737769746368206973207472D3
:1027100069676765726564004368616D6265722010
:1027200074656D7020737769746368206973206EB7
:102730006F726D616C004368616D626572207465D3
:102740006D7020737769746368206973207472698F
:1027500067676572656400546F7020646F6F7220E4
:10276000697320636C6F736500546F7020646F6FC2
:1027700072206973206F70656E0046726F6E7420F0
:10278000646F6F7220697320636C6F7365004672AB
:102790006F6E7420646F6F72206973206F70656E46
:1027A000004F666600466164652048656967687425
:1027B0002000426564204C6576656C696E67200078
:1027C0004572726F723A00466164650066697273A1
:1027D000742072756E20686173206E6F742062655C
:1027E000656E20646F6E653A00666972737420725C
:1027F000756E20686173206265656E20646F6E651A
:102800003A006F6B204D3232312053006F6B204DF8
:102810003232302053002C002C002C0020006F6B33
:10282000204D3231383A00496E76616C756564200E
:102830006F66667365745B5A5D00496E76616C7590
:102840006564206F66667365745B595D00496E76DA
:10285000616C756564206F66667365745B585D00B6
:102860002200556E6B6E6F776E20636F6D6D616EBB
:10287000643A20002074656D705F6F6666736574DE
:102880005F5A00205A00205900204D32303620581F
:10289000004D3139312048656174696E6720656E7D
:1028A00064004D3139312048656174696E67207369
:1028B00074617274004D3139302048656174696EFD
:1028C0006720656E64004D31393020486561746958
:1028D0006E6720737461727400205A5F55503A001D
:1028E00020595F46524F4E543A0020585F4C45469F
:1028F000543A00204C5F52494748543A00204C5FFC
:102900004C4546543A00205A5F4D41583A00205AEF
:102910005F4D494E3A0020595F4D41583A002059C9
:102920005F4D494E3A0020585F4D41583A002058BB
:102930005F4D494E3A006F6B204D313139200050C8
:10294000524F2036313048545F56312E312E352EBD
:10295000380046573A003A00204653002050533A78
:1029600000204C3A00205A3A0020593A0020436F88
:10297000756E7420583A200020453A00205A3A00DB
:1029800020593A006F6B20583A004D3130362054B0
:10299000312050004D3130362054302050004D3120
:1029A00030362054312050004D3130362054302004
:1029B00050002057493A002057543A003A00205717
:1029C0000000202F003A00204800202F003A00206D
:1029D0004600202F0020423A00202F0020433A00DA
:1029E000202F002054313A00202F006F6B205430EC
:1029F0003A006D61785F696E6163746976655F74D2
:102A0000696D653A002569206D696E2C2025692065
:102A1000736563006F6B205245204D323420533173
:102A20000066656564726174655F6D6D5F733D001E
:102A300066656564726174653D004C6173744E3AFD
:102A40000020523A004C3A004D313920004D6F744D
:102A50006572206F6666004D6F746572206F6E0040
:102A6000546F7020646F6F72206973206E6F7420D2
:102A7000636C6F73650046726F6E7420646F6F7263
:102A8000206973206E6F7420636C6F736500496EEC
:102A9000207072696E74696E672C206E6F7420618D
:102AA0006C6C6F7720746F2073746F70207468651E
:102AB0002076616375756D2073797374656D2E0072
:102AC0006F6B20524520473932006F6B006F6B00EF
:102AD00044502E4F4E20627574746F6E20697320BF
:102AE0006E6F7420707265737365642E0044502E8F
:102AF0004F4E20627574746F6E206973206E6F7410
:102B000020707265737365642E0044502E4F4E2002
:102B1000627574746F6E206973206E6F74207072AA
:102B200065737365642E006F6B2052452047323801
:102B300020533000776169743F00776169743F000A
:102B4000776169743F006F6B20524520473238200F
:102B50005331004477656C6C2F48656174696E670A
:102B600020656E640044502E4F4E20627574746F61
:102B70006E206973206E6F74207072657373656464
:102B80002E004477656C6C2F48656174696E672010
:102B90007374617274004E0020443A006F6B2055CC
:102BA0003133006F6B2072653336363A005532335D
:102BB000006F6B20524520553330204D006F6B2045
:102BC0005245205533302053006F6B20524520551D
:102BD00033302045006F6B20524520553239205349
:102BE0000067636F64655F4C6173744E0062756665
:102BF0006C656E0070617573650000002100240033
:102C000027002A002D0030003300010100000401DC
:102C100007010A0100002200250028002B002E00D9
:102C20003100340002010000050108010B01000021
:102C300020002300260029002C002F003200000174
:102C4000000003010601090105050505070508083F
:102C50000808020202020A0A080804040404010126
:102C6000010101010101030303030303030304073B
:102C700007070C0C0C0C0C0C0C0C020202020606D2
:102C80000606060606060B0B0B0B0B0B0B0B0102C5
:102C9000102020080810204010204080020102016E
:102CA0000804020101020408102040808040201026
:102CB000080402018004020180402010080402017F
:102CC00008040201010204081020408001020408E7
:102CD0001020408000000A0B02090C0D0E080703AB
:102CE00004010000000000000000000000000000DF
:102CF00000000000000000000000000000000000D4
:102D00001211100000000000000000000000000090
:102D100000000000000000000000203A203E3E3E7F
:102D20002072756E5F7A5F70726F62650A00202094
:102D300063757272656E745F706F736974696F6EBC
:102D40003D006F6B205245204732392053300050F0
:102D5000726F62696E67206661696C6564003C3CF5
:102D60003C2070726F62655F707400205A3A2000D8
:102D700020593A200042656420583A2000203A2029
:102D80000A00202063757272656E745F706F7369DC
:102D900074696F6E3D0073746F7729002C20002CCE
:102DA00020003E3E3E2070726F62655F70742800A6
:102DB000206669727374005A0059005800486F6D9C
:102DC0006520006563686F3A0000CE0011241FBEC5
:102DD000CFEFD1E2DEBFCDBF00E00CBF14E0A0E03A
:102DE000B2E0ECE3F5E202E00BBF02C007900D9207
:102DF000AE36B107D9F729E1AEE6B4E001C01D92C5
:102E0000A039B207E1F716E1C6EED6E100E006C050
:102E100021970109802FFE010F94920EC53ED10724
:102E200080E00807A9F70E94B7B80D949C120C9493
:102E3000000090E080E008951092FA0689988A9840
:102E400008952F923F924F925F926F927F928F924E
:102E50009F92AF92BF92CF92DF92EF92FF920F9329
:102E60001F93CF93DF93EC0129E330E090E080E003
:102E7000BC01620F731F75956795AB01440F551F19
:102E8000440F551FFA01E25DF24EA591B491AC17C3
:102E9000BD0711F5FA01E05DF24E65917491072EC0
:102EA000000C880B990B0F94CA0A4B015C01C501F9
:102EB000B401DF91CF911F910F91FF90EF90DF90C0
:102EC000CF90BF90AF909F908F907F906F905F90CA
:102ED0004F903F902F900895AC17BD070CF06AC03B
:102EE000CB010196281739070CF0C2CF37FF02C07B
:102EF00030E020E0220F331F220F331FF901E25D83
:102F0000F24EE590F4908A33910514F089E390E055
:102F1000880F991F880F991FFC01E25DF24E059101
:102F20001491F901E05DF24EC590D490FC01E05D92
:102F3000F24E25903490B6010D2C000C880B990BA5
:102F40000F94CA0A4B015C01E016F10609F4AFCFF9
:102F5000BE016E197F09072E000C880B990B0F9488
:102F6000CA0A2B013C01B1016C197D09072E000C26
:102F7000880B990B0F94CA0A9B01AC01C301B201E3
:102F80000F946A062B013C01B8016E197F09072EC8
:102F9000000C880B990B0F94CA0A9B01AC01C3016A
:102FA000B2010F94A90F9B01AC01C501B4010F94AC
:102FB000AF0E7BCF9B012150310994CF2F923F92CE
:102FC0004F925F926F927F928F929F92AF92BF9239
:102FD000CF92DF92EF92FF920F931F93CF93DF93E5
:102FE000EC012CE330E090E080E0BC01620F731F45
:102FF00075956795AB01440F551F440F551FFA0196
:10300000E65CF34EA591B491AC17BD0711F5FA013A
:10301000E45CF34E65917491072E000C880B990BBC
:103020000F94CA0A4B015C01C501B401DF91CF9135
:103030001F910F91FF90EF90DF90CF90BF90AF90D6
:103040009F908F907F906F905F904F903F902F90C8
:103050000895AC17BD070CF06AC0CB010196281784
:1030600039070CF0C2CF37FF02C030E020E0220F5A
:10307000331F220F331FF901E65CF34EE590F49005
:103080008D33910514F08CE390E0880F991F880F21
:10309000991FFC01E65CF34E05911491F901E45C83
:1030A000F34EC590D490FC01E45CF34E259034902F
:1030B000B6010D2C000C880B990B0F94CA0A4B011A
:1030C0005C01E016F10609F4AFCFBE016E197F096D
:1030D000072E000C880B990B0F94CA0A2B013C0198
:1030E000B1016C197D09072E000C880B990B0F9408
:1030F000CA0A9B01AC01C301B2010F946A062B01FD
:103100003C01B8016E197F09072E000C880B990B42
:103110000F94CA0A9B01AC01C301B2010F94A90F1D
:103120009B01AC01C501B4010F94AF0E7BCF9B0195
:103130002150310994CF2F923F924F925F926F921C
:103140007F928F929F92AF92BF92CF92DF92EF9237
:10315000FF920F931F93CF93DF935B01EA01FC0172
:103160004080518062807380BA017727463008F032
:103170006AC0660F771F660F771FFB01E658FD4E8A
:1031800085919591A591B491282E092F1A2F3B2E48
:1031900086E08A9DF0018B9DF00D1124EC0FFD1F40
:1031A000EE0FFF1FEE0FFF1FE75CF84FC080D180CE
:1031B000E280F380C530D10514F0C4E0D0E026E011
:1031C0002A9DC0012B9D900D11242196C80FD91F57
:1031D000CC0FDD1FCC0FDD1FC75CD84FA7019601B8
:1031E000688179818A819B810F94AE0E4B015C01CD
:1031F000222D302F412F532DC301B2010F94AE0E5B
:1032000029E838E848E05CE30F946A069B01AC01CA
:10321000C501B4010F946A06A70196010F94AF0E81
:10322000DF91CF911F910F91FF90EF90DF90CF90A2
:10323000BF90AF909F908F907F906F905F904F90D6
:103240003F902F900895072E000C880B990B0F9438
:10325000CA0A20E030E040EF52E40F946A0620E012
:1032600030E042E852E40F94AE0E262E072F182FBE
:10327000392E8ECF2F923F924F925F926F927F9214
:103280008F929F92AF92BF92CF92DF92EF92FF9276
:103290000F931F93CF93DF93EB015A01FC01408002
:1032A0005180628073807727C73008F06AC0660F4C
:1032B000771F660F771FFB01E65AFD4E85919591AA
:1032C000A591B491282E092F1A2F3B2E86E08C9FB2
:1032D000F0018D9FF00D1124EA0DFB1DEE0FFF1F75
:1032E000EE0FFF1FE75CF84FC080D180E280F380D3
:1032F000C630D10514F0C5E0D0E0219626E02C9F21
:10330000F0012D9FF00D1124EA0DFB1DEE0FFF1FA4
:10331000EE0FFF1FE75CF84FA701960160817181F6
:10332000828193810F94AE0E4B015C01222D302FD0
:10333000412F532DC301B2010F94AE0E29E838E896
:1033400048E05CE30F946A069B01AC01C501B4013F
:103350000F946A06A70196010F94AF0EDF91CF91EB
:103360001F910F91FF90EF90DF90CF90BF90AF90A3
:103370009F908F907F906F905F904F903F902F9095
:103380000895072E000C880B990B0F94CA0A20E0B1
:1033900030E040EF52E40F946A0620E030E046E966
:1033A00052E40F94AE0E262E072F182F392E8ECFF3
:1033B0008F929F92AF92BF92CF92DF92EF92FF9245
:1033C000CF93DF93EC018090E1079090E207A0900B
:1033D000E307B090E40720E030E0A901C501B401A3
:1033E0000F94C30A882309F454C0C880D980EA80A6
:1033F000FB80A7019601C501B4010F94C30A1816FA
:103400000CF04CC020910207309103074091040753
:1034100050910507C701B6010F94C30A882331F103
:10342000C0920207D0920307E0920407F0920507CA
:10343000209106073091070740910807509109072E
:10344000688179818A819B810F946A069B01AC0116
:1034500060E070E080E89FE30F94AE0E609311028D
:1034600070931202809313029093140260911102E0
:10347000709112028091130290911402DF91CF910A
:10348000FF90EF90DF90CF90BF90AF909F908F9084
:10349000089560E070E080E89FE3F0CF60E070E0C6
:1034A000CB01ECCFCF92DF92EF92FF92CF93DF93DD
:1034B000EC01C0907F02D0908002E0908102F090F9
:1034C0008202A7019601688179818A819B810F948C
:1034D000C30A87FF04C0C882D982EA82FB82C090F7
:1034E0008302D0908402E0908502F0908602A701CA
:1034F00096016C817D818E819F810F94C30A87FF25
:1035000004C0CC82DD82EE82FF8220E030E040EA1F
:1035100050E46091870270918802809189029091B5
:103520008A020F94AE0E6B017C01AC019B01688591
:1035300079858A859B850F94C30A87FF04C0C88656
:10354000D986EA86FB86C0903902D0903A02E09094
:103550003B02F0903C02A7019601688179818A8143
:103560009B810F940F11181624F4C882D982EA8225
:10357000FB82C0903D02D0903E02E0903F02F0906E
:103580004002A70196016C817D818E819F810F94FD
:103590000F11181624F4CC82DD82EE82FF82C090D7
:1035A0004102D0904202E0904302F0904402A70111
:1035B0009601688579858A859B850F940F11181669
:1035C00024F4C886D986EA86FB86DF91CF91FF90E6
:1035D000EF90DF90CF9008958091C80085FFFCCFD9
:1035E0006093CE0008958091BC0087FFFCCF84E9F2
:1035F0008093BC0008959091BC0097FFFCCF80930E
:10360000BB0084E88093BC000895CF93DF93D82F4C
:10361000C62F84EA8093BC0088E40E94FB1A8D2F99
:103620000E94FB1A8C2F0E94FB1ADF91CF910C9401
:10363000F31ACF93DF93D82FC62F84EA8093BC0070
:103640008AE40E94FB1A8D2F0E94FB1A8C2F0E9485
:10365000FB1ADF91CF910C94F31A80E1EEEBFAE0C4
:10366000A5E3B9E101900D928A95E1F70895CF9213
:10367000DF92EF92FF920F931F93CF93DF937C0122
:10368000CB018A0120917618222389F0EB016B018E
:10369000C40ED51ECC15DD0569F06991D701ED91F9
:1036A000FC910190F081E02DC7011995F3CF642FB3
:1036B0000E94CAABC801DF91CF911F910F91FF907B
:1036C000EF90DF90CF900895CF93DF931F92CDB707
:1036D000DEB76983209176182223F9F0209199189A
:1036E000203258F021E030E0FC013383228390E067
:1036F00080E00F90DF91CF91089580917718E82FA7
:10370000F0E0E858F74E998190838F5F80937718A7
:103710008093991881E090E0ECCF61E0CE010196B2
:103720000E94CAABF7CF4F925F926F927F92AF9297
:10373000BF92CF92DF92EF92FF920F931F93CF939E
:10374000DF938C01EB01FC0142A053A064A075A0A3
:10375000AAA0BBA0CCA0DDA09501A601C301B20127
:103760000F94C30A87FF3DC0A3019201C301B201B8
:103770000F946A062B013C01F80166A577A580A984
:1037800091A990589B01AC010F94AF0EF80122A5AE
:1037900033A544A555A50F946A069B01AC01C3014E
:1037A000B2010F94AE0E0F9404127B018C019B01A9
:1037B000AC01B501C6010F94C30A87FF02C07501B1
:1037C00086019701A801B501C6010F94C30A882399
:1037D00041F0C701D8018AA39BA3ACA3BDA381E09C
:1037E0008B8FDF91CF911F910F91FF90EF90DF9022
:1037F000CF90BF90AF907F906F905F904F90089563
:103800002F923F924F925F926F927F928F929F92F0
:10381000AF92BF92CF92DF92EF92FF920F931F93DE
:10382000CF93DF93CDB7DEB766970FB6F894DEBFC0
:103830000FBECDBF1C014A015B017901FC0182A9C9
:1038400093A9A4A9BC018A2F90E00F94C80A6987A4
:103850007A878B879C87A50194010F946A060F9441
:103860008D0F0F9422104B015C01A701980169850F
:103870007A858B859C850F946A060F948D0F0F9423
:1038800022108D829E82AF82B8862D813E814F812B
:103890005885283731054105510540F428E730E0C7
:1038A00040E050E02D833E834F83588769837A83BD
:1038B0008B839C8389819A81AB81BC8188379105F8
:1038C000A105B10540F428E730E040E050E029834D
:1038D0003A834B835C83F10183AD94ADA5AD9C012C
:1038E0004A2F50E0298B3A8B4B8B5C8BCA01B90174
:1038F0000F94CA0A6B017C0120E030E0A9010F940B
:10390000C30A882309F4FCC06D817E818F8198856C
:103910000F94C80A4B015C0129853A854B855C856B
:10392000CA01B9010F946A062B013C01A50194015B
:10393000C501B4010F946A069B01AC01C301B20139
:103940000F94AE0E4B015C01A7019601C701B601B1
:103950000F94AF0E9B01AC01C501B4010F94A90FE8
:103960006D877E878F87988B6D857E858F859889FB
:103970000F948D0F0F941B102B013C0169897A89DC
:103980008B899C8990958095709561957F4F8F4F1D
:103990009F4F0F94CA0A6B017C0120E030E0A9011F
:1039A0000F94C30A882309F4B0C069817A818B819E
:1039B0009C810F94C80A9B01AC010F946A064B01CD
:1039C0005C0129853A854B855C85CA01B9010F9454
:1039D0006A069B01AC01C501B4010F94AE0E4B0108
:1039E0005C01A7019601C701B6010F94AF0E9B01C0
:1039F000AC01C501B4010F94A90F6B017C01C70193
:103A0000B6010F948D0FD1011D968D909D90AC90B5
:103A10000A2C000CBB08A50194012419350946099C
:103A2000570929873A874B875C870F941B10298594
:103A30003A854B855C85261B370B480B590BDA0101
:103A4000C901B7FF29C0C501B4010F94CA0A2D8569
:103A50003E854F8558890F94AF0EA70196010F94AC
:103A6000AE0E20E030E040E05FE30F946A060F9472
:103A70008D0F0F941B1097FF03C060E070E0CB0127
:103A80002B013C0184149504A604B70410F424010E
:103A9000350180E090E0DC012FB7F894F101328D20
:103AA000311114C0518A408A840D951DA61D828B48
:103AB000938BA48B8D819E81AF8185AB96ABA7AB99
:103AC00089819A81AB8180AF91AFA2AF2FBF6696FB
:103AD0000FB6F894DEBF0FBECDBFDF91CF911F911F
:103AE0000F91FF90EF90DF90CF90BF90AF909F909D
:103AF0008F907F906F905F904F903F902F900895A0
:103B00001D861E861F86188A2FCFC12CD12C7601C8
:103B100076CF45E15AEB64E276E280E097E00F94DD
:103B2000EE0D40917305509174056091750570918B
:103B3000760584E097E00F94EE0D40916F0550916B
:103B40007005609171057091720588E097E00F949F
:103B5000EE0D40916B0550916C0560916D05709173
:103B60006E058CE097E00F94EE0D40916705509143
:103B700068056091690570916A0580E197E00F948E
:103B8000EE0D40916305509164056091650570915B
:103B9000660584E197E00F94EE0D40915F0550912A
:103BA0006005609161057091620588E197E00D9470
:103BB000EE0D4F925F926F927F928F929F92AF9293
:103BC000BF92CF92DF92EF92FF920F931F93CF930A
:103BD000DF93EC016091360570913705072E000CDC
:103BE000880B990B0F94CA0A9B01AC0168817981FB
:103BF0008A819B810F94AE0E6B017C016091380528
:103C000070913905072E000C880B990B0F94CA0A86
:103C10009B01AC016C817D818E819F810F94AE0EE2
:103C20004B015C01A701960160910C0270910D029D
:103C300080910E0290910F020F94C30A882309F419
:103C400054C0C0920C02D0920D02E0920E02F0928B
:103C50000F0220912E0530912F0540913005509193
:103C60003105C701B6010F946A062B013C010F9480
:103C700051106B017C0120E030E0A9010F94C30AD0
:103C800087FD74C020E030E040EC50E4C701B6018D
:103C90000F940F11181634F4C12CD12CC0ECEC2E5B
:103CA000C0E4FC2EA7019601C301B2010F94AE0E31
:103CB0002B013C0120E030E0A9010F94C30A87FDED
:103CC00059C040922A0550922B0560922C057092A3
:103CD0002D05C701B6010F941B10609329056530AF
:103CE0000CF051C06F5F60932805D09107021091CE
:103CF0002905A50194016091080270910902809143
:103D00000A0290910B020F94C30A81113EC0D11395
:103D100090C020910A0530910B0540910C055091FF
:103D20000D0560912A0570912B0580912C059091CD
:103D30002D050F946A0620910E0530910F054091D4
:103D40001005509111050F94AF0EDF91CF911F9187
:103D50000F91FF90EF90DF90CF90BF90AF909F902A
:103D60008F907F906F905F904F900895C12CD12CD1
:103D7000760198CF10922A0510922B0510922C05EF
:103D800010922D05A6CF66E0AECF809208029092E9
:103D90000902A0920A02B0920B02209132053091E2
:103DA00033054091340550913505C501B4010F9498
:103DB0006A064B015C010F9451106B017C0120E0FD
:103DC00030E0A9010F94C30A87FDF3C020E030E082
:103DD00040EA50E4C701B6010F940F11181634F4ED
:103DE000C12CD12CB0EAEB2EB0E4FB2EA70196013A
:103DF000C501B4010F94AE0E4B015C0120E030E030
:103E0000A9010F94C30A87FDD8C08092240590921F
:103E10002505A0922605B0922705C701B6010F948B
:103E20001B106093230564300CF0D0C06F5F60936B
:103E30002205C0912305D11305C0809106028C177D
:103E400009F46CC010930702C09306020C2E000CFC
:103E5000DD0B26E01203C0011124FC01EC0FFD1F55
:103E6000EE0FFF1FEE0FFF1FE75CF84F208131813F
:103E70004281538120931E0530931F0540932005F6
:103E80005093210500912205002E000C110BFC011E
:103E9000E00FF11FEE0FFF1FEE0FFF1FE75CF84F63
:103EA00060817181828193810F94AE0E60931A05B7
:103EB00070931B0580931C0590931D052091280588
:103EC00036E02303F0011124CE0FDF1FCC0FDD1FDE
:103ED000CC0FDD1FC75CD84F288139814A815B81B7
:103EE0002093160530931705409318055093190534
:103EF000E00FF11FEE0FFF1FEE0FFF1FE75CF84F03
:103F000060817181828193810F94AE0E609312055E
:103F100070931305809314059093150580902405E4
:103F200090902505A0902605B090270520911A05B0
:103F300030911B0540911C0550911D05C501B40130
:103F40000F946A0620911E0530911F0540912005AF
:103F5000509121050F94AF0E6B017C01C0920E05AC
:103F6000D0920F05E0921005F092110520911205F4
:103F7000309113054091140550911505C501B40108
:103F80000F946A0620911605309117054091180587
:103F9000509119050F94AF0EA70196010F94AE0E24
:103FA00060930A0570930B0580930C0590930D05A3
:103FB000B0CEC12CD12C760119CF109224051092CD
:103FC0002505109226051092270527CF65E02FCFF3
:103FD000EF92FF920F931F93CF938C017B01C42F1D
:103FE000F70161917F01F801808191810F94E00DCB
:103FF000F80180819181019691838083C15081F77E
:10400000CF911F910F91FF90EF9008951F920F9203
:104010000FB60F9211240BB60F922F923F924F9230
:104020005F926F927F928F929F92AF92BF92CF9248
:10403000DF92EF92FF920F931F932F933F934F9333
:104040005F936F937F938F939F93AF93BF93EF9300
:10405000FF93CF93DF93CDB7DEB72B97DEBFCDBFF6
:104060007894209182062983223008F083C1222E81
:10407000312C8101000F111F000F111FF801E85EA4
:10408000F44F80809180A280B380F101EE0FFF1F7A
:10409000EC5EF44FE080F180B7010F2C000C880B30
:1040A000990B0F94CA0AA50194010F94AE0E2B012F
:1040B0003C0120E030E040E252E40F940F11F101A6
:1040C000E058F94FFE83ED8318164CF481E08083AD
:1040D000C12CD12C5FE7E52E53E4F52EDEC020E0A5
:1040E00030E040E251ECC301B2010F94C30A87FDF6
:1040F00002C0EF2841F481E0ED81FE818083C12C74
:10410000D12C7601CAC0ED81FE818081882351F0D7
:10411000F801E858F94F1082118212821382ED8162
:10412000FE8110822091610230916202409163020F
:1041300050916402C301B2010F946A066D837E83BD
:104140008F839887F801E858F94F208131814281A7
:104150005381C301B2010F94AF0EC62E7B878987AE
:10416000792EF801E059F94FD080E180F280638028
:104170002D2D3E2D4F2D562D0F94C30A87FD17C0B0
:10418000F801E859F94FD080E180F28063802D2D4D
:104190003E2D4F2D562D6C2D7B858985972D0F94A7
:1041A0000F11181624F0DC2CEB84F984672C8D2D6C
:1041B0009E2DAF2DB62DF801E858F94F80839183DD
:1041C000A283B38320915D0230915E0240915F0231
:1041D000509160026D2D7E2D8F2D962D0F946A06C5
:1041E0002B013C01F801E05AF94F208131814281D5
:1041F0005381C501B4010F94AE0E20915902309144
:104200005A0240915B0250915C020F946A0620EDC5
:104210003CEC4CE45DE30F946A066B017C0123E304
:1042200033E343E75FE3C801885A994F9A87898748
:10423000FC0160817181828193810F946A069B01E8
:10424000AC01C701B6010F94AF0E6B017C01E9858B
:10425000FA85C082D182E282F382A30192016D814C
:104260007E818F8198850F94AF0EA70196010F94E0
:10427000AE0E6B017C0120E030E0A9010F94C30A6F
:1042800087FD3DCF20E030E04FE753E4C701B601A2
:104290000F940F1118160CF41BCFF801E05AF94FC8
:1042A00080829182A282B3829101220F331F3E83CA
:1042B0002D83F901EC5AF94F60817181072E000CB2
:1042C000880B990B0F94CA0AA50194010F94C30A95
:1042D00081010150194F87FF4AC08D819E81855E03
:1042E0009D4FFC0160817181072E000C880B990B9A
:1042F0000F94CA0AA50194010F940F111816BCF56A
:10430000C701B6010F941B1075956795F80160837E
:1043100089818F5F809382062B960FB6F894DEBF5B
:104320000FBECDBFDF91CF91FF91EF91BF91AF91C4
:104330009F918F917F916F915F914F913F912F91BD
:104340001F910F91FF90EF90DF90CF90BF90AF90B3
:104350009F908F907F906F905F904F903F902F90A5
:104360000F900BBE0F900FBE0F901F901895F80185
:104370001082CECFC090F10AD090F20AE090F30AFA
:10438000F090F40A6091F50A7091F60A072E000C7D
:10439000880B990B0F94CA0AA70196010F94AE0ED1
:1043A0004B015C0120915102309152024091530225
:1043B000509154020F946A062B013C012091500643
:1043C000309151064091520650915306C501B401F7
:1043D0000F94AF0E4B015C0100914C0610914D06FD
:1043E000F0914E06FD8320914F06298398014F2FAF
:1043F00059810F94C30A87FD16C000914806109199
:10440000490630914A063D8380914B068983980185
:104410004D81582FB401C5010F940F1118161CF0CF
:104420008401AD82B982C801AD81B9818093500603
:1044300090935106A0935206B093530620914D02DB
:1044400030914E0240914F0250915002B801CD017F
:104450000F946A0669837A838B839C832091440638
:10446000309145064091460650914706C701B60176
:104470000F94AE0E2091490230914A0240914B02B6
:1044800050914C020F946A0620ED3CEC4CE45DE345
:104490000F946A064B015C0123E333E343E75FE3D8
:1044A00060914006709141068091420690914306CA
:1044B0000F946A069B01AC01C501B4010F94AF0EC5
:1044C0004B015C018092400690924106A092420608
:1044D000B0924306C0924406D0924506E09246064A
:1044E000F092470629813A814B815C81C301B20178
:1044F0000F94AF0EA50194010F94AE0E4B015C0119
:1045000020E030E0A9010F94C30A87FD29C020E014
:1045100030E04FE753E4C501B4010F940F111816B2
:104520001CF120E030E040EA50E4C701B6010F94EE
:104530000F11181604F520E030E846EB53E4C701EC
:10454000B6010F94C30A87FF16C0C501B4010F94CA
:104550001B10759567956093F60610928206DCCE67
:10456000812C912C5401DDCF812C912C9FE7A92E19
:1045700093E4B92ED6CF1092F606EFCFCF93DF9308
:10458000C091FB02D091FC02BE010D2E000C880BE5
:10459000990B0F94CA0A20E030E0A9010F94C30AD6
:1045A00087FD2AC01092170B1092160B1092B10AB9
:1045B0001092B00A1092F60A1092F50A1092150B9A
:1045C0001092140B1092FF0674981092170B109211
:1045D000160B1092000775981092B10A1092B00A4B
:1045E000109201071092F60A1092F50A1092F60640
:1045F000A598DF91CF910895D093170BC093160B18
:10460000D5CF20915D0230915E0240915F025091C2
:10461000600260E070E081E693E40F94A90FE8E6A1
:10462000F6E06083718382839383648375838683DA
:10463000978320914D0230914E0240914F0250914C
:10464000500260E070E081E693E40F94A90F60935C
:1046500048067093490680934A0690934B06089546
:10466000CF93DF93EB019FB78823A1F1F89480915A
:104670000B01806480930B019FBF62E370E080E0D8
:1046800090E00E9468B490E080E0FE01319763EC16
:1046900070E02BEC37E08C179D070CF037C05FB74C
:1046A00083309105E4F4F89440910B014068409305
:1046B0000B015FBFD9011197F1F75FB7F8944091F3
:1046C0000B014F7740930B015FBFD9011197F1F7B1
:1046D0000196E1CFF89480910B018F7BCBCF8E17A1
:1046E0009F070CF7F89440910B01406840930B0131
:1046F0005FBFDB011197F1F75FB7F89440910B01B1
:104700004F7740930B015FBFDB01E0CFDF91CF918B
:1047100008952FB7F89494E0899FF0011124E8518F
:10472000F74E60817181828193812FBF0895CF936D
:10473000DF93C82F0E94892324E0C29FE001112447
:10474000C953DA4F0F94CA0A288139814A815B81A3
:104750000F946A06DF91CF91089580916F008D7F4D
:1047600080936F0080E00E9489230F94CA0A2091F1
:1047700025193091261940912719509128190F9425
:10478000A90F609335197093361980933719909358
:10479000381981E00E9489230F94CA0A20912919AF
:1047A00030912A1940912B1950912C190F94A90F6F
:1047B0006093391970933A1980933B1990933C197F
:1047C00082E00E9489230F94CA0A20912D1930910A
:1047D0002E1940912F19509130190F94A90F609301
:1047E0003D1970933E1980933F199093401983E0CF
:1047F0000E9489230F94CA0A2091311930913219ED
:1048000040913319509134190F94A90F60934119B5
:104810007093421980934319909344194DE359E1E1
:1048200069E379E185E399E10E9427AD94E4209161
:1048300052198091531928131BC01092210B10920A
:10484000200B80910D0090910E00A0910F000A2E78
:10485000000CBB0B8093BB059093BC05A093BD05DA
:10486000B093BE0580916F00826080936F000895C1
:1048700020915219809153192817C9F2E0915319C8
:104880009E9FF0011124E25DF44F128EE0915319C6
:104890009E9FF0011124E25DF44F1586168617865F
:1048A000809153198F5F8F7180935319C0CF1F92DE
:1048B0000F920FB60F9211240BB60F928F929F9208
:1048C000AF92BF92CF92DF92EF92FF920F931F931E
:1048D0002F933F934F935F936F937F938F939F9308
:1048E000AF93BF93CF93DF93EF93FF938091C80073
:1048F00087FF1AC02091CE00809172189091731892
:104900004091741850917518019693704817590783
:1049100059F0E0917218F0917318EE58FB4E208315
:1049200090937318809372188091200B9091210BB3
:10493000892B09F037C1909152198091531998171A
:1049400009F4F6C3E09153194E2F50E004E4E09FC0
:10495000F0011124E25DF44F81E0828FF093210B8E
:10496000E093200B309709F4E3C3DF01AF5BBF4F47
:104970008D919D91AC91B0E08093B30A9093B40A6D
:10498000A093B50AB093B60A80819181A2811816CE
:1049900019061A060CF44EC383819481A58118165A
:1049A00019061A060CF446C386819781A08518164D
:1049B00019061A060CF43EC31092660A1092670A92
:1049C0001092680A1092690A84E4849FF001859F1E
:1049D000F00D1124E25DF44F21E0228F1092BA0510
:1049E0001092B6051092B7051092B8051092B9054D
:1049F00082A993A981341CE9910708F030C3813260
:104A00003EE4930708F42EC396958795969587956F
:104A100024E02093B5058097803D17E0910708F4C6
:104A200032C3E92FFF27EE0FFF1FEE0FFF1F9F017D
:104A30002554394EF9013296C591D491AA278D9FFC
:104A4000B0018C9F610D7A1F06946A1F7A1F112492
:104A5000F90185919491861B970B8C39910510F47F
:104A60008CE990E09093B4058093B3058091B505EF
:104A7000082E000C990B9093B2058093B10584E445
:104A8000849FF001859FF00D1124E25DF44F85A90C
:104A900096A99093B0058093AF0581342CE99207D5
:104AA00008F010C381323EE4930708F40EC39695D4
:104AB00087959695879524E02093B5058097803D4E
:104AC00017E0910708F413C3E92FFF27EE0FFF1F2C
:104AD000EE0FFF1F9F012554394EF9013296C59103
:104AE000D491AA278D9FB0018C9F610D7A1F0694E7
:104AF0006A1F7A1F1124F90185919491861B970BE7
:104B00008C39910510F48CE990E0909389008093A2
:104B100088001092AB051092AC051092AD05109272
:104B2000AE0584E4849FF001859FF00D1124E25DC1
:104B3000F44F85859685A7850A2E000CBB0BB5958D
:104B4000A79597958795B095A095909581959F4F3E
:104B5000AF4FBF4F8093A7059093A805A093A905D9
:104B6000B093AA058093A3059093A405A093A505EF
:104B7000B093A60580939F059093A005A093A105EF
:104B8000B093A20580939B0590939C05A0939D05EF
:104B9000B0939E051092BB051092BC051092BD0506
:104BA0001092BE05E091200BF091210B309709F493
:104BB00063C68091BA0581113BC0808D80939A05B0
:104BC00080FFBDC2119A8FEF8093150280919A05E4
:104BD00081FFB8C244988FEF8093160280919A05A6
:104BE00082FFB3C2419A00000000000000000000F4
:104BF000000000000000000000008FEF809317020B
:104C0000E091200BF091210B818D90919A0593FFFB
:104C1000B0C2813009F0A6C2A198809105018F7BB6
:104C2000809305018FEF8093180281E08093BA058D
:104C300080919905823009F4A8C30CF0ABC2E091D1
:104C4000200BF091210B882309F4D3C2813009F4A1
:104C50001AC38091C80087FF1AC02091CE008091AE
:104C600072189091731840917418509175180196AC
:104C700093704817590759F0E0917218F091731822
:104C8000EE58FB4E2083909373188093721820E0A7
:104C9000E091200BF091210B8091B505082E000CBE
:104CA000990B281719060CF0FFC481859285A385FE
:104CB000B48540919B0550919C0560919D05709134
:104CC0009E05840F951FA61FB71F80939B05909389
:104CD0009C05A0939D05B0939E05181619061A060B
:104CE0001B060CF051C0818D813009F0C7C4729A47
:104CF00080910501806880930501E091200BF0917F
:104D0000210B85859685A7857C010A2F002E000C36
:104D1000110BB801A70180919B0590919C05A09172
:104D20009D05B0919E05841B950BA60BB70B809338
:104D30009B0590939C05A0939D05B0939E05909133
:104D400018024091F4185091F5186091F61870917E
:104D5000F718892F990F990BAA0BBB0B840F951F7E
:104D6000A61FB71F8093F4189093F518A093F61818
:104D7000B093F718818D813009F08BC472988091BF
:104D800005018F7780930501E091200BF091210BB5
:104D900080819181A2810A2E000CBB0B4091A70556
:104DA0005091A8056091A9057091AA05840F951FDF
:104DB000A61FB71F8093A7059093A805A093A905E8
:104DC000B093AA05181619061A061B060CF03FC068
:104DD000139AE091200BF091210B85859685A7858C
:104DE0007C010A2F002E000C110BB801A701809145
:104DF000A7059091A805A091A905B091AA05841BCB
:104E0000950BA60BB70B8093A7059093A805A093CD
:104E1000A905B093AA05909115024091E818509108
:104E2000E9186091EA187091EB18892F990F990B86
:104E3000AA0BBB0B840F951FA61FB71F8093E81802
:104E40009093E918A093EA18B093EB181398E091A7
:104E5000200BF091210B83819481A5810A2E000CF7
:104E6000BB0B4091A3055091A4056091A5057091DD
:104E7000A605840F951FA61FB71F8093A3059093C7
:104E8000A405A093A505B093A605181619061A0641
:104E90001B060CF03FC0459AE091200BF091210BCE
:104EA00085859685A7857C010A2F002E000C110BA5
:104EB000B801A7018091A3059091A405A091A50533
:104EC000B091A605841B950BA60BB70B8093A30589
:104ED0009093A405A093A505B093A6059091160202
:104EE0004091EC185091ED186091EE187091EF1808
:104EF000892F990F990BAA0BBB0B840F951FA61F27
:104F0000B71F8093EC189093ED18A093EE18B09310
:104F1000EF184598E091200BF091210B8681978145
:104F2000A0850A2E000CBB0B40919F055091A00557
:104F30006091A1057091A205840F951FA61FB71F50
:104F400080939F059093A005A093A105B093A2051F
:104F5000181619061A061B060CF03FC0429AE0917B
:104F6000200BF091210B85859685A7857C010A2F62
:104F7000002E000C110BB801A70180919F059091A4
:104F8000A005A091A105B091A205841B950BA60BCD
:104F9000B70B80939F059093A005A093A105B093B4
:104FA000A205909117024091F0185091F11860916C
:104FB000F2187091F318892F990F990BAA0BBB0B5C
:104FC000840F951FA61FB71F8093F0189093F118B8
:104FD000A093F218B093F31842988091BB0590917A
:104FE000BC05A091BD05B091BE050196A11DB11DE6
:104FF0008093BB059093BC05A093BD05B093BE05FF
:105000004091BB055091BC056091BD057091BE05F6
:10501000E091200BF091210B85859685A7850A2EBE
:10502000000CBB0B481759076A077B0708F03CC305
:105030002F5F2ECE84E4849FF001859FF00D112414
:10504000E25DF44F868D978DA0A1B1A18093660A91
:105050009093670AA093680AB093690AB5CC80E47C
:105060009CE9D2CC813107E2900720F09695879594
:1050700022E0CFCC2093B5058032910508F0CBCC4F
:1050800080E290E0C8CC9C01369527952C7F255472
:105090003D4EF90165917491F9013296A591B49153
:1050A000877099278A9F90018B9F300D9A9F300DB2
:1050B000112413E0369527951A95E1F7CB01821B51
:1050C000930BCBCC80E49CE9F2CC813107E29007D2
:1050D00020F09695879522E0EFCC21E02093B5054E
:1050E0008032910508F0EACC80E290E0E7CC9C01A8
:1050F000369527952C7F25543D4EF9016591749185
:10510000F9013296A591B4919C01277033272A9F0B
:10511000C0012B9F900D3A9F900D1124E3E09695CE
:105120008795EA95E1F79B01281B390BC901E8CC6B
:1051300080ED97E0909389008093880033CD11989B
:1051400081E042CD449A81E047CD419800000000C3
:10515000000000000000000000000000000000004F
:1051600081E04CCD5C9880910B018B7F80930B018B
:1051700059CD813041F4A19A8091050180648093DA
:10518000050181E050CD5C9A80910B018460809391
:105190000B01F7CF843009F4E6C1E091200BF091C8
:1051A000210B84300CF459C1853009F052CD109296
:1051B000990590912B0280919A0582FF23C2992331
:1051C00009F447CD2681378140851216130614064F
:1051D0000CF03FCD8091DC0A853009F0F2C122B39A
:1051E000822F817020FDF4C17D99F2C180939805D2
:1051F00030CD81E08093990590912B02992309F499
:1052000028CD2681378140851216130614060CF02E
:1052100020CD9091DC0A953051F592B3292F217061
:1052200090FF2EC090919805992351F14091F0186C
:105230005091F1186091F2187091F3184093940511
:1052400050939505609396057093970580938B0511
:1052500085859685A7850A2E000CBB0B8093BB0520
:105260009093BC05A093BD05B093BE0509C0809185
:105270003002882309F4EDCC21E07D99A3C020E021
:1052800020939805E6CC82E08093990580912B02CB
:1052900090919A0590FF41C0882309F4DACC80816F
:1052A0009181A281181619061A060CF0D2CC8091B1
:1052B000DC0A853079F580B1817049F190918A05D9
:1052C000992329F14091E8185091E9186091EA1862
:1052D0007091EB1840938C0550938D0560938E056B
:1052E00070938F0591E090938905258536854785D4
:1052F0007901042F002E000C110BB801A701409377
:10530000BB055093BC056093BD057093BE058093AB
:105310008A059FCC80910301CFCF882309F499CCD3
:1053200080819181A281181619061A060CF091CC81
:1053300021E0069904C020E0209388058ACC809162
:1053400088058823C9F38091E8189091E918A09105
:10535000EA18B091EB1880938C0590938D05A0937B
:105360008E05B0938F0581E08093890585859685AC
:10537000A7850A2E000CBB0B8093BB059093BC0540
:10538000A093BD05B093BE05D7CF83E08093990568
:1053900080912B02882309F45CCCE091200BF091E2
:1053A000210B86819781A085181619061A060CF024
:1053B00050CC8091DC0A8530E1F482B3282F217033
:1053C00080FF5ECF80919805882309F459CF8091A2
:1053D000F0189091F118A091F218B091F318809301
:1053E000940590939505A0939605B093970581E059
:1053F0002DCF80913002882309F42BCC81E07D9958
:1054000002C080E0F3CE90919805992309F4EECE86
:105410004091F0185091F1186091F2187091F318C2
:105420004093940550939505609396057093970566
:1054300080938B052585368547857901042F002EBD
:10544000000C110BB801A7014093BB055093BC059C
:105450006093BD057093BE05C9CE84E08093990525
:1054600080912B0290919A0591FF45C0882309F401
:10547000F0CB83819481A581181619061A060CF0C9
:10548000E8CB8091DC0A853089F580B18295817006
:10549000882349F190918705992329F14091EC18CF
:1054A0005091ED186091EE187091EF1840939005AF
:1054B00050939105609392057093930591E09093BA
:1054C00086052585368547857901042F002E000C39
:1054D000110BB801A7014093BB055093BC05609325
:1054E000BD057093BE0580938705B3CB8091030102
:1054F00086958170CDCF882309F4ABCB83819481CD
:10550000A581181619061A060CF0A3CB21E0029902
:1055100004C020E0209385059CCB809185058823DD
:10552000C9F38091EC189091ED18A091EE18B0910C
:10553000EF188093900590939105A0939205B093F6
:10554000930581E08093860585859685A7850A2E3B
:10555000000CBB0B8093BB059093BC05A093BD05CD
:10556000B093BE05D7CF85E0809399058091060161
:1055700085FF24C081E08093280B0E94AD23FF911A
:10558000EF91DF91CF91BF91AF919F918F917F91DB
:105590006F915F914F913F912F911F910F91FF90CC
:1055A000EF90DF90CF90BF90AF909F908F900F9033
:1055B0000BBE0F900FBE0F901F9018951092280BE6
:1055C00048CB80913002882309F410CE7D9B19CFFF
:1055D000809198058823A1F04091F0185091F1181E
:1055E0006091F2187091F3184093940550939505CB
:1055F000609396057093970591E090938B051ACF71
:10560000892FF4CD992309F424CB86819781A08535
:10561000181619061A060CF01CCB80B1881F8827B3
:10562000881F49F190918405992329F14091F01840
:105630005091F1186091F2187091F318409394050D
:1056400050939505609396057093970591E090931C
:105650008B052585368547857901042F002E000CA2
:10566000110BB801A7014093BB055093BC05609393
:10567000BD057093BE0580938405EBCA809102013D
:1056800080688093020180910B01816080930B01FF
:1056900034CB809102018F778093020180910B01BE
:1056A0008E7F80930B0170CBE091200BF091210B4A
:1056B0004091BB055091BC056091BD057091BE0540
:1056C00080899189B0E0A0E084179507A607B70705
:1056D00008F42DC10091AB051091AC052091AD05EA
:1056E0003091AE0585899689A789AC016A2F70E053
:1056F000AA27059FB12D169F6001269FD00C259FDC
:10570000C00CD11C069FB00DC11CDA1E159FB00D38
:10571000C11CDA1E249FB00DC11CDA1E149FB10DEE
:10572000CA1EDA1EB695CA1EDA1E1124D092B00522
:10573000C092AF0582A993A9A4A9860130E020E018
:10574000AC016A2F70E0401751076207730708F039
:10575000B3C09093B0058093AF058091AF05909151
:10576000B00581340CE9900708F0ABC081321EE42B
:10577000910708F4A9C0969587959695879524E09A
:105780002093B5058097803D37E0930708F4AEC0BD
:10579000E92FFF27EE0FFF1FEE0FFF1F9F0125547C
:1057A000394EF901329665917491AA27879FA0011D
:1057B000869F410D5A1F06944A1F5A1F1124F90152
:1057C00085919491841B950B8C39910510F48CE98B
:1057D00090E090938900809388004091AB055091B0
:1057E000AC056091AD057091AE05480F591F611D64
:1057F000711D4093AB055093AC056093AD0570935C
:10580000AE054091BB055091BC056091BD057091FE
:10581000BE05E091200BF091210B85859685A7852B
:105820000A2E000CBB0B481759076A077B0720F1AB
:105830001092210B1092200B9091521980915319C4
:105840009817D1F0A0915319E4E4EA9FD0011124F4
:10585000A25DB44F5A961C9280915319E89FF001B3
:105860001124E25DF44F1586168617868091531930
:105870008F5F8F71809353198091C80087FF7FCE0F
:105880002091CE00809172189091731840917418F5
:1058900050917518019693704817590709F46FCE07
:1058A000E0917218F0917318EE58FB4E208390939C
:1058B00073188093721863CE85A996A98C0D9D1DCF
:1058C00048CF80E49CE957CF813127E2920720F04E
:1058D0009695879522E054CF21E02093B50580323C
:1058E000910508F04FCF80E290E04CCF9C013695B7
:1058F00027952C7F25543D4EF90145915491F9018E
:105900003296659174919C0127703327269FC001C0
:10591000279F900D369F900D112403E09695879553
:105920000A95E1F77A01E81AF90AC7014DCF4091CB
:10593000BB055091BC056091BD057091BE05828983
:105940009389A489B0E084179507A607B70708F0E4
:10595000C6C04091B6055091B7056091B8057091E9
:10596000B90585899689A7898C012A2F30E0AA2755
:10597000419FB12D529FE001629FD00D619FC00DEC
:10598000D11D429FB00DC11DDA1F519FB00DC11D29
:10599000DA1F609FB00DC11DDA1F509FB10DCA1FE5
:1059A000DA1FB695CA1FDA1F11248091AF059091B6
:1059B000B005C0ACD1ACE2AC8C179D0708F056C066
:1059C000C6018C0130E020E04601AE2CB12C081558
:1059D00019052A053B0508F4C60181340CE9900736
:1059E00008F047C081321EE4910708F445C096953F
:1059F00087959695879524E02093B5058097803DFF
:105A000037E0930708F44AC0E92FFF27EE0FFF1F86
:105A1000EE0FFF1F9F012554394EF9013296059173
:105A20001491AA27819FE001809FC10DDA1F06947F
:105A3000CA1FDA1F1124F901859194918C1B9D0BCB
:105A40008C39910510F48CE990E090938900809353
:105A50008800480F591F611D711D4093B605509372
:105A6000B7056093B8057093B905CBCE8C1B9D0B21
:105A7000A8CF80E49CE9BBCF813127E2920720F0D8
:105A80009695879522E0B8CF21E02093B505803226
:105A9000910508F0B3CF80E290E0B0CF9C0136953D
:105AA00027952C7F25543D4EF901A591B491F9011C
:105AB0003296C591D4919C01277033272C9FC00149
:105AC0002D9F900D3C9F900D1124F3E096958795A6
:105AD000FA95E1F77D01E81AF90AC701B1CF809183
:105AE000B3059091B40590938900809388008091CC
:105AF000B1058093B50585CE109289051092860573
:105B000010928B050895FC01249121110BC0FB011B
:105B10008191882379F09091C80095FFFCCF809304
:105B2000CE00F6CF3091C80035FFFCCF2093CE00D9
:105B30000196E9CF08958F929F92AF92BF92EF9214
:105B4000FF920F931F93CF93DF93CDE4DAE085E2CA
:105B5000E82E89E1F82E0CE71AE069917991899194
:105B60009991F70181909190A190B1907F010F944C
:105B7000C80AA50194010F946A060F942210F80137
:105B800061937193819391938F01FAE0CD35DF0793
:105B900021F7DF91CF911F910F91FF90EF90BF9070
:105BA000AF909F908F9008958091521990915319C2
:105BB000891B8F71089520913119309132194091CC
:105BC000331950913419FC01608171818281938174
:105BD0000F946A06E091141924E0E29FF001112469
:105BE000E45FF64E20813181428153810F946A0631
:105BF0000F94C311E5E1F9E164877587868797877C
:105C00008FB7F89444855585668577854093F41859
:105C10005093F5186093F6187093F7188FBF089596
:105C2000CF92DF92EF92FF92CF93DF93EC01089631
:105C30000E94D8196B017C018091B20A8823E1F09F
:105C400020E030E0A901C701B6010F94C30A882300
:105C500099F0CE010E94D91DA70196010F946A0602
:105C60009B01AC01688579858A859B850F94AE0E72
:105C7000688779878A879B87DF91CF91FF90EF9024
:105C8000DF90CF9008958F929F92AF92BF92CF9264
:105C9000DF92EF92FF920F931F93CF93DF93CDB7D5
:105CA000DEB72C970FB6F894DEBF0FBECDBF2091A4
:105CB000B20A2223D9F18A017B016C01CA010E9438
:105CC000D8194B015C0120E030E0A9010F94C30A10
:105CD000882361F119861A861B861C86F60180814D
:105CE0009181A281B38189839A83AB83BC83F701BD
:105CF00080819181A281B3818D839E83AF83B88798
:105D0000CE0101960E94D91DA50194010F946A0647
:105D10009B01AC01F80160817181828193810F94B4
:105D2000AF0EF80160837183828393832C960FB644
:105D3000F894DEBF0FBECDBFDF91CF911F910F91C1
:105D4000FF90EF90DF90CF90BF90AF909F908F909B
:105D500008954F925F926F927F928F929F92AF922F
:105D6000BF92CF92DF92EF92FF92CF93DF93CDB7A6
:105D7000DEB760970FB6F894DEBF0FBECDBF0E94AE
:105D80009AB42B013C0180915B0590915C05A09138
:105D90005D05B0915E0584159505A605B70508F06B
:105DA00018C1805A9541AF4FBF4F80935B059093C8
:105DB0005C05A0935D05B0935E058091730590919D
:105DC0007405A0917505B09176050196A11DB11DD0
:105DD0008093730590937405A0937505B093760531
:105DE0008091670590916805A0916905B0916A0559
:105DF0000196A11DB11D8093670590936805A0933E
:105E00006905B0936A0580915A05882309F4E1C0B9
:105E100080916F0590917005A0917105B091720508
:105E20000196A11DB11D80936F0590937005A093FD
:105E30007105B09372058091630590916405A091FE
:105E40006505B09166050196A11DB11D809363059E
:105E500090936405A0936505B09366052091411960
:105E600030914219409143195091441929833A8342
:105E70004B835C832091560530915705409158051E
:105E80005091590569817A818B819C810F94AE0E66
:105E90006B017C0120E030E0A9010F940F1118166E
:105EA0000CF08BC020E030E041EE54E4C701B601B5
:105EB0000F94C30A87FF81C0E091141934E0E39F77
:105EC000F0011124E45FF64E20813181428153813B
:105ED000C701B6010F946A0620915205309153050F
:105EE00040915405509155050F94AF0E4B015C0144
:105EF00080916B0590916C05A0916D05B0916E0538
:105F0000C0905F05D0906005E0906105F09062055B
:105F10009C01AD012C193D094E095F092D873E8773
:105F20004F87588B8D859E85AF85B8898C0D9D1DBB
:105F3000AE1DBF1D89879A87AB87BC87A7019601D5
:105F40002F5F3F4F4F4F5F4F2D833E834F835887C7
:105F500020E030E040E251E4C501B4010F940F119C
:105F600018167CF420E030E040E251E4C501B401B1
:105F70000F94AE0E4B015C01CD80DE80EF80F88483
:105F8000D1CF89859A85AB85BC8580936B0590932D
:105F90006C05A0936D05B0936E05C0925F05D0921D
:105FA0006005E0926105F092620580925205909240
:105FB0005305A0925405B092550529813A814B8131
:105FC0005C812093560530935705409358055093B4
:105FD000590580914E0590914F05A0915005B091C3
:105FE000510584159505A605B70520F5D301C20115
:105FF00080589141A94CBF4F80934E0590934F0517
:10600000A0935005B093510560960FB6F894DEBF8B
:106010000FBECDBFDF91CF91FF90EF90DF90CF907B
:10602000BF90AF909F908F907F906F905F904F90B8
:106030000C94891D60960FB6F894DEBF0FBECDBFDD
:10604000DF91CF91FF90EF90DF90CF90BF90AF9016
:106050009F908F907F906F905F904F9008950E94D7
:106060009AB46093CE0A7093CF0A8093D00A90932B
:10607000D10A8091AE13807C803469F0E3EAFDE0C0
:106080008491882371F19091C80095FFFCCF809393
:10609000CE003196F5CF8091EE0A882379F3E0EABD
:1060A000FDE0849181110DC0EEE9FDE0849188232B
:1060B00081F09091C80095FFFCCF8093CE0031967F
:1060C000F5CF9091C80095FFFCCF8093CE0031961C
:1060D000E8CF8091C80085FFFCCF8AE08093CE0096
:1060E00008958091C80085FFFCCFF7CFFC01659132
:1060F00075918591949108950F931F93CF93DF939A
:10610000EC01CC0FDD1FCC0FDD1FCE018253984F69
:106110000E9476308E010B5C164EFE01ED53FD4F52
:1061200020813181428153810F94AE0EF80160834A
:10613000718382839383CE018E53984F0E94763071
:10614000FE01E158FD4F6083718382839383CE010A
:106150008A54984F0E947630C75CDD4F68837983FC
:106160008A839B83DF91CF911F910F910895682FB0
:10617000880F770B9091EC0A2AE4929FC0011124BA
:106180008751984F0F947C129C019093DB0A809367
:10619000DA0A81E0232B09F480E008958091DA0A7D
:1061A0009091DB0A4AE050E070E060E001960D94C7
:1061B0002A098091DA0A9091DB0A70E060E001968A
:1061C0000D94CC071F93CF93DF93EC0180911419AA
:1061D0008093BD0A84E50E94B730182F811106C054
:1061E00010E0812FDF91CF911F9108950E94D93047
:1061F0000F9422106093BD0A623090F3E3ECFDE24D
:106200008491882341F09091C80095FFFCCF809342
:10621000CE003196F5CFC936D10599F1A4F4E4ED5D
:10622000F3E0C836D105C9F16091BD0A70E090E095
:1062300080E00E94EC1A8091C80085FFFCCF8AE0C4
:106240008093CE00CECFCD36D10579F0EFE8F3E0E4
:10625000CA3DD10549F78191882331F39091C80057
:1062600095FFFCCF8093CE00F6CFE6EAF3E0819174
:106270008823D1F29091C80095FFFCCF8093CE0087
:10628000F6CFEDEBF3E08191882371F29091C80095
:1062900095FFFCCF8093CE00F6CF8191882321F229
:1062A0009091C80095FFFCCF8093CE00F6CF0F935E
:1062B0001F93CF93DF93CDB7DEB72C970FB6F8942B
:1062C000DEBF0FBECDBF80916E1485FF06C067E7AD
:1062D00074E08EE894E00E94D6AD80913D199091D3
:1062E0003E19A0913F19B091401940913919509130
:1062F0003A1960913B1970913C1900913519109130
:106300003619209137193091381909831A832B8354
:106310003C834D835E836F83788789879A87AB87B9
:10632000BC87AE01475F5F4FBE016B5F7F4FCE0101
:1063300001960E94432EAE01475F5F4FBE016B5F27
:106340007F4FCE0101960E9427AD2C960FB6F89490
:10635000DEBF0FBECDBFDF91CF911F910F9108958A
:106360001F93CF93DF93CDB7DEB72C970FB6F8947A
:10637000DEBF0FBECDBF882331F02091E5073091FD
:10638000E607232BD1F09091B20A9817B1F0182F9D
:106390008CE0EBE0F3E0DE01119601900D928A951E
:1063A000E1F7CE0101960E94D91D1093B20A111196
:1063B0000EC00E94FCAC0E9457312C960FB6F89488
:1063C000DEBF0FBECDBFDF91CF911F91089585E352
:1063D00099E10E94102EEFCF80916E1485FF14C0BA
:1063E000EEE4F8E08491882341F09091C80095FF95
:1063F000FCCF8093CE003196F5CF8091C80085FF09
:10640000FCCF8AE08093CE0080E00E94B0311092F1
:10641000E8071092E7071092E6071092E50710923E
:10642000390510923805109237051092360529E388
:1064300037E087E040E050E060EC7FE7F90196E06C
:1064400041935193619371939150D1F78150285E9C
:106450003F4F8111F3CF08958091AF13882381F0CE
:106460001092EC0A1092AB041092AF13E9EEF7E031
:1064700080E592E0DF019C011D9221503040E1F760
:106480000895CF92DF92EF92FF926A017B01FC01A7
:106490002491222341F03091C80035FFFCCF209396
:1064A000CE000196F4CF42E0C701B601FF90EF9015
:1064B000DF90CF900C947DAC4F925F926F927F9261
:1064C000AF92BF92CF92DF92EF92FF920F931F9302
:1064D000CF93DF9300D000D0CDB7DEB77E836D833E
:1064E00029833A834B835C8327013801FC01249183
:1064F000222341F03091C80035FFFCCF2093CE001D
:106500000196F4CF8091C80085FFFCCF88E280938C
:10651000CE0042E069817A818B819C810E947DACB2
:10652000B301A20184E794E00E944132B601A501C3
:1065300081E794E00E9441328091C80085FFFCCF42
:1065400089E28093CE008D819E81009761F0FC01ED
:106550008491882379F09091C80095FFFCCF8093B7
:10656000CE003196F5CF8091C80085FFFCCF8AE040
:106570008093CE0026960FB6F894DEBF0FBECDBF37
:10658000DF91CF911F910F91FF90EF90DF90CF900F
:10659000BF90AF907F906F905F904F9008959091D3
:1065A000D00095FFFCCF8093D6000895A39A80EC8D
:1065B0000E94CF3288E00E94CF3281E00E94CF3229
:1065C00082E00E94CF3280E00E94CF3280E00E94C1
:1065D000CF3283EF0E94CF3283E20E94CF3281E03C
:1065E0000C94CF32CF93DF93A39A80EC0E94CF32EA
:1065F00088E00E94CF3281E00E94CF3281E00E9489
:10660000CF3280E00E94CF3280E00E94CF328CE116
:106610000E94CF3287E40E94CF3281E00E94CF32C5
:10662000C5EFD1E0219759F08091DD0A893838F023
:1066300061E070E080E090E00E9468B4F3CFDF9109
:10664000CF9108954F925F926F927F928F929F9217
:10665000AF92BF92EF92FF920F931F93CF93DF936E
:10666000CDB7DEB7A4970FB6F894DEBF0FBECDBF8F
:106670004115510561057105E1F48091C80085FF60
:10668000FCCF80E38093CE00A4960FB6F894DEBFD3
:106690000FBECDBFDF91CF911F910F91FF90EF9073
:1066A000BF90AF909F908F907F906F905F904F9032
:1066B00008958E010F5F1F4F812C912C540178019A
:1066C000422E512C712C612CCB01BA01A3019201F5
:1066D0000F941B0EF42FE52FD501C4010196A11DC7
:1066E000B11D89A39AA3ABA3BCA3D8016D938D015F
:1066F000A9016F2F7E2F4115510561057105C9F460
:10670000F701E80DF91D80818A30C0F4805D909119
:10671000C80095FFFCCF8093CE00B1E08B1A9108A2
:10672000A108B1088FEF88169806A806B80641F7A9
:10673000ABCF89A09AA0ABA0BCA0C6CF895CE7CFA5
:10674000FC012491222341F03091C80035FFFCCF99
:106750002093CE000196F4CF2AE085E499E10C94D1
:106760002233CF93DF93EC010E94BE228091D60AA0
:106770009091D70A892B09F095C01092FC06809160
:10678000380780934C05D093D70AC093D60A83E08C
:1067900080933807E091531984E4E89FF0011124B5
:1067A000E159F44F80819181A281B0E08093340758
:1067B00090933507A0933607B0933707EFEDFEE0CF
:1067C0002A9768F0E6EEFEE08491882399F0909194
:1067D000C80095FFFCCF8093CE003196F5CF849111
:1067E000882341F09091C80095FFFCCF8093CE00A4
:1067F0003196F5CF4091D60A5091D70A70E060E00B
:106800002AE085E499E10E9422338091C80085FF47
:10681000FCCF8AE08093CE008091200B9091210BD9
:10682000009709F042C0809153198150990B8F71E4
:10683000992724E4289FF001299FF00D1124E159A4
:10684000F44F80819181A281AC016A2F70E08AEDC2
:106850009EE00E94A0338091C80085FFFCCF8AE0B3
:106860008093CE001092D20A1092D30A1092D40ACA
:106870001092D50A9FB7F8948091050180628093A9
:1068800005019FBF9FB7F894809105018F7E80938B
:1068900005019FBF9FB7F89480910501877F809382
:1068A00005019FBFDF91CF9108958F5B9F4FFC0142
:1068B00080819181A281AC016A2F70E085ED9EE01C
:1068C0000E94A0338091C80085FFFCCFC8CF2091E3
:1068D0004B052817190609F457C0209138072111D4
:1068E00053C02091220B20934B0510924C0590939E
:1068F000230B8093220B21E020933807E3EBFEE08B
:106900000A9768F0EAEBFEE08491882399F0909171
:10691000C80095FFFCCF8093CE003196F5CF8491CF
:10692000882341F09091C80095FFFCCF8093CE0062
:106930003196F5CF4091220B5091230B70E060E02F
:106940002AE085E499E10E9422338091C80085FF06
:10695000FCCF8AE08093CE009FB7F8948091050128
:106960008F7D809305019FBF9FB7F89480910501AB
:106970008F7E809305019FBF9FB7F894809105019A
:106980008860809305019FBF08951F920F920FB6F4
:106990000F9211240BB60F92EF92FF920F931F9359
:1069A0002F933F934F935F936F937F938F939F9317
:1069B000AF93BF93CF93DF93EF93FF93789480913E
:1069C000090181FD07C08091F906882319F081E053
:1069D0008093260B80910901869581708093F9063A
:1069E0008091141981116FC180918B0681110DC0A6
:1069F0000E949AB4609387067093880680938906F4
:106A000090938A0681E080938B06C3B1C170809118
:106A1000860681110FC1CC23F9F0E091200BF09193
:106A2000210B30990FC180915E0A90915F0AA0916D
:106A3000600AB091610A0196A11DB11D80935E0AA2
:106A400090935F0AA093600AB093610A808D83FDE2
:106A500003C081E080938506C093860680915E0A1C
:106A600090915F0AA091600AB091610A8F3F9F4F99
:106A7000AF4FBF4761F080915E0A90915F0AA0918D
:106A8000600AB091610A0097A105B04881F41092A4
:106A90005E0A10925F0A1092600A1092610A1092C8
:106AA0002707109228071092290710922A070E94A0
:106AB0009AB400918706109188062091890630913A
:106AC0008A06601B710B820B930B6133754781053E
:106AD000910508F10E949AB4609387067093880626
:106AE0008093890690938A061092830620918406EB
:106AF0008091F0023091F102932F917028171906BE
:106B000041F03CF08091AE13803419F481E0809321
:106B1000120B1092840680912602811131C080915F
:106B2000FF068093F8068111749A80910007809384
:106B3000F7068111759A8091F6068093F50681110A
:106B4000A59AE1EFF6E0ADEEB6E090E080E02191AD
:106B50002D93222389F08230910509F4A2C183305C
:106B6000910509F4A2C18130910509F494C12091E5
:106B7000020128602093020101968430910539F7C3
:106B80009091F80680912602891708F074989091E8
:106B9000F70680912602891708F075989091F506FE
:106BA00080912602891708F0A598EDEEF6E090E0B6
:106BB00080E0319120912602231788F082309105E0
:106BC00009F47DC18330910509F47DC181309105BF
:106BD00009F46FC120910201277F209302010196E1
:106BE0008430910531F7809126028F5F8F778093F3
:106BF0002602E0912502E23108F077C1F0E0882713
:106C0000EB5FF94C8F4F0D94920E6737E238FC38EA
:106C10000939233930394A39573971397D3997392A
:106C2000A439C339C539C739D339ED39F939109287
:106C3000850612CF189910CFE091200BF091210B0F
:106C40003099F1CE80915E0A90915F0AA091600A1E
:106C5000B091610A0197A109B10980935E0A9093EE
:106C60005F0AA093600AB093610A81859285A3852B
:106C7000B485892B8A2B8B2B09F4EECE808D83FD76
:106C8000D6CF8091840691E0980F909384069091DE
:106C90008506911106C091E09093850689508093F6
:106CA0008406809183068111D7CE81E0809383068C
:106CB0000E949AB460938706709388068093890631
:106CC00090938A06C9CE80919B0681110DC00E94C7
:106CD0009AB4609397067093980680939906909360
:106CE0009A0681E080939B0689B1C1E0982F90724B
:106CF00085FFC0E080919606811184C09923F9F048
:106D0000E091200BF091210B679984C08091620A79
:106D10009091630AA091640AB091650A0196A11D41
:106D2000B11D8093620A9093630AA093640AB093A2
:106D3000650A808D83FD03C081E080939506C09332
:106D400096068091620A9091630AA091640AB091BC
:106D5000650A8F3F9F4FAF4FBF4761F08091620A36
:106D60009091630AA091640AB091650A0097A10509
:106D7000B04881F41092620A1092630A1092640A79
:106D80001092650A10922B0710922C0710922D0773
:106D900010922E070E949AB40091970610919806BF
:106DA0002091990630919A06601B710B820B930B10
:106DB000613375478105910508F4ADCE0E949AB400
:106DC00060939706709398068093990690939A061D
:106DD00010929306209194068091F0023091F10276
:106DE000932F9170281719063CF08091AE138034D0
:106DF00019F481E08093130B109294068CCE1092BC
:106E000095069DCF4D999BCFE091200BF091210BE2
:106E100067997CCF8091620A9091630AA091640A7D
:106E2000B091650A0197A109B1098093620A909314
:106E3000630AA093640AB093650A81859285A3854D
:106E4000B485892B8A2B8B2B09F479CF808D83FD18
:106E5000D6CF8091940691E0980F909394069091EC
:106E60009506911106C091E0909395068950809304
:106E7000940680919306811162CF81E080939306FE
:106E80000E949AB46093970670939806809399062F
:106E900090939A0654CF20910B01206220930B010E
:106EA0006BCE20910B012061F9CF20910B0128605E
:106EB000F5CF20910B012F7D20930B0190CE2091D7
:106EC0000B012F7EF9CF20910B01277FF5CF88E0B2
:106ED00080937B0081E480937C0080917A008064C1
:106EE00080937A0081E0809325028091BF068031F3
:106EF00008F44FC18091FE061091FA06C12FD0E030
:106F00009E01220F331F811131C08091E9069091BB
:106F1000EA069093BC068093BB068091DD069091B3
:106F2000DE069093BE068093BD068091E5069091A3
:106F3000E6069093BA068093B9068091E106909197
:106F4000E2069093B8068093B7068091C4069091AC
:106F5000C5069093B6068093B5068091C0069091C1
:106F6000C106F901E355F94F918380834091D90619
:106F70005091DA0667E0649FC001659F900D11246F
:106F8000883DE9E59E070CF054C28091A9069091D6
:106F9000AA06A091AB06B091AC060196A11DB11D49
:106FA0008093A9069093AA06A093AB06B093AC0673
:106FB0008091A9069091AA06A091AB06B091AC066B
:106FC0000497A105B10518F081E08093ED0AC9018D
:106FD0008459954F7C01CC0FDD1FCC0FDD1FC753AB
:106FE000D94F688179818A819B810F94C80A26EFE5
:106FF00038E24CE95EE30F946A069B01AC010F9402
:10700000AF0E24EA30E74DE75FE30F946A060F9472
:107010001B10F70171836083188219821A821B8208
:107020001F5F143008F014C21093FA068091FA061C
:10703000813009F413C208F40EC2823009F411C27F
:10704000833009F411C281E08093FE061092BF06DE
:107050001092E9061092EA061092EB061092EC06E6
:107060001092DD061092DE061092DF061092E00606
:107070001092E5061092E6061092E7061092E806D6
:107080001092D9061092DA061092DB061092DC06F6
:107090001092E1061092E2061092E3061092E406C6
:1070A0001092C4061092C5061092C6061092C7062A
:1070B0001092C0061092C1061092C2061092C3062A
:1070C0002091BB063091BC068091A8064091210218
:1070D00050912202241735070CF4C8C120383C43D4
:1070E0000CF0C7C18F5F8093A806853630F00E94F0
:1070F000BE2281E090E00E94B1332091BD06309124
:10710000BE068091A70640912302509124022417C5
:1071100035070CF4BEC120383C430CF0BDC18F5F75
:107120008093A706853630F00E94BE2282E090E070
:107130000E94B1332091B9063091BA068091A4061D
:107140004091A5065091A606421753070CF4B4C10E
:107150008F5F8093A406853620F083E090E00E9444
:10716000B1332091B7063091B8068091A3064091C3
:107170001F0250912002241735070CF4B2C18F5F13
:107180008093A306853628F0A59884E090E00E94BD
:10719000B133FF91EF91DF91CF91BF91AF919F916B
:1071A0008F917F916F915F914F913F912F911F919F
:1071B0000F91FF90EF900F900BBE0F900FBE0F90AE
:1071C0001F90189520917800309179008091E90600
:1071D0009091EA06A091EB06B091EC06820F931F06
:1071E000A11DB11D8093E9069093EA06A093EB06DA
:1071F000B093EC0682E077CE88E080937B0084E455
:1072000080937C0080917A00806480937A0083E090
:107210006ACE20917800309179008091E5069091B6
:10722000E606A091E706B091E806820F931FA11D24
:10723000B11D8093E5069093E606A093E706B09310
:10724000E80684E050CE88E080937B0083E480935E
:107250007C0080917A00806480937A0085E043CE40
:1072600020917800309179008091E1069091E206BA
:10727000A091E306B091E406820F931FA11DB11DFA
:107280008093E1069093E206A093E306B093E406B0
:1072900086E029CE88E080937B0082E480937C00A6
:1072A00080917A00806480937A0087E01CCE2091E0
:1072B0007800309179008091DD069091DE06A091F2
:1072C000DF06B091E006820F931FA11DB11D8093D0
:1072D000DD069093DE06A093DF06B093E00688E01B
:1072E00002CE10927B0084E480937C0080917A002F
:1072F000806480937A0089E0F6CD20917800309107
:1073000079008091D9069091DA06A091DB06B091C0
:10731000DC06820F931FA11DB11D8093D9069093A7
:10732000DA06A093DB06B093DC068AE0DCCD88E0C9
:1073300080937B0086E480937C0080917A00806457
:1073400080937A008BE0CFCD209178003091790046
:10735000E091FA0684E0E89FF0011124E753F94F29
:1073600080819181A281B381820F931FA11DB11DE4
:1073700080839183A283B3838091C8068F5F8093BB
:10738000C8068CE0B0CD8DE0AECD8EE0ACCD1092D5
:107390007B0087E480937C0080917A0080648093F6
:1073A0007A008FE0A0CD2091780030917900809113
:1073B000C4069091C506A091C606B091C706820F7B
:1073C000931FA11DB11D8093C4069093C506A09381
:1073D000C606B093C70680E186CD10927B0083E499
:1073E00080937C0080917A00806480937A0081E1B0
:1073F0007ACD20917800309179008091C0069091EB
:10740000C106A091C206B091C306820F931FA11DB1
:10741000B11D8093C0069093C106A093C206B0939D
:10742000C3068091BF068F5F8093BF06109225022E
:107430005CCD813C9D450CF4BBCD1092A906109209
:10744000AA061092AB061092AC061092ED0AB0CDCF
:107450001092FA06EBCD0E941C17F5CD899A8A98F6
:10746000F2CD89988A9AEFCD899AFCCF20383C4397
:107470004CF08F5F8093A806853608F43ECE86E0F8
:1074800090E039CE882309F438CE81508093A80645
:1074900034CE20383C434CF08F5F8093A70685366E
:1074A00008F448CE87E090E043CE882309F442CE2A
:1074B00081508093A7063ECE26313F435CF08F5F1C
:1074C0008093A406853608F44CCE83E090E00E94B9
:1074D000673447CE882309F444CE81508093A406B4
:1074E00040CE1216130654F08F5F8093A3068536A4
:1074F00008F44FCEA59889E090E049CE882309F49E
:1075000048CE81508093A30644CE77FF0EC02091D1
:10751000C80025FFFCCF2DE22093CE00709560952A
:10752000509541955F4F6F4F7F4F2AE00C94223367
:10753000FC012491222341F03091C80035FFFCCF9B
:107540002093CE000196F4CF83E895E00C94853A21
:107550008091FD0681113EC180916F008D7F8093E7
:107560006F0082E00E9489230F94CA0A2091CF0500
:107570003091D0054091D1055091D2050F946A0603
:1075800060933D1970933E1980933F199093401971
:107590006093C3057093C4058093C5059093C60599
:1075A00083E00E9489230F94CA0A2091D305309169
:1075B000D4054091D5055091D6050F946A06609385
:1075C0004119709342198093431990934419609321
:1075D000BF057093C0058093C1059093C20580E0FC
:1075E0000E9489230F94CA0A2091251930912619E7
:1075F00040912719509128190F94A90F60933519BC
:1076000070933619809337199093381981E00E944E
:1076100089230F94CA0A2091291930912A1940917F
:107620002B1950912C190F94A90F6093391970934D
:107630003A1980933B1990933C194DE359E169E362
:1076400079E185E399E10E9427AD4091411950917C
:10765000421960914319709144198EE49BE10E9494
:1076600041328091C80085FFFCCF8AE08093CE0034
:107670004091351950913619609137197091381928
:1076800089E29BE10E9441328091C80085FFFCCFD6
:107690008AE08093CE004091391950913A19609157
:1076A0003B1970913C1984E09BE10E94413280912A
:1076B000C80085FFFCCF8AE08093CE0040913D1941
:1076C00050913E1960913F19709140198FED9AE1E8
:1076D0000E9441328091C80085FFFCCF8AE08093F0
:1076E000CE008091200B9091210B009709F04FC0A4
:1076F000E091531984E4E89FF0011124E159F44F1B
:1077000080819181A281B0E00197A109B1098093A4
:10771000340790933507A0933607B093370740910D
:1077200034075091350760913607709137078AEC1E
:107730009AE10E94983A8091C80085FFFCCF8AE0C8
:107740008093CE0094E4209152198091531928130C
:1077500022C01092210B1092200B80910D0090916D
:107760000E00A0910F000A2E000CBB0B8093BB05EE
:107770009093BC05A093BD05B093BE0580916F00AA
:10778000826080936F0081E08093FD0608958F5B97
:107790009F4FFC01B5CF20915219809153192817A2
:1077A00091F2E09153199E9FF0011124E25DF44F94
:1077B000128EE09153199E9FF0011124E25DF44F67
:1077C000158616861786809153198F5F8F71809367
:1077D0005319B9CF089580918905882391F0E5EB7D
:1077E000F2E18491811116C0E6EAF2E184918823E6
:1077F000C9F09091C80095FFFCCF8093CE003196E0
:10780000F5CF809186058111EACF80918B0581119A
:10781000E6CF08959091C80095FFFCCF8093CE00ED
:107820003196DFCF809189058823D1F060918C0556
:1078300070918D0580918E0590918F050F94CA0AE5
:107840002091251930912619409127195091281916
:107850000F94A90FAB01BC0182EA92E10E94413270
:10786000809186058823D1F06091900570919105F3
:1078700080919205909193050F94CA0A209129193D
:1078800030912A1940912B1950912C190F94A90F5E
:10789000AB01BC018EE992E10E94413280918B05DF
:1078A0008823D1F06091940570919505809196059B
:1078B000909197050F94CA0A20912D1930912E1995
:1078C00040912F19509130190F94A90FAB01BC01B1
:1078D0008AE992E10E9441328091C80085FFFCCF85
:1078E0008AE08093CE0080918905882331F00E9440
:1078F000AD2380E290E00E94B13380918605882319
:1079000031F00E94AD2381E290E00E94B13380917A
:107910008B05882321F00E94A83A0E942C321092F5
:1079200089051092860510928B050895CF93DF93F9
:1079300020914B052817190609F4A2C02091380799
:10794000223008F09DC03091220B30934B052093DC
:107950004C059093230B8093220B82E08093380791
:10796000EFECFEE08491882341F09091C80095FFF0
:10797000FCCF8093CE003196F5CF4091220B5091F1
:10798000230B70E060E02AE085E499E10E94223355
:107990008091C80085FFFCCF8AE08093CE00809163
:1079A000FD06811182C080912A0B90912B0BA09132
:1079B0002C0BB0912D0B8093340790933507A09337
:1079C0003607B09337078091200B9091210B0097D9
:1079D00009F059C0809153198150990B8F719927E3
:1079E00024E4289FF001299FF00D1124E159F44F60
:1079F00080819181A281AC016A2F70E08AEC9EE0C7
:107A00000E94A0338091C80085FFFCCF8AE080935C
:107A1000CE008091AE138F738230D1F4C091FB02FF
:107A2000D091FC02BE010D2E000C880B990B0F9417
:107A3000CA0A20E030E0A9010F94C30A87FD46C0BE
:107A40001092150B1092140B1092170B1092160B2C
:107A50009FB7F894809105018F7D809305019FBFAA
:107A60009FB7F894809105018061809305019FBFC5
:107A70009FB7F89480910501877F809305019FBF90
:107A8000DF91CF9108958F5B9F4FFC0180819181A1
:107A9000A281AC016A2F70E085EC9EE00E94A033C9
:107AA0008091C80085FFFCCFB1CF40913407509141
:107AB0003507609136077091370780EC9EE00E9491
:107AC000983A8091C80085FFFCCFA0CFD093150BCA
:107AD000C093140BD093170BC093160BB9CFFC01B6
:107AE0002491222341F03091C80035FFFCCF209330
:107AF000CE000196F4CFAB01770F660B770B83E8CE
:107B000095E00C94853A60914C0580913807861772
:107B100009F45AC080914B0590E09093230B809319
:107B2000220B8091FC0690E09093D70A8093D60AAE
:107B30006093380770E08EEE9EE00E946F3D80916A
:107B4000220B9091230B0A9768F4ECEEFEE08491EF
:107B5000882341F09091C80095FFFCCF8093CE0020
:107B60003196F5CF4091220B5091230B70E060E0ED
:107B70002AE085E499E10E9422338091C80085FFC4
:107B8000FCCF8AE08093CE00809138078230E9F004
:107B900018F0833081F108959FB7F8948091050122
:107BA0008F7D809305019FBF9FB7F8948091050159
:107BB0008F7E809305019FBF9FB7F8948091050148
:107BC0008860809305019FBF08959FB7F8948091C6
:107BD00005018F7D809305019FBF9FB7F894809129
:107BE00005018061809305019FBF9FB7F894809144
:107BF0000501877FE6CF9FB7F894809105018062E9
:107C0000809305019FBF9FB7F894809105018F7EF7
:107C1000E9CF1F920F920FB60F9211240BB60F925D
:107C20002F933F934F935F936F937F938F939F9384
:107C3000AF93BF93CF93EF93FF93C091D600809102
:107C4000A304E82FF0E0EB57FB4FC083909184042E
:107C5000913009F06BC08D3170F01092A304109236
:107C6000840490918304903E09F069C09093E20AE5
:107C7000109283046CC08C3049F5C13091F710929A
:107C8000A304109284048091890481708093EB0A8C
:107C900060918A0470918B0476276727762790E09D
:107CA00080E00F94C80A2AE037ED43E25CE30F94CA
:107CB0006A066093E30A7093E40A8093E50A90935E
:107CC000E60A80918E0480938304CBCF883049F6F6
:107CD000C13039F61092A304109284046091880494
:107CE00070E083EA93E00E946F3D8091C80085FFB9
:107CF000FCCF8AE08093CE0080918804813009F027
:107D0000B0CFECE9F3E08491882341F09091C80072
:107D100095FFFCCF8093CE003196F5CF8091C800BF
:107D200085FFFCCF8AE08093CE009BCFC03C09F05A
:107D300098CF81E0809384041092A30492CF809125
:107D400082048F5F80938204843008F08FCF80910B
:107D5000A3048F5F8E31C1F08093A304C093DD0A2A
:107D6000FF91EF91CF91BF91AF919F918F917F91B3
:107D70006F915F914F913F912F910F900BBE0F909C
:107D80000FBE0F901F9018951092A304E7CF8F920B
:107D90009F92AF92BF92CF92DF92EF92FF920F939A
:107DA0001F93CF93DF9389E7C82E83E0D82E95E306
:107DB000E92E99E1F92E0EEB1AE0D0E0C0E0F601D1
:107DC00061916F01062E000C770B8091D80A90917B
:107DD000D90A0F947C129093DB0A8093DA0A892BDC
:107DE00009F464C00E94D9304B015C01FE01EC55DE
:107DF000F54F6081611102C06091B70A70E090E0B8
:107E000080E00F94CA0AF7012081318142815381B9
:107E10000F946A06A50194010F94AF0EF8016083D8
:107E20007183828393832196F4E0EF0EF11C0C5F43
:107E30001F4FC430D10519F6C090C60AD090C70AAA
:107E4000E090C80AF090C90A20E030E0A901C7011B
:107E5000B6010F94C30A87FF3BC0A701960160914A
:107E60003D1970913E1980913F19909140190F94DE
:107E7000AE0E20E030E040E85FE30F940F1187FD85
:107E800027C01092C60A1092C70A1092C80A109210
:107E9000C90AE9E4FEE08491882399F09091C80032
:107EA00095FFFCCF8093CE003196F5CFF70180810E
:107EB0009181A281B381F80180839183A283B383EE
:107EC000B2CF8091C80085FFFCCF8AE08093CE00BE
:107ED0008091AE13803409F0BBC02091C60A309166
:107EE000C70A4091C80A5091C90A60913D19709122
:107EF0003E1980913F19909140190F94AE0E20E0E9
:107F000030E040EA50E40F940F1187FDA1C0E091EA
:107F1000EC0A8AE4E89FF0011124E751F84F8191BF
:107F2000882339F09091C80095FFFCCF8093CE0054
:107F3000F6CF8091C80085FFFCCF8AE08093CE0009
:107F4000E1E0FEE08491882341F09091C80095FF24
:107F5000FCCF8093CE003196F5CF8091C80085FF8D
:107F6000FCCF8AE08093CE004091C60A5091C70AA8
:107F70006091C80A7091C90A8DEE9DE00E9441325D
:107F80008091C80085FFFCCF8AE08093CE004091AD
:107F90003D1950913E1960913F197091401988ED3B
:107FA0009DE00E9441328091C80085FFFCCF8AE0AD
:107FB0008093CE008091DE0A9091DF0AA091E00AC2
:107FC000B091E10A83339105A105B1050CF440C0DD
:107FD00040913D1950913E1960913F19709140199F
:107FE0004093C60A5093C70A6093C80A7093C90A9F
:107FF0002091AF13821B9109A109B10980932A0B2B
:1080000090932B0BA0932C0BB0932D0B0E9455B08B
:10801000EFECFDE08491882341F09091C80095FF3A
:10802000FCCF8093CE003196F5CF40912A0B509132
:108030002B0B60912C0B70912D0B85E499E10E9424
:10804000853A8091C80085FFFCCF8AE08093CE00FE
:108050002091CA0A3091CB0A4091CC0A5091CD0AA6
:10806000609141197091421980914319909144197E
:108070000F94AE0E6B017C0120E030E0A9010F945B
:108080000F11181604F5C701B6010F941B10EB0170
:108090008091AE13803409F06AC0C932D1050CF466
:1080A00066C0E091EC0A8AE4E89FF0011124E751F0
:1080B000F84F8191882359F09091C80095FFFCCF2B
:1080C0008093CE00F6CFC701B6019058DECF8091E5
:1080D000C80085FFFCCF8AE08093CE004091CA0A99
:1080E0005091CB0A6091CC0A7091CD0A8BEB9DE048
:1080F0000E9441328091C80085FFFCCF8AE08093C6
:10810000CE004091411950914219609143197091EC
:10811000441986EA9DE00E9441328091C80085FFA3
:10812000FCCF8AE08093CE00CB35D10504F120E06E
:1081300030E040E050E460913D1970913E1980912B
:108140003F19909140190F940F11181684F48091E3
:10815000411990914219A0914319B091441980930B
:10816000CA0A9093CB0AA093CC0AB093CD0A86E4B6
:108170000E94B730882319F10E94D9306B017C012D
:1081800020E030E0A9010F940F111816C4F4C0923A
:10819000E902D092EA02E092EB02F092EC0220E0D7
:1081A00030E040E752E4C701B6010F94A90F609395
:1081B0000303709304038093050390930603DF91F8
:1081C000CF911F910F91FF90EF90DF90CF90BF90D4
:1081D000AF909F908F9008950E94C73E89E40E94BF
:1081E000B7308823D1F00E94D93060933B0570935B
:1081F0003C0580933D0590933E058AE40E94B7308C
:108200008823A1F00E94D93060933F057093400508
:108210008093410590934205089510923B0510927A
:108220003C0510923D0510923E05E7CF10923F05A8
:1082300010924005109241051092420508954F9208
:108240005F926F927F928F929F92AF92BF92EF92C6
:10825000FF920F931F93CF93DF938091B704811107
:108260000DC00E949AB46093B3047093B4048093D9
:10827000B5049093B60481E08093B7040E949AB449
:108280000091B3041091B4042091B5043091B60468
:10829000601B710B820B930B613D7740810591054B
:1082A00008F412C2E2E4FDE08491882341F0909149
:1082B000C80095FFFCCF8093CE003196F5CF60913A
:1082C000180B7091190B80911A0B90911B0B41E0C8
:1082D0000E947DACEFE3FDE08491882341F0909112
:1082E000C80095FFFCCF8093CE003196F5CF60910A
:1082F000140B7091150B072E000C880B990B0F9423
:10830000CA0A41E00E947DACEAE3FDE08491882343
:1083100041F09091C80095FFFCCF8093CE0031963C
:10832000F5CF60911C0B70911D0B80911E0B9091ED
:108330001F0B41E00E947DACE7E3FDE084918823C0
:1083400041F09091C80095FFFCCF8093CE0031960C
:10835000F5CF6091160B7091170B072E000C880B50
:10836000990B0F94CA0A41E00E947DACE3E3FDE063
:108370008491882341F09091C80095FFFCCF8093B1
:10838000CE003196F5CF6091F10A7091F20A80919A
:10839000F30A9091F40A41E00E947DACE0E3FDE035
:1083A0008491882341F09091C80095FFFCCF809381
:1083B000CE003196F5CF6091F50A7091F60A072E3E
:1083C000000C880B990B0F94CA0A41E00E947DAC07
:1083D000ECE2FDE08491882341F09091C80095FF84
:1083E000FCCF8093CE003196F5CF6091AC0A7091AE
:1083F000AD0A8091AE0A9091AF0A41E00E947DAC37
:10840000E9E2FDE08491882341F09091C80095FF56
:10841000FCCF8093CE003196F5CF6091B00A709179
:10842000B10A072E000C880B990B0F94CA0A41E081
:108430000E947DACC3EAD2E009E613E094E7E92E9E
:108440009AE0F92E2BEAA22E22E0B22E412C512CDA
:108450003201E6E2FDE08491882341F09091C8006A
:1084600095FFFCCF8093CE003196F5CFB301A201EA
:1084700085E499E10E94853AE4E2FDE08491882355
:1084800041F09091C80095FFFCCF8093CE003196CB
:10849000F5CFF50161917191819191915F0141E079
:1084A0000E947DACE1E2FDE08491882341F090914F
:1084B000C80095FFFCCF8093CE003196F5CFF70131
:1084C000619171917F01072E000C880B990B0F941D
:1084D000CA0A41E00E947DACEEE1FDE08491882370
:1084E00041F09091C80095FFFCCF8093CE0031966B
:1084F000F5CFB301A20185E499E10E94853AECE150
:10850000FDE08491882341F09091C80095FFFCCF55
:108510008093CE003196F5CFF801619171918191F0
:1085200091918F0141E00E947DACE9E1FDE08491F1
:10853000882341F09091C80095FFFCCF8093CE0036
:108540003196F5CF69917991072E000C880B990B24
:108550000F94CA0A41E00E947DACE8E1FDE08491FD
:10856000882341F09091C80095FFFCCF8093CE0006
:108570003196F5CFFFEF4F1A5F0A6F0A7F0A24E0AA
:10858000421651046104710409F063CF8CE6E82EB1
:108590008AE0F82E0BE912E0CBE8D2E0412C512C16
:1085A0003201E5E1FDE08491882341F09091C8001B
:1085B00095FFFCCF8093CE003196F5CFB301A20199
:1085C00085E499E10E94853AE3E1FDE08491882306
:1085D00041F09091C80095FFFCCF8093CE0031967A
:1085E000F5CFF701619171917F01F801819191912E
:1085F0008F0189909990A990B990681B790B072EEB
:10860000000C880B990B0F94CA0AA50194010F94D2
:108610006A060F941B1077FF02C070E060E0AB01A8
:10862000770F660B770B85E499E10E94853AFFEF9F
:108630004F1A5F0A6F0A7F0A24E042165104610450
:10864000710409F0AECFEEE0FDE08491882341F0A3
:108650009091C80095FFFCCF8093CE003196F5CF66
:108660006091E70A7091E80A8091E90A9091EA0A1C
:1086700042E00E947DACE9E0FDE08491882341F076
:108680009091C80095FFFCCF8093CE003196F5CF36
:108690006091E30A7091E40A8091E50A9091E60AFC
:1086A00042E00E947DAC8091C80085FFFCCF8AE04B
:1086B0008093CE000E949AB46093B3047093B40484
:1086C0008093B5049093B604DF91CF911F910F91E1
:1086D000FF90EF90BF90AF909F908F907F906F90A2
:1086E0005F904F9008954F925F926F927F928F921A
:1086F0009F92AF92BF92CF92DF92EF92FF920F9331
:108700001F93CF93DF93E4E7F8E08491882341F04F
:108710009091C80095FFFCCF8093CE003196F5CFA5
:108720008091C80085FFFCCF8AE08093CE00C12CE9
:10873000D12C7601C0E287E0815039F09091C800D9
:1087400095FFFCCFC093CE00F7CFB701A60185E41B
:1087500099E10E94853A8FEFC81AD80AE80AF80A08
:10876000E7E0CE16D104E104F10429F78091C800B6
:1087700085FFFCCF8AE08093CE00C9E3D7E0C12C0F
:10878000D12C760190E2692E2BE2422E3AE0532E54
:108790008091C80085FFFCCF6092CE00B701A60192
:1087A00085E499E10E94853A8E0187E0782E8091D8
:1087B000C80085FFFCCF6092CE00F80180809180D8
:1087C000A280B380A5019401C501B4010F944412A5
:1087D000811144C020E030E0A901C501B4010F942B
:1087E0000F1187FD06C08091C80085FFFCCF409225
:1087F000CE0043E0C501B4010E947DAC7A94085ECE
:108800001F4F7110D4CF8091C80085FFFCCF5092CC
:10881000CE002496FFEFCF1ADF0AEF0AFF0A86E0A8
:10882000C816D104E104F10409F0B2CF8091C80068
:1088300085FFFCCF8AE08093CE00DF91CF911F911E
:108840000F91FF90EF90DF90CF90BF90AF909F90EF
:108850008F907F906F905F904F90089580E090E2AE
:108860002091C80025FFFCCF9093CE008F5F9DE341
:108870008630B1F7C3CF2F923F924F925F926F92A3
:108880007F928F929F92AF92BF92CF92DF92EF92A0
:10889000FF920F931F93CF93DF93CDB7DEB72C9743
:1088A0000FB6F894DEBF0FBECDBF182F062F4A8338
:1088B000298380916E1485FF55C0E6E6F8E0849127
:1088C000882341F09091C80095FFFCCF8093CE00A3
:1088D0003196F5CF8091C80085FFFCCF80E2809370
:1088E000CE00412F50E070E060E085E499E10E9405
:1088F000853A4A8180E2442321F08DE2413009F437
:108900008BE29091C80095FFFCCF8093CE008091C0
:10891000C80085FFFCCF80E28093CE008091C80024
:1089200085FFFCCF80E28093CE00402F50E070E0C6
:1089300060E085E499E10E94853A598180E25523FF
:1089400021F08DE2513009F48BE29091C80095FF3F
:10895000FCCF8093CE008091C80085FFFCCF8DE5D1
:108960008093CE00A02EB12C812F90E09A8789872A
:10897000F50196E0199FE00DF11D1124EE0FFF1F88
:10898000EE0FFF1FE75CF84F608171818281938158
:108990009B01AC010F944412811131C080916E147F
:1089A00085FF14C0EEE5F8E08491882341F09091B2
:1089B000C80095FFFCCF8093CE003196F5CF809113
:1089C000C80085FFFCCF8AE08093CE002C960FB6BE
:1089D000F894DEBF0FBECDBFDF91CF911F910F91F5
:1089E000FF90EF90DF90CF90BF90AF909F908F90CF
:1089F0007F906F905F904F903F902F90089580915F
:108A0000C80085FFFCCF8AE08093CE00AA811A0FB0
:108A10006981600F76E0719FF0011124DF01AA0DDA
:108A2000BB1DAA0FBB1FAA0FBB1FA75CB84FCC90E2
:108A30001196DC9011971296EC9012971396FC9079
:108A4000BA811B0F719FA0011124DA01AA0DBB1D71
:108A5000AA0FBB1FAA0FBB1FA75CB84F0C911196A2
:108A60001C91119712968C9112978C8713969C905B
:108A7000262F30E0A985BA857A9FC0017B9F900D93
:108A80001124DC01A20FB31FAA0FBB1FAA0FBB1F2B
:108A9000A75CB84F8C9011967C90119712966C90B1
:108AA000129713965C90B9816B0F70E0DC01A60FF2
:108AB000B71FAA0FBB1FAA0FBB1FA75CB84F4C90D4
:108AC00011963C90119712968C9112978B87139662
:108AD0002C90E20FF31FEE0FFF1FEE0FFF1FE75C5E
:108AE000F84F90819983A181AA83B281BB8383814E
:108AF0008C83FA01E60FF71FEE0FFF1FEE0FFF1F2B
:108B0000E75CF84F90819D83A181AE83B281BF83E2
:108B10004381488798014C85592DB8018C85992D42
:108B20000F944412882321F000E010E01C86912C61
:108B30009601A701B601C7010F944412882319F0CA
:108B40006801EC84F92C242D332D4B85522D642D96
:108B5000732D8B85922D0F944412882321F0412C84
:108B6000312C1B86212C282D372D462D552D682D77
:108B7000772D862D952D0F944412882321F0842C77
:108B8000732C6B84522C2D813E814F8158856D81D1
:108B90007E818F8198850F944412882321F01D8255
:108BA0001E821F82188629813A814B815C816981EE
:108BB0007A818B819C810F944412882341F05D81DE
:108BC00059837E817A838F818B8398859C8386E00D
:108BD000A985BA858A9F90018B9F300D1124A20E22
:108BE000B31EAA0CBB1CAA0CBB1CF501E75CF84F1A
:108BF0005F019601A701B601C7010F94AF0E98015E
:108C00004C85592D0F94AE0E6B017C01282D372D0C
:108C1000462D552D682D772D862D952D0F94AF0E51
:108C2000242D332D4B85522D0F94AE0E9B01AC019C
:108C3000C701B6010F94AF0E6B017C0129813A8107
:108C40004B815C8169817A818B819C810F94AF0E0D
:108C50002D813E814F8158850F94AE0E9B01AC0152
:108C6000C701B6010F94AF0E20E030E040E450E4BD
:108C70000F94A90FD5016D937D938D939C931397BA
:108C8000A5CE1F920F920FB60F9211240BB60F9222
:108C90002F934F935F938F939F93EF93FF93209125
:108CA000CE00809172189091731840917418509171
:108CB0007518019693704817590759F0E09172188A
:108CC000F0917318EE58FB4E2083909373188093A5
:108CD0007218FF91EF919F918F915F914F912F911A
:108CE0000F900BBE0F900FBE0F901F901895CF9353
:108CF000DF93D1E0D0937618C4E2C0939818109215
:108D0000771810929918682F86E499E10E94641BE5
:108D10000E941DAFD0937618C093981810927718C0
:108D20001092991884E290E00E944EAE90E080E0AC
:108D30003091C6182091C718321729F086E499E1BE
:108D40000E9419AAF5CFDF91CF910895FF920F935A
:108D50001F93CF93DF9381E00E947746EDEDFBE018
:108D60009491992341F02091C80025FFFCCF909366
:108D7000CE003196F5CFE3EBFBE082FD0DC0EAECCF
:108D8000FBE09491992399F02091C80025FFFCCF36
:108D90009093CE003196F5CF9491992341F0209194
:108DA000C80025FFFCCF9093CE003196F5CFE9E8BF
:108DB000FBE083FD0DC0E0EAFBE09491992399F07C
:108DC0002091C80025FFFCCF9093CE003196F5CFBF
:108DD0009491992341F02091C80025FFFCCF9093F6
:108DE000CE003196F5CFEFE5FBE084FD0DC0E6E760
:108DF000FBE09491992399F02091C80025FFFCCFC6
:108E00009093CE003196F5CF9491992341F0209123
:108E1000C80025FFFCCF9093CE003196F5CFE1E25C
:108E2000FBE085FD21C0EDE4FBE08491882341F067
:108E30009091C80095FFFCCF8093CE003196F5CF7E
:108E40008091C80085FFFCCF8AE08093CE00E7E3E5
:108E5000FBE084918823C1F09091C80095FFFCCF7E
:108E60008093CE003196F5CF8491882341F0909184
:108E7000C80095FFFCCF8093CE003196F5CF80914E
:108E8000C80085FFFCCFE0CF0BED15E0CFEDD5E0BE
:108E9000FF24F394F80141918F014F2550E070E0D9
:108EA00060E085E499E10E94853AC017D10791F707
:108EB000E0E2FBE08491882341F09091C80095FFA7
:108EC000FCCF8093CE003196F5CF8091C80085FF0E
:108ED000FCCF8AE08093CE00DF91CF911F910F915C
:108EE000FF900895CF93DF93D1E0D0937618C5E239
:108EF000C09398181092771810929918682F86E4EA
:108F000099E10E94641B0E941DAFD0937618C09314
:108F10009818109277181092991885E290E00E94A4
:108F20004EAE90E080E03091C6182091C7183217FD
:108F300029F086E499E10E9419AAF5CFDF91CF913B
:108F400008950F931F93CF93DF938C0182E00E94CB
:108F50007247682F6F7C82E00E94191B68EE73E0F5
:108F600080E090E00E9468B40430110520F4109372
:108F700047020093460282E00E947247EC01807330
:108F80009927E0ECFFE0892BC1F50130110529F1AB
:108F9000C4F46C2F6F7C01151105D9F0B8016F5F17
:108FA0007F4F8CED9FE00E946F3D8091C80085FF50
:108FB000FCCF8AE08093CE00DF91CF911F910F917B
:108FC00008950230110589F06C2F6063033011059C
:108FD00029F782E00E94191BE1CF6C2F6F7D82E0A0
:108FE0000E94191B6C2F6061F4CF6C2F6F7E82E0A2
:108FF0000E94191B6C2F6062ECCF8491882341F092
:109000009091C80095FFFCCF8093CE003196F5CFAC
:109010008091C80085FFFCCFCCCF0F931F93CF93D7
:10902000DF938C0182E00E947247C82FD82FD37F34
:109030006D2F82E00E94191B04301105D0F41093AB
:109040002407009323070230110531F16C2F6C6067
:109050000330110559F06D2F0130110539F46C2FD3
:10906000677F82E00E94191B6C2F646082E00E947F
:10907000191BB8016F5F7F4F87EA9FE00E946F3D29
:109080008091C80085FFFCCF8AE08093CE00DF91FD
:10909000CF911F910F9108956C2F6B7F82E00E94FA
:1090A000191B6C2F6860E2CF90E080E00E940D48B1
:1090B00081E00E9477468C709927892B09F042C085
:1090C00081E08093120781E090E00E940D4881E0EA
:1090D0000E9477468C709927892B09F04AC081E05D
:1090E0008093130780911207813009F059C090E0F6
:1090F00080E00E940D4882E090E00E94A14781E05C
:109100000E94774680739927892B09F051C081E02E
:109110008093140783E090E00E94A14781E00E94C1
:10912000774680739927892B09F059C081E0809395
:10913000150780911407813009F068C082E090E043
:109140000C94A14710921207E0E8FFE08491882375
:1091500041F09091C80095FFFCCF8093CE003196EE
:10916000F5CF8091C80085FFFCCF8AE08093CE00C8
:10917000AACF10921307E9E5FFE08491882341F01C
:109180009091C80095FFFCCF8093CE003196F5CF2B
:109190008091C80085FFFCCF8AE08093CE00A2CFEB
:1091A00080911307813009F0A2CF81E090E0A1CF38
:1091B00010921407E2E3FFE08491882341F090913C
:1091C000C80095FFFCCF8093CE003196F5CF8091FB
:1091D000C80085FFFCCF8AE08093CE009BCF109221
:1091E0001507EBE0FFE08491882341F09091C800DF
:1091F00095FFFCCF8093CE003196F5CF8091C800CB
:1092000085FFFCCF8AE08093CE0093CF8091150735
:10921000813009F093CF83E090E092CFCF93DF933A
:10922000D82FC62F84EA8093BC008CE40E94FB1ADE
:109230008D2F0E94FB1A8C2F0E94FB1ADF91CF9179
:109240000C94F31A0E9404B0682F636083E00E94BC
:109250000E4981E08093EF0A61E070E082E092E1E4
:109260000E946F3D8091C80085FFFCCF8AE080930B
:10927000CE0008950E9404B0682F6C7F83E00E94A6
:109280000E491092EF0A70E060E088EF91E10E94D1
:109290006F3D8091C80085FFFCCF8AE08093CE00AF
:1092A00008950E9404B0682F6F7D83E00E940E49EC
:1092B0001092F70AE6EEF1E1849181110DC0E2EE21
:1092C000F1E18491882381F09091C80095FFFCCF53
:1092D0008093CE003196F5CF9091C80095FFFCCFDA
:1092E0008093CE003196E8CF4091F70A50E070E0CD
:1092F00060E085E499E10E94853A8091C80085FF8D
:10930000FCCF8AE08093CE0008950E9404B0682FBD
:10931000606283E00E940E4981E08093F70AEBEDE2
:10932000F1E1849181110DC0E7EDF1E18491882391
:1093300081F09091C80095FFFCCF8093CE003196CC
:10934000F5CF9091C80095FFFCCF8093CE00319669
:10935000E8CF4091F70A50E070E060E085E499E1E1
:109360000E94853A8091C80085FFFCCF8AE08093F7
:10937000CE000895F8940E94BE2268EE82E00E941A
:109380000E4968EE82E00E940E4968EE82E00E947B
:109390000E4968EE82E00E940E491092270BE0EC25
:1093A000F7E2849181110DC0E4E9FEE08491882305
:1093B00081F09091C80095FFFCCF8093CE0031964C
:1093C000F5CF9091C80095FFFCCF8093CE003196E9
:1093D000E8CF8091C80085FFFCCF8AE08093CE0063
:1093E000FFCF2F923F924F925F926F927F928F9218
:1093F0009F92AF92BF92CF92DF92EF92FF920F9324
:109400001F93CF93DF93EC01623059F5E3E3FCE166
:109410008491882341F09091C80095FFFCCF809300
:10942000CE003196F5CF42E050E060E070E085E498
:1094300099E10E94853AE6E1FCE18491882341F0BC
:109440009091C80095FFFCCF8093CE003196F5CF68
:109450008091C80085FFFCCF8AE08093CE000E94F7
:10946000BA4970E0FB01EE0FFF1FEC59FC4F808101
:109470009181009709F4B4C06E597C4FFB01E080E4
:10948000F12CB70161507109AB01B0E0A0E04A17BF
:109490005B070CF43FC08D01040F151F1595079550
:1094A0009801220F331F220F331FFC01E20FF31F1D
:1094B000C590D490CC15DD0519F5F9013296E80F69
:1094C000F91F65917491072E000C880B990B0F946E
:1094D000CA0A4B015C01C501B401DF91CF911F9114
:1094E0000F91FF90EF90DF90CF90BF90AF909F9043
:1094F0008F907F906F905F904F903F902F90089546
:10950000CC16DD061CF4D8011196C1CFA80141503C
:109510005109BDCF4F3F540711F450E040E0AE1564
:10952000BF050CF4BD01440F551F440F551FFC012E
:10953000E40FF51FE590F490660F771F660F771F15
:10954000FC01E60FF71F05911491FA013296E80F1E
:10955000F91FC590D490FB013296E80FF91F2590B2
:109560003490B6010D2C000C880B990B0F94CA0A8D
:109570004B015C01E016F10609F4ADCFBE016E1996
:109580007F09072E000C880B990B0F94CA0A2B0138
:109590003C01B1016C197D09072E000C880B990B59
:1095A0000F94CA0A9B01AC01C301B2010F946A0671
:1095B0002B013C01B8016E197F09072E000C880BA6
:1095C000990B0F94CA0A9B01AC01C301B2010F941D
:1095D000A90F9B01AC01C501B4010F94AF0E79CF67
:1095E000BE01DD0F880B990B0F94CA0A20E030E012
:1095F0004AEF5EE30F946A0620E030E040E85DE366
:109600000F946A0620E030E0A901E7CF2F923F9245
:109610004F925F926F927F928F929F92AF92BF9282
:10962000CF92DF92EF92FF920F931F93CF93DF932E
:1096300000D01F921F92CDB7DEB7FBEBAF2EF6E046
:10964000BF2EACE3EA2EA6E0FA2E0AE316E02AE1EA
:1096500036E03D832C8388E19BE09B838A831982DB
:109660006981F501819191915F010E94F1492B017E
:109670003C01F701C190D1907F01F80121908F0149
:10968000312C4101880C991C2C813D81820E931E46
:10969000F40180819181C81AD90AC301B2010F94E3
:1096A0001B10F40171836083B601DD0C880B990BEC
:1096B0000F94CA0AA30192010F94AF0E0F941B10CE
:1096C000F701329771836083F80131972FEF221AE7
:1096D000320A37E0232233242082E3E07595679530
:1096E000EA95E1F7072E000C880B990B0F94CA0A34
:1096F000EA81FB816193719381939193FB83EA8368
:109700002C813D81205F3F4F3D832C833981313057
:1097100009F01FC18091B9069091BA060E94DE1728
:109720006093AC0A7093AD0A8093AE0A9093AF0A2F
:109730008091B7069091B8060E94211727E73EEB6B
:109740004FE55FE30F946A0623E333E343E750E416
:109750000F94AF0E209135023091360240913702BE
:10976000509138020F946A064B015C018091090602
:10977000E82FF0E0FB83EA83CF01880F991F9C015B
:10978000265F394F79010091070610910806F9010B
:1097900080819181081B190BC501B4010F941B1026
:1097A000F70171836083B801110F880B990B0F9437
:1097B000CA0AA50194010F94AF0E0F941B10709369
:1097C0000806609307062A813B812F5F3F4F277071
:1097D00033273B832A832093090653E075956795C9
:1097E0005A95E1F7072E000C880B990B0F94CA0AC3
:1097F0006093F10A7093F20A8093F30A9093F40A4B
:109800008091B5069091B6060E94DE176093E70A34
:109810007093E80A8093E90A9093EA0A3091FA0675
:10982000832F90E09B838A83FC01EE0FFF1FE3559B
:10983000F94F6081718144E050E081E090E0DA010D
:10984000AA5EB14EFD0125913491621773070CF0A9
:1098500083C00197880F991F880F991F8C01085E9C
:10986000114EF801859094908A5E914EFC012591ED
:109870003491FA01E85EF14EE590F490F801A5907C
:10988000B490FD0105911491FC01C590D490621B28
:10989000730B072E000C880B990B0F94CA0A2B012F
:1098A0003C01B7016A197B09072E000C880B990B44
:1098B0000F94CA0A9B01AC01C301B2010F946A065E
:1098C0002B013C01B8016C197D09072E000C880B97
:1098D000990B0F94CA0A9B01AC01C301B2010F940A
:1098E000A90F6B017C01B401990C880B990B0F94A3
:1098F000CA0A9B01AC01C701B6010F94AF0EEA8101
:10990000FB81EE0FFF1FEE0FFF1FE555FD4F60833C
:10991000718382839383A8958FB7F8941092FE0683
:109920008FBF0F900F900F900F900F90DF91CF91FE
:109930001F910F91FF90EF90DF90CF90BF90AF906D
:109940009F908F907F906F905F904F903F902F905F
:10995000089591E0998384CE01964C5F5F4F443A1D
:10996000510509F06CCFE8EBFEE165917491072E8B
:10997000000C880B990B0F94CA0AC1CF2F923F920B
:109980004F925F926F927F928F929F92AF92BF920F
:10999000CF92DF92EF92FF920F931F93CF93DF93BB
:1099A00000D01F921F92CDB7DEB78091AE138034E6
:1099B00009F07AC08091DC0A811176C00E949AB4C5
:1099C0000091CE0A1091CF0A2091D00A3091D10A8D
:1099D000601B710B820B930B61397F4581409105B0
:1099E00008F41FC10E949AB4009103061091040666
:1099F0002091050630910606601B710B820B930BBC
:109A0000683E73408105910578F00E949AB4609396
:109A100003067093040680930506909306068091D2
:109A200002068F5F80930206809102068B3078F1E8
:109A300080910106109202068F5F80930106EBEF82
:109A4000FBE18491882341F09091C80095FFFCCF01
:109A50008093CE003196F5CF8091C80085FFFCCF72
:109A60008AE08093CE00E7EFFBE18491882341F008
:109A70009091C80095FFFCCF8093CE003196F5CF32
:109A80008091C80085FFFCCF8AE08093CE00809152
:109A90000106873048F00E9455B086E490E00E94AD
:109AA000B13382E08093DC0A88E19BE09A8389836A
:109AB00044E1C42E4BE0D42E59EF852E55E0952E6F
:109AC00065EFE62E65E0F62E03EF15E07BEE272E20
:109AD00075E0372E1B82E981FA81408051806280D7
:109AE0007380F6010190F081E02DFD83EC83BF01CE
:109AF0006A507109072E000C880B990B0F94CA0A43
:109B00009B01AC01C301B2010F94C30A87FFCEC20F
:109B10000E949AB4F401408051806280738064197D
:109B2000750986099709683E73408105910588F09B
:109B30000E949AB4F4016083718382839383F70156
:109B400080819181019691838083F80180818F5F6C
:109B50008083F801F081FC83E981FA8140805180A3
:109B600062807380FC81FE3108F44EC220E030E058
:109B700048EC52E4C301B2010F94C30A181694F5DD
:109B80002C812C3308F440C220E030E048EC52E451
:109B9000C301B2010F940F11181654F420E030E005
:109BA00046E953E4C301B2010F94C30A1816D4F472
:109BB0003C813A3508F428C220E030E046E953E41D
:109BC000C301B2010F940F1118160CF01DC220E052
:109BD00030E048EC53E4C301B2010F94C30A1816F5
:109BE0000CF412C2F1012081318142815381C30101
:109BF000B2010F94AE0E20E030E040E251E40F9449
:109C0000C30A18160CF44AC0E2EEFBE184918823E3
:109C100081F09091C80095FFFCCF8093CE003196E3
:109C2000F5CF10920206109201063ECF91E09B8381
:109C300052CFE981FA81608171818281938142E012
:109C40000E947DAC8091C80085FFFCCFFAE0F093C4
:109C5000CE00E8ECFBE18491882341F09091C800AC
:109C600095FFFCCF8093CE003196F5CFF101608156
:109C700071818281938142E00E947DAC8091C80015
:109C800085FFFCCFFAE0F093CE002B818AE090E0D4
:109C9000213011F48BE090E00E94B133F801108282
:109CA000E981FA8180819181A281B381F101808370
:109CB0009183A283B383F701A080B180F8E7AF1648
:109CC000B10438F0F60180819181873E91050CF452
:109CD00054C0B50190E080E00F94C80A2B013C010C
:109CE00020E030E040E453E40F940F1187FD9AC167
:109CF000F6010190F081E02DFD83EC83E73EF10554
:109D00000CF490C1ED32F140C4F130EFA316B10470
:109D100008F097C120E030E04CE953E4C301B20100
:109D20000F940F1187FD9DC1F6010190F081E02D88
:109D3000FD83EC83EF35F1400CF493C18C819D8160
:109D400081399140D4F020E030E040EC53E4C3018D
:109D5000B2010F940F1187FF98C120E030E040E17D
:109D600054E4C301B2010F940F1187FD12C0F60134
:109D700080819181833C914064F0F70111821082CF
:109D8000FB818CE090E0F13011F48DE090E00E94D6
:109D9000B13329813A812C5F3F4F3A83298332E0E6
:109DA000C30ED11C84E0880E911C92E0E90EF11CD8
:109DB0000F5F1F4FE4E02E0E311CFB81F13009F0E4
:109DC00035CF88EE93E090931A02809319020E9497
:109DD0009AB40091E7051091E8052091E9053091CA
:109DE000EA05AB01BC01401B510B620B730B809168
:109DF000190290911A02B0E0A0E0481759076A07CB
:109E00007B07C8F10E949AB46093E7057093E80558
:109E10008093E9059093EA05A39A80EC0E94CF32E3
:109E20008CE00E94CF3281E00E94CF3283E00E941A
:109E3000CF3280E00E94CF3280E00E94CF3280E0BB
:109E40000E94CF3280E00E94CF3280E00E94CF3269
:109E500080E00E94CF3289E60E94CF328EEF0E94CE
:109E6000CF3281E00E94CF3262E070E080E090E08B
:109E70000E9468B4A3980E94064BC090AC0AD09090
:109E8000AD0AE090AE0AF090AF0A20E030E040EA80
:109E900050E4C701B6010F940F111816E4F420E046
:109EA00030E045EA53E4C701B6010F94C30A87FFC7
:109EB00012C06091B00A7091B10A072E000C880B95
:109EC000990B0F94CA0A9B01AC01C701B6010F940C
:109ED0000F1187FD30C1109201078BEA882E82E0B6
:109EE000982E97EDC92E95E0D92E24E7E22E2AE090
:109EF000F22E3BED232E35E0332E0FED15E01A82C6
:109F00001982F40141905190619071904F0120E0CD
:109F100030E040EA50E4C301B2010F940F1187FD15
:109F200030C120E030E040EA52E4C301B2010F94B6
:109F3000C30A18160CF425C1F80111821082F7012A
:109F40008081918197FFFBC011821082F701A08070
:109F5000B180B5010B2C000C880B990B0F94CA0A29
:109F60009B01AC01C301B2010F940F1118160CF044
:109F7000EFC0E981FA81EF50F94F108281E00E9431
:109F80007746E091FA06F0E0E552FA4F881F8827FD
:109F9000881F8083F10181911F01882309F4C0C1CA
:109FA000F701808191818397DCF0F60180818E3109
:109FB00008F4B3C1108229813A818BE290E022300B
:109FC000310561F08CE290E02330310539F087E112
:109FD00090E02130310511F48AE290E00E9467346C
:109FE00089819A8101969A8389839FEFC91AD90A38
:109FF000E2E0EE0EF11C0E5F1F4F29813A81243002
:10A00000310509F07ECFB8C120E030E048EC53E4E0
:10A01000C301B2010F940F1118160CF04CCEF801C9
:10A02000108249CE30EFA316B10408F473CEF601C6
:10A030000190F081E02DFD83EC83ED32F1400CF4D2
:10A0400069CE8C819D818F3591400CF496CE20E0B5
:10A0500030E04CE953E4C301B2010F940F1187FFC4
:10A060006DCE20E030E040EC53E4C301B2010F9428
:10A070000F1187FD72CEF6010190F081E02DFD8376
:10A08000EC83E139F1400CF468CE8C819D81833CF6
:10A0900091400CF472CE20E030E040E154E4C30182
:10A0A000B2010F940F1187FF68CE73CE6C817D8152
:10A0B0006C597F4F072E000C880B990B0F94CA0A1E
:10A0C0009B01AC01C301B2010F940F11181644F5A6
:10A0D0002C813D81213A31051CF10E949AB4F40192
:10A0E00040805180628073806419750986099709E0
:10A0F000683E73408105910508F44BCE0E949AB4E6
:10A10000F4016083718382839383F701808191815D
:10A11000019691838083F80180818F5F808339CE9F
:10A12000F70111821082F8011082F1014082518200
:10A13000628273822ECE8FE780930107CECE873462
:10A1400091050CF403CF26E430E031832083FECE6A
:10A15000B50161507109072E000C880B990B0F9403
:10A16000CA0A9B01AC01C301B2010F94C30A1816BD
:10A170000CF404CFE981FA81EF50F94F2FEF2083DF
:10A18000FDCE20E030E04AEA52E4C301B2010F9470
:10A190000F1118160CF05FC020E030E048E453E4E3
:10A1A000C301B2010F94C30A87FF55C0F801808133
:10A1B00091818436910508F4ABC069817A818DE97B
:10A1C0009BE10E946F3D8091C80085FFFCCFFAE0C3
:10A1D000F093CE00F80111821082F70111821082F3
:10A1E000E981FA81EF50F94F108229813A819FB7B6
:10A1F00022303105E1F02330310519F121303105EC
:10A2000061F0F89480910201877F809302019FBFE3
:10A2100085E090E00E946734B1CEF89480910B0104
:10A220008F7D80930B019FBF87E290E0F3CFF8947E
:10A2300080910B018F7E80930B019FBF88E290E09D
:10A24000E9CFF89480910B01877F80930B019FBF2A
:10A2500089E290E0DFCF20E030E040EA50E4C30143
:10A26000B2010F94C30A87FF89CEF80180819181E2
:10A270008436910508F44CC069817A8183E79BE1BB
:10A280000E946F3D8091C80085FFFCCFFAE0F093FB
:10A29000CE00F80111821082F70111821082E9814B
:10A2A000FA81EF50F94F108229813A819FB722300D
:10A2B0003105D1F02330310509F12130310551F05C
:10A2C000F89480910201877F809302019FBF8EE204
:10A2D00090E0A0CFF89480910B018F7D80930B01CB
:10A2E0009FBF8FE290E096CFF89480910B018F7E14
:10A2F00080930B019FBF80E390E08CCFF894809116
:10A300000B01877F80930B019FBF81E390E082CF99
:10A310000196F8019183808331CE8F5F808360CE78
:10A32000F60110828091220B9091230B29813A81B2
:10A3300022303105E1F023303105E1F021303105E3
:10A3400031F0479709F04CCE0E94833D49CE8A9761
:10A35000D9F389819A8101969A8389839FEFC91ADB
:10A36000D90AE2E0EE0EF11C0E5F1F4FCACD8B97AB
:10A3700081F7EACF8C9741F30F900F900F900F90D9
:10A380000F90DF91CF911F910F91FF90EF90DF9091
:10A39000CF90BF90AF909F908F907F906F905F9085
:10A3A0004F903F902F900895CF92DF92EF92FF92BF
:10A3B0000F931F93CF930E949AB40091A00A10911B
:10A3C000A10A2091A20A3091A30AC090CE0AD0908F
:10A3D000CF0AE090D00AF090D10A6C197D098E095D
:10A3E0009F09061717072807390730F4012B022B9E
:10A3F000032B11F00E94BA490E949AB40091CE0A30
:10A400001091CF0A2091D00A3091D10A601B710BB4
:10A41000820B930B61367A4E8105910540F0909145
:10A42000521980915319981302C01092270BC091B2
:10A430006B0A9091531980915219981781F080916D
:10A44000531994E4899FF0011124E25DF44FC6ADE5
:10A4500090915219981719F08F5F8F71F9CFCC2313
:10A46000E9F18091470590914805A0914905B09187
:10A470004A05892B8A2B8B2B81F40E949AB46C5944
:10A480007F4F8F4F9F4F6093470570934805809390
:10A49000490590934A05CFEF0FC00E949AB40091EE
:10A4A0004705109148052091490530914A056017EC
:10A4B00071078207930778F36C2F70E087E00E94A2
:10A4C00091B360916A0A70E08AE0CF911F910F9179
:10A4D000FF90EF90DF90CF900C9491B310924705CE
:10A4E000109248051092490510924A05E5CFCF9386
:10A4F000CAE09091521980915319981701F10E9466
:10A50000BE4C0E94D4510E94A92E8091020689302F
:10A5100081F710920206EBEBFAE18491882341F077
:10A520009091C80095FFFCCF8093CE003196F5CF77
:10A530008091C80085FFFCCFC093CE00DACFCF91C9
:10A5400008950E94775268EE82E00E940E4968EEFC
:10A5500082E00E940E4968EE82E00E940E4968EE99
:10A5600082E00E940E491092270B08952F923F928D
:10A570004F925F926F927F928F929F92AF92BF9213
:10A58000CF92DF92EF92FF920F931F93CF93DF93BF
:10A59000CDB7DEB7CE56D1090FB6F894DEBF0FBEE9
:10A5A000CDBF4C015B015AA349A33AAF29AFEBA23F
:10A5B000FFA20BA718AF1601809152198F5F2E963C
:10A5C0008FAF2E97803219F42E961FAE2E972E96AF
:10A5D0002FAD2E97022F022E000C110BBAE07B2E0E
:10A5E000C22E220FDD08EE08FF0880915319801754
:10A5F000110609F0C4C080910206893009F0A8C094
:10A6000060916F0070E090E080E00E94EC1AE4E559
:10A61000F2E18491882341F09091C80095FFFCCF2E
:10A620008093CE003196F5CF8091C80085FFFCCF96
:10A630007092CE006091521970E090E080E00E942C
:10A64000EC1A6091531970E090E080E00E94EC1ADF
:10A65000B701A60185E499E10E94853A8091200B1B
:10A660009091210BEBE4F2E1892B09F078C0EFE443
:10A67000F2E18491882341F09091C80095FFFCCFCE
:10A680008093CE003196F5CF8091C80085FFFCCF36
:10A690007092CE00E091200BF091210B45855685FC
:10A6A0006785062E000C770B83E492E10E94983AAE
:10A6B000E091200BF091210B4185528563857485D3
:10A6C00081E492E10E94983AE091200BF091210BF5
:10A6D000408151816281062E000C770B8FE392E15D
:10A6E0000E94983AE091200BF091210B4381548114
:10A6F0006581062E000C770B8DE392E10E94983A5B
:10A70000E091200BF091210B468157816085062E48
:10A71000000C770B8BE392E10E94983A60918800DD
:10A720007091890087E392E10E946F3D4091BB05E3
:10A730005091BC056091BD057091BE0580E392E12A
:10A740000E94A0338091C80085FFFCCF7092CE009C
:10A750000E94BE4C0E94D4510E94A92E46CF8491E3
:10A76000882341F09091C80095FFFCCF8093CE00E4
:10A770003196F5CF8091C80085FFFCCF89CF4091FD
:10A7800025195091261960912719709128196A96F8
:10A790004CAF5DAF6EAF7FAF6A9760912919709132
:10A7A0002A1980912B1990912C19AB966CAF7DAF23
:10A7B0008EAF9FAFAB9780912D1990912E19A091DC
:10A7C0002F19B0913019AF968CAF9DAFAEAFBFAF20
:10A7D000AF9720913119309132194091331950912E
:10A7E000341921962CAF3DAF4EAF5FAF2197D10109
:10A7F0000C91B4E00B9F80011124F801E45FF64E48
:10A80000C080D180E280F380F401208131814281D7
:10A8100053816A966CAD7DAD8EAD9FAD6A970F94F6
:10A820006A062B013C0120E030E0A9010F940F11D2
:10A8300020E030E040E05FE387FD05C1C301B201E5
:10A840000F94AF0E0F941B106E966CAF7DAF8EAF52
:10A850009FAF6E97D5012D913D914D915C91AB9637
:10A860006CAD7DAD8EAD9FADAB970F946A064B017D
:10A870005C0120E030E0A9010F940F1120E030E0EE
:10A8800040E05FE387FDE4C0C501B4010F94AF0E63
:10A890000F941B10A2966CAF7DAF8EAF9FAFA297A7
:10A8A000E9A1FAA12081318142815381AF966CAD3B
:10A8B0007DAD8EAD9FADAF970F946A064B015C01E5
:10A8C00020E030E0A9010F940F1120E030E040E0DB
:10A8D0005FE387FDC2C0C501B4010F94AF0E0F94B2
:10A8E0001B10A6966CAF7DAF8EAF9FAFA697A9AD9C
:10A8F000BAAD2D913D914D915C9121966CAD7DADA0
:10A900008EAD9FAD21970F946A06A70196010F9413
:10A910006A066B017C0120E030E0A9010F940F1161
:10A9200020E030E040E05FE387FD9CC0C701B60156
:10A930000F94AF0E0F941B1069AF7AAF8BAF9CAF23
:10A940008091211990912219A0912319B091241975
:10A9500029AD3AAD4BAD5CAD82179307A407B5079F
:10A9600009F494C0F801E85EF44F208131814281FE
:10A970005381609127027091280280912902909161
:10A980002A020F940F11181664F449AD5AAD6BAD3D
:10A990007CAD409321195093221960932319709331
:10A9A00024198091211990912219A0912319B09115
:10A9B000241929AD3AAD4BAD5CAD281B390B4A0BC0
:10A9C0005B0BCA01B90197FF07C090958095709500
:10A9D00061957F4F8F4F9F4F0F94CA0A6B017C0187
:10A9E00020E030E44CE955E421966CAD7DAD8EADB0
:10A9F0009FAD21970F946A069B01AC01C701B60178
:10AA00000F940F1118160CF041C049AD5AAD6BAD43
:10AA10007CAD4093211950932219609323197093B0
:10AA20002419EAE2F2E18491811121C0ECE0F2E123
:10AA30008491882321F19091C80095FFFCCF8093E9
:10AA4000CE003196F5CFC301B2010F94AE0EFACE0F
:10AA5000C501B4010F94AE0E1BCFC501B4010F9414
:10AA6000AE0E3DCFC701B6010F94AE0E63CF9091ED
:10AA7000C80095FFFCCF8093CE003196D4CF809153
:10AA8000C80085FFFCCF8AE08093CE005091521918
:10AA9000A7965FAFA797652F70E07AA369A384E4B8
:10AAA000589FF0011124E25DF44FDF01AF5BBF4F0F
:10AAB0002091D20A3091D30A4091D40A2D933D932C
:10AAC0004C93128E20911519309116194091171937
:10AAD0005091181929962CAF3DAF4EAF5FAF299713
:10AAE0006E968CAD9DADAEADBFAD6E97821B930BD8
:10AAF000A40BB50BB7FF07C0B095A09590958195B5
:10AB00009F4FAF4FBF4F2C016A2E24E449A15AA199
:10AB1000249FF001259FF00D1124E25DF44F808306
:10AB20009183A2836091191970911A1980911B1950
:10AB300090911C192D966CAF7DAF8EAF9FAF2D9766
:10AB4000A2968CAD9DADAEADBFADA2972D962CADAE
:10AB50003DAD4EAD5FAD2D97821B930BA40BB50B96
:10AB6000B7FF07C0B095A095909581959F4FAF4FC7
:10AB7000BF4F24968DAF9EAFAFAF249724E449A179
:10AB80005AA1249FF001259FF00D1124E25DF44F9E
:10AB900083839483A58360911D1970911E19809100
:10ABA0001F199091201962966CAF7DAF8EAF9FAF49
:10ABB0006297A6968CAD9DADAEADBFADA6976296E1
:10ABC0002CAD3DAD4EAD5FAD6297821B930BA40BD8
:10ABD000B50BB7FF07C0B095A095909581959F4F95
:10ABE000AF4FBF4F8CA79DA7AEA724E449A15AA1A0
:10ABF000249FF001259FF00D1124E25DF44F868320
:10AC00009783A0876091211970912219809123194F
:10AC10009091241966966CAF7DAF8EAF9FAF66970B
:10AC200029AD3AAD4BAD5CAD261B370B480B590B2C
:10AC300057FF07C050954095309521953F4F4F4F96
:10AC40005F4F84E4A9A1BAA18A9F80018B9F100D58
:10AC50001124025D144FF8012187328743875487FE
:10AC6000D101EC91F0E0EB59FD4FA081B0E00F94E1
:10AC70005C0E24E630E040E050E00F943D0E6901A8
:10AC80007A01F801C186D286E386F486462D9201C8
:10AC9000042E000C550B28AB39AB4AAB5BAB2496AA
:10ACA0004DAD5EAD6FAD2497062E000C770B4CAB0F
:10ACB0005DAB6EAB7FAB6CA57DA58EA5082E000CA1
:10ACC000990B4B015C01D701C601C814D904EA04F1
:10ACD000FB0414F4D501C4012CA93DA94EA95FA918
:10ACE00082179307A407B50714F00C94E75F68A9CF
:10ACF00079A98AA99BA926173707480759071CF481
:10AD0000A62DC20105C024968DAD9EADAFAD249792
:10AD100024E449A15AA1249FF001259FF00D11249C
:10AD2000E25DF44F85879687A787181619061A06DD
:10AD300014F00C94CD5F80916B0A86AF29966CADB0
:10AD40007DAD8EAD9FAD29976E962CAD3DAD4EADD0
:10AD50005FAD6E9726173707480759070CF40CC6E6
:10AD6000108E2D964CAD5DAD6EAD7FAD2D97A2963C
:10AD70008CAD9DADAEADBFADA29784179507A6076C
:10AD8000B7076CF484E4A9A1BAA18A9FF0018B9F54
:10AD9000F00D1124E25DF44F808D8260808F629609
:10ADA0002CAD3DAD4EAD5FAD6297A6966CAD7DAD61
:10ADB0008EAD9FADA69762177307840795076CF455
:10ADC00084E4A9A1BAA18A9FF0018B9FF00D112400
:10ADD000E25DF44F808D8460808F66962CAD3DAD32
:10ADE0004EAD5FAD669769AD7AAD8BAD9CAD621728
:10ADF0007307840795076CF484E4A9A1BAA18A9F1C
:10AE0000F0018B9FF00D1124E25DF44F808D88607E
:10AE1000808FF101808194E429A13AA1929FF001F1
:10AE2000939FF00D1124E25DF44F818FC114D10482
:10AE3000E104F10409F4A3C520900E0730900F0738
:10AE400000911007109111072BA13FA14BA558AD00
:10AE5000B101C8010F940F11181624F42BA23FA2C0
:10AE60000BA718AF81E08093270B68A979A98AA95D
:10AE70009BA90F94CA0A68AB79AB8AAB9BAB6A9665
:10AE80002CAD3DAD4EAD5FAD6A9760E070E080E8FF
:10AE90009FE30F94A90F9B01AC0168A979A98AA926
:10AEA0009BA90F946A0668AB79AB8AAB9BAB6983AD
:10AEB0007A838B839C836CA97DA98EA99FA90F940B
:10AEC000CA0A6CAB7DAB8EAB9FABAB962CAD3DADE8
:10AED0004EAD5FADAB9760E070E080E89FE30F940C
:10AEE000A90F9B01AC016CA97DA98EA99FA90F9404
:10AEF0006A066CAB7DAB8EAB9FAB6D837E838F831D
:10AF00009887C501B4010F94CA0A4B015C01AF9642
:10AF10002CAD3DAD4EAD5FADAF9760E070E080E829
:10AF20009FE30F94A90F9B01AC01C501B4010F94DD
:10AF30006A0629966CAF7DAF8EAF9FAF2997698760
:10AF40007A878B879C87C701B6010F94CA0A6B0169
:10AF50007C0121962CAD3DAD4EAD5FAD219760E0FB
:10AF600070E080E89FE30F94A90F9B01AC01C7013B
:10AF7000B6010F946A066B017C01CD86DE86EF86F2
:10AF8000F88A0F941B104B011414150416040CF4CA
:10AF9000FFC424964DAD5EAD6FAD24971416150613
:10AFA00016060CF4F5C46CA57DA58EA5161617061D
:10AFB00018060CF4EDC484E4A9A1BAA18A9FF0019B
:10AFC0008B9FF00D1124E25DF44FE894F7F8C2A6D0
:10AFD000D3A6E4A6F5A6FF969182808284E469A1B7
:10AFE0007AA1869FF001879FF00D1124E25DF44F56
:10AFF00082A593A5A4A5B5A525968CAF9DAFAEAFB0
:10B00000BFAF25979C01AD0160E070E080E89FE351
:10B010000F94A90F6CA77DA78EA79FA79B01AC01DA
:10B020006BA17FA18BA598AD0F946A066B017C0183
:10B030008091521990915319891B8F7188AF893073
:10B04000A0F520E030E040E050E425966CAD7DAD09
:10B050008EAD9FAD25970F94C30A87FF26C0A8AD7C
:10B060006A2F70E090E080E00F94CA0A20E030E0A0
:10B0700040E05EE30F946A064B015C012AE939E97E
:10B0800049E95EE30F94C30A87FF07C0AAE98A2E45
:10B09000A9E99A2EA92CAEE3BA2EA5019401C70105
:10B0A000B6010F946A066B017C01A70196012596F3
:10B0B0006CAD7DAD8EAD9FAD25970F946A062D9634
:10B0C0006CAF7DAF8EAF9FAF2D9784E4E9A1FAA15D
:10B0D0008E9F80018F9F100D1124025D144F2D96BD
:10B0E0002CAD3DAD4EAD5FAD2D97D8015E962D9345
:10B0F0003D934D935C9391971D966D917D918C91AD
:10B10000082E000C990B0F94CA0A6BA37CA38DA385
:10B110009EA3A70196010F946A060F948D0F0F94BA
:10B1200022102B013C01F80142AA53AA64AA9E01F5
:10B130002F5F3F4F3EAF2DAF8E010F5E1F4F4CE88C
:10B140005AE064965FAF4EAF649768961FAF0EAF3C
:10B150006897212C312C50E85FA36FE36BA7ADAD4E
:10B16000BEAD6D917D918D919D91BEAFADAFA701AB
:10B1700096010F946A066896EEADFFAD68976193ED
:10B180007193819391936896FFAFEEAF68974B01EF
:10B190005C01E894B7F86496AEADBFAD64972D91AD
:10B1A0003D914D915D916496BFAFAEAF649762964D
:10B1B0002CAF3DAF4EAF5FAF6297C501B4010F94A6
:10B1C0000F111816B4F4A501940162966CAD7DAD13
:10B1D0008EAD9FAD62970F94A90F5B014C01910159
:10B1E0004FA15BA50F940F1118161CF015018FA22B
:10B1F0009BA6EDADFEAD0E171F0709F0B0CF20E006
:10B2000030E040E85FE3B1018FA19BA50F94C30A32
:10B2100087FF47C07801F0E1EF0EF11CD8016D9176
:10B220007D918D919D918D016D01B4E0CB1AD10876
:10B2300091014FA15BA50F946A06F60160837183AB
:10B2400082839383E016F10649F784E429A13AA1A9
:10B25000829F8001839F100D1124025D144F910184
:10B260004FA15BA52D966CAD7DAD8EAD9FAD2D979D
:10B270000F946A06D8015E966D937D938D939C938F
:10B280009197862DB20190E00F94C80A91014FA1C9
:10B290005BA50F946A060F942210F80162AB73ABA2
:10B2A00084AB25962CAD3DAD4EAD5FAD25976BA122
:10B2B0007CA18DA19EA10F94A90F6B017C0184E458
:10B2C00029A13AA1829F8001839F100D1124025D64
:10B2D000144FD8016D907D908C9012976114710479
:10B2E000810409F09DC313968D919D91AC91892B9A
:10B2F0008A2B09F095C3F80186819781A08520915A
:10B30000450A3091460A4091470A5091480A892BD4
:10B310008A2B09F072C3C701B6010F946A060F9415
:10B320008D0F0F942210D801DB966D937D938C9333
:10B3300024E449A15AA1249FC001259F900D112406
:10B34000BC01625D744F3B01FB0183AD94ADA5ADC3
:10B35000BC018A2F90E00F94C80A4B015C01A70141
:10B3600096010F94A90F6FA378A789A79AA7D30175
:10B370009E966D937D938D939C93D1978301035FEC
:10B380001F4F2DEB37E346E051E4C501B4010F94A4
:10B390006A060F941B10F801608771878287C0903E
:10B3A0003D0AD0903E0AE0903F0AF090400A2CA55A
:10B3B0003DA54EA55FA568A979A98AA99BA90F9467
:10B3C0006A0621966CAF7DAF8EAF9FAF21972CA5FB
:10B3D0003DA54EA55FA56CA97DA98EA99FA90F9437
:10B3E0006A062D966CAF7DAF8EAF9FAF2D972CA5C3
:10B3F0003DA54EA55FA529966CAD7DAD8EAD9FADEB
:10B4000029970F946A0629966CAF7DAF8EAF9FAFD8
:10B4100029979091521980915319981709F483C470
:10B42000509008194090091930900A1920900B1972
:10B4300020E030E0A901652D742D832D922D0F940D
:10B440000F1118160CF076C4D3015E961C915E970E
:10B450005F960C915F979096BC91BBA3F30161A09E
:10B46000212F302F4B2F562D652D742D832D922D8E
:10B470000F94C30A87FFFCC35BA64CA638AA2CAA6C
:10B4800020917705309178054091790550917A05A2
:10B4900021966CAD7DAD8EAD9FAD21970F946A0660
:10B4A0004B015C0120917B0530917C0540917D052D
:10B4B00050917E052D966CAD7DAD8EAD9FAD2D97D7
:10B4C0000F946A069B01AC01C501B4010F94AF0E45
:10B4D0004B015C0120917F053091800540918105F1
:10B4E0005091820529966CAD7DAD8EAD9FAD2997AB
:10B4F0000F946A069B01AC01C501B4010F94AF0E15
:10B500004B015C0123E333E343E75FE30F940F1147
:10B5100018160CF0B3C3212F302F4BA1562D652DDB
:10B52000742D832D922D0F94AF0E20E030E040E07B
:10B530005FE30F946A066BA3272E8C0121966CADF6
:10B540007DAD8EAD9FAD21976093770570937805A3
:10B550008093790590937A052D968CAD9DADAEAD17
:10B56000BFAD2D9780937B0590937C05A0937D05BF
:10B57000B0937E0529962CAD3DAD4EAD5FAD2997BC
:10B5800020937F0530938005409381055093820579
:10B5900049895A896B897C8948AB59AB6AAB7BABCB
:10B5A0006D897E898F89988D6CAB7DAB8EAB9FAB9F
:10B5B00078AD723008F4C8C3309008198091091929
:10B5C0008BA790910A1998AFA0910B19ACA727E10E
:10B5D00037EB41ED58E3632D782F892F9A2F0F9485
:10B5E0000F1118160CF0B0C32091F8183091F9180B
:10B5F0004091FA185091FB1868A979A98AA99BA9CA
:10B600000F94AE0E0F9466064B015C012091FC185E
:10B610003091FD184091FE185091FF186CA97DA93A
:10B620008EA99FA90F94AE0E0F9466069B01AC01E4
:10B63000C501B4010F94AF0E0F9404124B015C01CD
:10B64000AC019B01C701B6010F94C30A87FF75C304
:10B65000A5019401C701B6010F94A90F6B017C01EC
:10B66000209100193091011940910219509103194C
:10B67000698D7A8D8B8D9C8D0F94AE0E4B015C0184
:10B68000E894B7F84090390A50903A0A60903B0A23
:10B6900070903C0AA3019201C501B4010F940F11EF
:10B6A000181684F4A5019401C301B2010F94A90FE7
:10B6B0004B015C019601A7010F940F11181614F0AD
:10B6C0006401750120910419309105194091061902
:10B6D000509107196D8D7E8D8F8D98A10F94AE0EB0
:10B6E0004B015C01E894B7F840909C0A50909D0A89
:10B6F00060909E0A70909F0AA3019201C501B40157
:10B700000F940F11181684F4A5019401C301B2011E
:10B710000F94A90F4B015C019601A7010F940F1123
:10B72000181614F0640175019601A7016BA1722D22
:10B73000C8010F946A066B017C019B01AC01632D6B
:10B740007BA588AD9CA50F94C30A87FF04C0C32CBA
:10B75000DBA4E8ACFCA484E429A13AA1829FF00117
:10B76000839FF00D1124E25DF44FC601D70186A33B
:10B7700097A3A0A7B1A76FA178A589A59AA590586E
:10B780009B01AC010F94AF0E25962CAD3DAD4EAD97
:10B790005FAD25970F946A069B01AC016BE077EDD6
:10B7A00083E29CE30F94AE0E0F9404126FA3372E26
:10B7B0004C01262F372FAC01B601C7010F94C30AE5
:10B7C00087FD03C0CFA0D32C740124E449A15AA162
:10B7D000249FC001259F900D1124BC01625D744F10
:10B7E0005B01C601D701FB0182A393A3A4A3B5A368
:10B7F000468C578C60A071A02FA1332DA401C301EA
:10B80000B2010F94C30A18160CF4A2C281E0D5014C
:10B810005C968C9354E4352E29A13AA1329EF00116
:10B82000339EF00D1124E25DF44F81E0838F48A92F
:10B8300059A96AA97BA94093F8185093F918609305
:10B84000FA187093FB186CA97DA98EA99FA9609323
:10B85000FC187093FD188093FE189093FF18898D43
:10B860009A8DAB8DBC8D8093001990930119A09394
:10B870000219B09303198D8D9E8DAF8DB8A1809361
:10B88000041990930519A0930619B09307194092D3
:10B8900008195092091960920A1970920B19A301A4
:10B8A00092016BA1722DC8010F94A90F4B015C018D
:10B8B000A3019201B601C7010F94A90FAB01BC010E
:10B8C000A796AFADA797A39DC00111249501840150
:10B8D000825D944F0E94001C2E96BFAD2E97B093B0
:10B8E00052196E962CAD3DAD4EAD5FAD6E97209367
:10B8F0001519309316194093171950931819A296D9
:10B900004CAD5DAD6EAD7FADA297409319195093CC
:10B910001A1960931B1970931C19A6966CAD7DAD16
:10B920008EAD9FADA69760931D1970931E198093DD
:10B930001F199093201989AD9AADABADBCAD809322
:10B94000211990932219A0932319B093241980915F
:10B95000531994E420915219281709F419C3989F98
:10B96000F0011124E25DF44F238D211149C38F5F53
:10B97000803281F780E0EECF81E0808FF2C92090A5
:10B980000A0730900B0700910C0710910D075CCA55
:10B9900068A979A98AA99BA90F9466066B017C0105
:10B9A0006CA97DA98EA99FA90F9466069B01AC0185
:10B9B000C701B6010F94AF0E6B017C0129966CADE7
:10B9C0007DAD8EAD9FAD29970F9466069B01AC01AE
:10B9D000C701B6010F94AF0E0F94041224E449A1DD
:10B9E0005AA1249FF001259FF00D1124E25DF44F30
:10B9F00062A773A784A795A7EECAC701B6010F94E3
:10BA00006A060F948D0F0F9422109695879577955F
:10BA100067958F779927F80163AF74AF85AF88CCAE
:10BA20002091490A30914A0A40914B0A50914C0AA0
:10BA3000C701B6010F946A060F948D0F0F94221060
:10BA400024E449A15AA1249F8001259F100D1124AF
:10BA5000025D144FD801DB966D937D938C932090FB
:10BA60007C0A30907D0A40907E0A50907F0A90E0D8
:10BA70000F94C80A6FA378A789A79AA7482D9301A6
:10BA8000042E000C550BCA01B9010F94CA0A9B0180
:10BA9000AC016FA178A589A59AA50F946A062BA180
:10BAA0003CA14DA15EA10F94A90F4B015C01C20105
:10BAB000B1010F94C80A9B01AC01C501B4010F94F8
:10BAC0000F1118162CF4D801DB962D923D924C9252
:10BAD0008090800A9090810AA090820AB090830A98
:10BAE00084E4E9A1FAA18E9F80018F9F100D11249B
:10BAF000025D144FF80183AD94ADA5ADBC018A2F52
:10BB000090E00F94C80A2B013C01D80113966D9167
:10BB10007D918C91082E000C990B0F94CA0A9B0101
:10BB2000AC01C301B2010F946A062BA13CA14DA147
:10BB30005EA10F94A90F2B013C01C501B4010F9424
:10BB4000C80A9B01AC01C301B2010F940F11181672
:10BB500024F4F80183AE94AEA5AE8090880A90904C
:10BB6000890AA0908A0AB0908B0A84E429A13AA19C
:10BB7000829F8001839F100D1124025D144FF801F4
:10BB800083AD94ADA5ADBC018A2F90E00F94C80A97
:10BB90002B013C01D80119966D917D918D919C915D
:10BBA0001C970F94CA0A9B01AC01C301B2010F9408
:10BBB0006A062BA13CA14DA15EA10F94A90F2B01F8
:10BBC0003C01C501B4010F94C80A9B01AC01C3013B
:10BBD000B2010F940F11181624F4F80183AE94AE3D
:10BBE000A5AE8090840A9090850AA090860AB090B5
:10BBF000870A84E429A13AA1829F8001839F100DC6
:10BC00001124025D144FF80183AD94ADA5ADBC01C4
:10BC10008A2F90E00F94C80A2B013C01D801169698
:10BC20006D917D918C91082E000C990B0F94CA0A8E
:10BC30009B01AC01C301B2010F946A062BA13CA188
:10BC40004DA15EA10F94A90F2B013C01C501B401C8
:10BC50000F94C80A9B01AC01C301B2010F940F11EC
:10BC600018160CF065CBF80183AE94AEA5AE60CB90
:10BC70001BA70CA7FBA1F8AB6CAA02CC23E333E310
:10BC800043E75FEBC501B4010F94C30A87FF07C008
:10BC900020E030E040E05FE3C701B6014ACCA501F7
:10BCA000940160E070E080E89FE30F94AE0E20E026
:10BCB00030E040E05FE30F946A060F9404124B01FA
:10BCC0005C012DEC3CEC4CEC5DE36FA178A589A503
:10BCD0009AA50F946A06A50194010F946A062B0198
:10BCE0003C01A501940160E070E080E89FE30F94BF
:10BCF000AE0E9B01AC01C301B2010F94A90F0F94CA
:10BD000004126BA3272E8C012BA53CA548A95CA986
:10BD10000F940F1118160CF011CC2BA52BA32CA4EB
:10BD200008A91CA90BCC3DEC3BA3ECEC2E2E0CEC93
:10BD30001DE304CC4DEC4BA3F8CFC12CD12C60E813
:10BD4000E62E7FE3F72E8CCCCBA0D22C780103CD4E
:10BD5000F501148E5FCD8091521983508F71F82EAA
:10BD6000912C812C10E000E044E4542E44244394B0
:10BD70006F1409F453C1F11002C030E2F32EFA94AB
:10BD8000F59CC0011124DC01A25DB44FBAA3A9A3A4
:10BD90000115110509F466C08114910409F462C00B
:10BDA000F80176A0C7A0D0A4E1A4272D3C2D4D2DED
:10BDB0005E2D62A173A184A195A10F94C30A88236B
:10BDC00009F450C0D8015C968C9181114FC0F401E8
:10BDD00082A093A0A4A0B5A0A5019401672D7C2DFD
:10BDE0008D2D9E2D0F940F1118160CF03FC0A5013C
:10BDF0009401C501B4010F946A064B015C01D8019E
:10BE00009E966D917D918D919C91D19790589B01BB
:10BE1000AC010F94AF0EF80122A533A544A555A59A
:10BE20000F946A069B01AC01C501B4010F94AE0EDC
:10BE30000F9404121B014C019B01AC01672D7C2D5A
:10BE40008D2D9E2D0F94C30A87FF04C0272C3C2CF8
:10BE50008D2C9E2CC101D401F80182A393A3A4A32D
:10BE6000B5A3438E480109A11AA182CF872D9C2D2D
:10BE7000AD2DBE2DF1CF009741F0FC01248D211195
:10BE800004C06F2D702F0E94931BD0905319F12C7A
:10BE9000E12C84E4C82E8D2D0D2C000C990B2091E3
:10BEA00052192817190609F44CC0FD2D4C2DF40227
:10BEB00090011124B901625D744F1B01E114F1047A
:10BEC000C9F1D7015B962C9121110AC0C89EF001DF
:10BED000C99EF00D1124E25DF44F238D222351F110
:10BEE000F701468C578C60A071A0C89EF001C99ED6
:10BEF000F00D1124E25DF44FA301920162A173A140
:10BF000084A195A10F94A90F4B015C01A30192019B
:10BF1000D70192966D917D918D919C9195970F94FB
:10BF2000A90FAB01BC0195018401C7010E94001C4F
:10BF3000F701138ED394F0E2DF1201C0D12C71010E
:10BF4000AACFE114F10421F1D7015E968D909D9066
:10BF5000AD90BC909197A50194016DEC7CEC8CECBC
:10BF60009DE30F94A90F2B013C01A5019401F7015A
:10BF700062A173A184A195A10F94A90FAB01BC018B
:10BF800093018201C7010E94001CD7015B961C929D
:10BF900080916F00826080936F00C259DF4F0FB6AF
:10BFA000F894DEBF0FBECDBFDF91CF911F910F91EF
:10BFB000FF90EF90DF90CF90BF90AF909F908F90C9
:10BFC0007F906F905F904F903F902F90089528A999
:10BFD00039A94AA95BA982179307A407B50714F4E6
:10BFE0000C948056AE2DC601C814D904EA04FB0493
:10BFF00014F00C9488568CA59DA5AEA50C9488567B
:10C00000809152198FB7F894609053198FBF809127
:10C01000521986198F71843008F09DCE10915319F2
:10C02000F12C00E090E080E024E4E22E209152190F
:10C03000211709F420CF1E9D90011124F901E25D22
:10C04000F44F6F01009749F0DC015C962C912111AF
:10C0500004C06F2D702F0E94931B1F5F103209F4D4
:10C0600010E08F2D902FFC2C0D2DE0CFCF92DF9282
:10C07000EF92FF920F931F93CF93DF931F92CDB751
:10C08000DEB7E982F801E080F18002811381FE01D0
:10C0900031966F010E94B6520F90DF91CF911F91A0
:10C0A0000F91FF90EF90DF90CF9008952F923F92E5
:10C0B0004F925F926F927F928F929F92AF92BF92B8
:10C0C000CF92DF92EF92FF920F931F93CF93DF9364
:10C0D000CDB7DEB7C955D1090FB6F894DEBF0FBE94
:10C0E000CDBF182FC0903F05D0904005E09041058E
:10C0F000F090420540903B0550903C0560903D0516
:10C1000070903E05A7019601C301B2010F94221160
:10C1100069AF7AAF8BAF9CAF2091141926962FAFE1
:10C1200026976091E00270E090E080E00F94CA0AE8
:10C130002091E9023091EA024091EB025091EC0229
:10C140000F946A0620E030E040E752E40F94A90F14
:10C1500020E030E048EC52E40F94A90F6DA77EA7D1
:10C160008FA798AB20913519309136194091371926
:10C1700050913819C301B2010F94AF0E2A966CAFDB
:10C180007DAF8EAF9FAF2A972091391930913A1920
:10C1900040913B1950913C19C701B6010F94AF0E65
:10C1A0002E966CAF7DAF8EAF9FAF2E9780913D19CD
:10C1B00090913E19A0913F19B091401921968CAFF2
:10C1C0009DAFAEAFBFAF21979C01AD016091C60A94
:10C1D0007091C70A8091C80A9091C90A0F94AE0E57
:10C1E00025966CAF7DAF8EAF9FAF259777FA709491
:10C1F00077F87094D701C601B05889AB9AABABAB56
:10C20000BCAB2A962CAD3DAD4EAD5FAD2A9760918B
:10C21000BE0A7091BF0A8091C00A9091C10A0F9422
:10C22000AE0E6B017C012E962CAD3DAD4EAD5FADDB
:10C230002E976091C20A7091C30A8091C40A9091AE
:10C24000C50A0F94AE0E4B015C01A7019601C30114
:10C25000B2010F946A066DAB7EAB8FAB98AFA501B0
:10C26000940169A97AA98BA99CA90F946A069B01DC
:10C27000AC016DA97EA98FA998AD0F94AF0E6DABDF
:10C280007EAB8FAB98AFA5019401C301B2010F94AF
:10C290006A064B015C01A701960169A97AA98BA9DD
:10C2A0009CA90F946A069B01AC01C501B4010F94CF
:10C2B000AE0E2DA93EA94FA958AD0F942E0F6B01BC
:10C2C0007C0120E030E0A9010F94C30A87FF0AC077
:10C2D0002BED3FE049EC50E4C701B6010F94AF0EDF
:10C2E0006B017C01112351F02BED3FE049EC50E450
:10C2F000C701B6010F94AE0E6B017C01A701960138
:10C3000069AD7AAD8BAD9CAD0F946A0625962CADC8
:10C310003DAD4EAD5FAD25970F9422114B015C01F1
:10C320002FE632E143E85AE30F94C30A87FD22C2A5
:10C33000C501B4010F9451100F9422107EAB6DAB68
:10C34000DB01AB2B21F421E030E03EAB2DAB809143
:10C35000411990914219A0914319B09144196296E4
:10C360008CAF9DAFAEAFBFAF6297ADA9BEA9BD0107
:10C3700090E080E00F94C80A4B015C01AC019B0186
:10C38000C701B6010F94A90F69AF7AAF8BAF9CAF0D
:10C39000A501940125966CAD7DAD8EAD9FAD259721
:10C3A0000F94A90F66966CAF7DAF8EAF9FAF669767
:10C3B00062962CAD3DAD4EAD5FAD62976091CA0AFD
:10C3C0007091CB0A8091CC0A9091CD0A0F94AE0E59
:10C3D000A50194010F94A90F6A966CAF7DAF8EAF43
:10C3E0009FAF6A9720E030E040E05FE369AD7AAD4F
:10C3F0008BAD9CAD0F946A0629AD3AAD4BAD5CADEB
:10C400000F946A069B01AC0160E070E080E89FE356
:10C410000F94AE0E25966CAF7DAF8EAF9FAF259774
:10C4200021968CAD9DADAEADBFAD2197898F9A8F12
:10C43000AB8FBC8F62968CAD9DADAEADBFAD62973C
:10C440008D8F9E8FAF8FB8A3A12C22242394312CE3
:10C45000ADA9BEA9A215B30509F433C1B8E1BA1557
:10C460000CF4C0C0A301920169AD7AAD8BAD9CAD57
:10C470000F946A066B017C0129A93AA94BA95CA912
:10C4800025966CAD7DAD8EAD9FAD25970F946A0658
:10C490009B01AC01C701B6010F94AF0EB62ED72E8B
:10C4A0007C01A301920125966CAD7DAD8EAD9FAD53
:10C4B00025970F946A062B013C0129A93AA94BA99B
:10C4C0005CA969AD7AAD8BAD9CAD0F946A069B01FA
:10C4D000AC01C301B2010F94AE0E2B013C01A39439
:10C4E0008B2D9D2DD70189AB9AABABABBCABA30118
:10C4F00092012A966CAD7DAD8EAD9FAD2A970F94BB
:10C50000AF0E698B7A8B8B8B9C8B29A93AA94BA98F
:10C510005CA92E966CAD7DAD8EAD9FAD2E970F9420
:10C52000AF0E6D8B7E8B8F8B988F66962CAD3DAD4D
:10C530004EAD5FAD6697698D7A8D8B8D9C8D0F9416
:10C54000AF0E698F7A8F8B8F9C8F6A962CAD3DAD25
:10C550004EAD5FAD6A976D8D7E8D8F8D98A10F94D6
:10C56000AF0E6D8F7E8F8F8F98A3CE0141960E9464
:10C57000521A89899A89AB89BC8989839A83AB834A
:10C58000BC838D899E89AF89B88D8D839E83AF834F
:10C59000B887898D9A8DAB8DBC8D89879A87AB873B
:10C5A000BC87AE01475F5F4FBE016B5F7F4FCE011F
:10C5B00001960E94432E2696EFAC26978E01035DCE
:10C5C0001F4F9E01235E3F4FAE01475F5F4FBE018D
:10C5D0006B5F7F4FCE0101960E9436609FEF291A54
:10C5E000390A36CFB10190E080E00F94C80A29AD36
:10C5F0003AAD4BAD5CAD0F946A066B017C010F94B4
:10C60000A40F69AB7AAB8BAB9CABC701B6010F949F
:10C61000F6114B015C01C0903B05D0903C05E090C9
:10C620003D05F0903E05F7FAF094F7F8F09480910C
:10C630003F0590914005A0914105B091420521969A
:10C640008CAF9DAFAEAFBFAF2197A701960169A98F
:10C650007AA98BA99CA90F946A062B013C0121960B
:10C660002CAD3DAD4EAD5FAD2197C501B4010F942A
:10C670006A069B01AC01C301B2010F94AF0E2B01FE
:10C680003C01A7019601C501B4010F946A066B0134
:10C690007C0121962CAD3DAD4EAD5FAD219769A9D2
:10C6A0007AA98BA99CA90F946A069B01AC01C701CA
:10C6B000B6010F94AE0E69AB7AAB8BAB9CABA12CE1
:10C6C00016CFC090BE0AD090BF0AE090C00AF0908A
:10C6D000C10AC982DA82EB82FC824091C20A50917F
:10C6E000C30A6091C40A7091C50A4D835E836F834B
:10C6F00078878091C60A9091C70AA091C80AB09124
:10C70000C90A89879A87AB87BC878090CA0A9090AC
:10C71000CB0AA090CC0AB090CD0A8D869E86AF86BB
:10C72000B88AC9A2DAA2EBA2FCA24DA35EA36FA3B2
:10C7300078A789A79AA7ABA7BCA7AE01475D5F4FB3
:10C74000BE016B5D7F4FCE0181960E94432E2696DF
:10C75000EFAC26978E01035D1F4F9E01235F3F4F75
:10C76000AE01475D5F4FBE016B5D7F4FCE0181968D
:10C770000E943660EEEBFAE0A5E3B9E141915191F8
:10C78000619171914D935D936D937D932AE0EE3CA1
:10C79000F207A1F7C75ADF4F0FB6F894DEBF0FBEFE
:10C7A000CDBFDF91CF911F910F91FF90EF90DF9060
:10C7B000CF90BF90AF909F908F907F906F905F9041
:10C7C0004F903F902F9008952F923F924F925F92FB
:10C7D0006F927F928F929F92AF92BF92CF92DF9291
:10C7E000EF92FF920F931F93CF93DF93CDB7DEB7F6
:10C7F000C155D1090FB6F894DEBF0FBECDBF8EEB89
:10C800009AE00E94521AC090CA0AD090CB0AE090D7
:10C81000CC0AF090CD0A8090411990904219A090D6
:10C820004319B0904419A5019401C701B6010F94B2
:10C83000C30A882309F447C00091141924E0029F19
:10C8400080011124065A1C4FA5019401C701B601AD
:10C850000F94AE0E9F77D8012D913D914D915C9133
:10C860000F946A0620E030E44CE955E40F940F1170
:10C8700018164CF5C0924119D0924219E092431912
:10C88000F0924419E3ECFDE2849181110DC0E6E7DA
:10C89000FEE08491882381F09091C80095FFFCCF41
:10C8A0008093CE003196F5CF9091C80095FFFCCFD4
:10C8B0008093CE003196E8CF8091C80085FFFCCFF1
:10C8C0008AE08093CE004090C60A5090C70A6090DC
:10C8D000C80A7090C90A8091B20A809014192896EB
:10C8E0008FAE289700911002882361F120E030E09C
:10C8F000A901C301B2010F94C30A882321F011E0FA
:10C9000080913A05811110E0C090E107D090E207D4
:10C91000E090E307F090E40720E030E0A901C701D0
:10C92000B6010F94C30A882309F48FC0612F70E009
:10C9300090E080E00F94C80AA70196010F94C30A03
:10C9400087FD83C0602F70E090E080E00F94CA0AFA
:10C950002091030330910403409105035091060395
:10C960000F946A062AE037ED43E25CE30F946A060F
:10C970006B017C016091E00270E090E080E00F9438
:10C98000CA0A9B01AC01C701B6010F946A0620E0F8
:10C9900030E048EC52E40F94A90F69837A838B83CB
:10C9A0009C838091C20A9091C30AA091C40AB0915D
:10C9B000C50A4091BE0A5091BF0A6091C00A7091A9
:10C9C000C10A4D835E836F83788789879A87AB8797
:10C9D000BC874D865E866F86788AAE01435F5F4F67
:10C9E000BE01675F7F4FCE0105960E94432E2896B9
:10C9F000EFAC28978E010F5F1F4F2AEC3AE0AE0193
:10CA0000435F5F4FBE01675F7F4FCE0105960E9477
:10CA100036600E942D1BCF5ADF4F0FB6F894DEBF51
:10CA20000FBECDBFDF91CF911F910F91FF90EF907F
:10CA3000DF90CF90BF90AF909F908F907F906F903E
:10CA40005F904F903F902F900895602F70E090E09E
:10CA500080E00F94CA0A20910303309104034091AF
:10CA60000503509106030F946A062AE037ED43E26E
:10CA70005CE30F946A06698F7A8F8B8F9C8FE090AE
:10CA80003519F09036190091371910913819EDA227
:10CA9000FEA20FA318A720E030E046E952E4C80147
:10CAA000B7010F94AF0E29E838E848E05CE30F9433
:10CAB0006A060F941B1067300CF47DC166E0862E69
:10CAC000660F99089AA689A6E0903919F0903A194C
:10CAD00000913B1910913C19EBAEFCAE0DAF1EAFAF
:10CAE00020E030E042E852E4C801B7010F94AF0EF5
:10CAF00029E838E848E05CE30F946A060F941B10BD
:10CB000066300CF45CC165E0862E660F99082196AC
:10CB10009FAE8EAE21978090BE0A9090BF0AA090E3
:10CB2000C00AB090C10A20E030E046E952E4C501F5
:10CB3000B4010F94AF0E29E838E848E05CE30F94A5
:10CB40006A060F941B102D966FAF2D97E62F673056
:10CB50000CF439C1E6E00E2FEE0F110B18AB0FA746
:10CB6000C090C20AD090C30AE090C40AF090C50AEF
:10CB700020E030E042E852E4C701B6010F94AF0E66
:10CB800029E838E848E05CE30F946A060F941B102C
:10CB90002E966FAF2E97E62F66300CF41BC1E5E0A2
:10CBA0002E2FEE0F330B3AAB29AB49A55AA58FA513
:10CBB00098A94817590709F01EC12196AEADBFAD1F
:10CBC0002197A217B30709F016C16091BE0A7091B0
:10CBD000BF0A8091C00A9091C10AEFA5F8A9EE0F93
:10CBE000FF1FEE0FFF1FE65AFD4E2591359145912F
:10CBF000549116E08FA498A8189DD001199DB00DEE
:10CC00001124E9A9FAA9EA0FFB1FEE0FFF1FEE0F8F
:10CC1000FF1FE75CF84F4080518062807380F40111
:10CC200031961E9F50011F9FB00C1124E9A9FAA94B
:10CC3000EA0DFB1DEE0FFF1FEE0FFF1FE75CF84F25
:10CC4000E080F18002811381E9A2FAA20BA31CA368
:10CC5000E9A9FAA93196AE0FBF1FAA0FBB1FAA0FF1
:10CC6000BB1FA75CB84FCD90DD90ED90FC90EA0D16
:10CC7000FB1DEE0FFF1FEE0FFF1FE75CF84F8080DC
:10CC80009180A280B3808D8E9E8EAF8EB8A22D969D
:10CC90000FAD2D9706300CF0A4C00F94AE0E29E80E
:10CCA00038E848E05CE30F946A064B015C01A3019D
:10CCB000920169A17AA18BA19CA10F94AE0EA5014E
:10CCC00094010F946A06A30192010F94AF0E2B01F9
:10CCD0003C01A70196016D8D7E8D8F8D98A10F94DB
:10CCE000AE0EA50194010F946A06A70196010F9458
:10CCF000AF0E6B017C01E9A9FAA9EE0FFF1FEE0F41
:10CD0000FF1FE658FD4E25913591459154912E9681
:10CD10001FAD2E9715300CF06AC06091C20A709159
:10CD2000C30A8091C40A9091C50A0F94AE0E29E8F7
:10CD300038E848E05CE30F946A064B015C01A3010C
:10CD40009201C701B6010F94AE0E9B01AC01C50163
:10CD5000B4010F946A06A30192010F94AF0E6B0108
:10CD60007C0186EC9AE00E94D8199B01AC01C701B6
:10CD7000B6010F946A069B01AC016091C60A7091DE
:10CD8000C70A8091C80A9091C90A0F94AF0E6983AF
:10CD90007A838B839C832896EFAC28978E01075E5D
:10CDA0001F4F2AEC3AE0AE014F5F5F4F62EC7AE032
:10CDB0008EEB9AE02CCE67FF82CE60E080CE67FFDC
:10CDC000A3CE60E0A1CE2D96FFAC2D97F7FEC3CE8B
:10CDD000E0E0C1CE2E961FAD2E9717FFE1CEE0E02A
:10CDE000DFCEC12CD12C76012601370184CF20E083
:10CDF00030E0A901C2CF2DA13EA14FA158A5C50188
:10CE0000B4010F94AE0E4B015C012BAD3CAD4DADAA
:10CE10005EADC701B6010F94AE0E6B017C0120E040
:10CE200030E0A901C501B4010F94C30A87FFB6C45D
:10CE3000D501C401B0588FAB98AFA9AFBAAF20E00D
:10CE400030E0A901C701B6010F94C30A87FD1CC0D9
:10CE500081E090E009A51AA52FA538A902171307AC
:10CE600011F490E080E044275527481B590B5CA73C
:10CE70004BA7CBAADCAAEDAAFEAA81E090E09E8F88
:10CE80008D8F1AA219A2B5C421E030E03E8F2D8FFC
:10CE900094C481E090E09AA389A31CA61BA6A9C410
:10CEA000AD8DBE8DBAA3A9A3EFEFFFEFFCA7EBA753
:10CEB000A0C427961FAE1EAE2797B0C4A1E0B0E075
:10CEC0002796BFAFAEAF2797A9C4B7010F2C000CB0
:10CED000880B990B0F94CA0A20E030E040EF52E42F
:10CEE0000F946A0620E030E042E852E40F94AE0E60
:10CEF000B62EC72ED82E092F41C52BAD3CAD4DAD5A
:10CF00005EAD6B2D7C2D8D2D902F0F94AE0E259642
:10CF10002CAD3DAD4EAD5FAD25970F94A90F4FC51C
:10CF2000B701FF0C880B990B0F94CA0A20E030E080
:10CF300040EF52E40F946A0620E030E042E852E409
:10CF40000F94AE0E7B018C0166C5A3019201B7015F
:10CF5000C801AAC58091CA0A9091CB0AA091CC0AB7
:10CF6000B091CD0A8D8B9E8BAF8BB88FC090C60AC7
:10CF7000D090C70AE090C80AF090C90AC9C52091AC
:10CF8000BE0A3091BF0A4091C00A5091C10A609117
:10CF900035197091361980913719909138190F947D
:10CFA000C30A811112CE2091391930913A1940915A
:10CFB0003B1950913C196091C20A7091C30A80914B
:10CFC000C40A9091C50A0F94C30A8111FECD21CDE8
:10CFD00029A43AA48D8C9E8C280C391C2796AEACC3
:10CFE000BFAC2797AB2809F04CC1AFA4B8A8A80CD8
:10CFF000B91CBE8EAD8E8D8C9E8C8214930409F468
:10D0000083C2ABA4BCA42A0C3B1C81011127F22CC7
:10D0100046E0B42EB21408F4E7C0F801EE0FFF1F8B
:10D02000EE0FFF1FE65AFD4E4591559165917491A3
:10D03000F42FE52FCB012F2F3E2FAC0125966CADA1
:10D040007DAD8EAD9FAD25970F946A062BAD3CAD9F
:10D050004DAD5EAD0F94AF0E69877A878B879C8745
:10D06000812C912C540127E02216310458F421968A
:10D070004EAD5FAD2197B101CE0109960E949B187C
:10D080004B015C0186EC9AE00E94D81969A37AA34F
:10D090008BA39CA336E03F1508F4BCC0F801EE0F4B
:10D0A000FF1FEE0FFF1FE65AFD4E85919591A5914A
:10D0B000B4917C018D01C701D8018D839E83AF831C
:10D0C000B887409035195090361960903719709094
:10D0D0003819A3019201B701C8010F94C30A88232C
:10D0E00009F489CF2FEF3FEF4FE75FE76DA17EA1F6
:10D0F0008FA198A50F94441281110DC02FEF3FEF1F
:10D100004FE75FE76DA17EA18FA198A50F94C30A99
:10D1100018160CF4A1C02BA93CA94DA95EA96FA9B2
:10D1200078AD89AD9AAD0F940F1118160CF087C029
:10D13000A3019201B701C8010F94AE0E6B017C01EF
:10D14000AC019B012C966CAD7DAD8EAD9FAD2C9747
:10D150000F946A069B01AC016091411970914219CC
:10D1600080914319909144190F94AF0E6D8B7E8B73
:10D170008F8B988FA701960162966CAD7DAD8EADB9
:10D180009FAD62970F946A0620913D1930913E1928
:10D1900040913F19509140190F94AF0E6B017C01E3
:10D1A000A501940169A17AA18BA19CA10F946A06A3
:10D1B000A70196010F94AF0E69837A838B839C83BA
:10D1C0002896EFAC28978E01075E1F4F9E012B5EBD
:10D1D0003F4FAE014F5F5F4FBE01675F7F4FCE0194
:10D1E00005960E94366007CFB801012E000C880B0F
:10D1F000990B0F94CA0A20E030E040EF52E40F94FC
:10D200006A0620E030E046E952E40F94AE0EF62FB5
:10D21000E72F11CFB801110F880B990B0F94CA0A91
:10D2200020E030E040EF52E40F946A0620E030E066
:10D2300046E952E40F94AE0E7B018C013CCF209165
:10D24000391930913A1940913B1950913C1969852F
:10D250007A858B859C8570CF8091CA0A9091CB0A84
:10D26000A091CC0AB091CD0A8D8B9E8BAF8BB88FDD
:10D27000C090C60AD090C70AE090C80AF090C90AC8
:10D280008FCF21964EAC5FAC219789A89AA84818F9
:10D29000590869A57AA5AFA4B8A86A197B0977FFD0
:10D2A00003C07195619571097AA769A757FE03C0FC
:10D2B00051944194510821966EAC7FAC219789A07E
:10D2C0009AA0680C791CA9A4BAA4AB2821F4411433
:10D2D000510409F419C18BA5820D682F70E08730C5
:10D2E00008F037C1660F771F660F771FFB01E65AFC
:10D2F000FD4E85919591A591B4916C017D01C6017A
:10D30000D701898B9A8BAB8BBC8B26968FAD2697DA
:10D31000860D682F70E0863008F030C1660F771FE9
:10D32000660F771FFB01E658FD4E85919591A591FB
:10D33000B4915C018D01C501D8018D879E87AF87AF
:10D34000B88B9601A70125966CAD7DAD8EAD9FADD6
:10D3500025970F946A062BAD3CAD4DAD5EAD0F9495
:10D36000AF0E69877A878B879C872BAD3CAD4DAD1F
:10D370005EADB501C8010F94AE0E25962CAD3DAD46
:10D380004EAD5FAD25970F94A90F9B01AC012D8386
:10D390003E834F83588701E010E0B601C7010F9428
:10D3A000C30A87FD02C010E000E08D8C9E8C8016C1
:10D3B000910609F01EC12796AEACBFAC27976A0C48
:10D3C0007B1CB101681979096730710508F0EBC061
:10D3D00006E06016710408F0E6C0A301CE010596D0
:10D3E0000E943A196B017C0186EC9AE00E94D819E0
:10D3F000A70196010F946A064B015C012FEF3FEFE6
:10D400004FE75FE76DA17EA18FA198A50F9444120D
:10D4100081110DC02FEF3FEF4FE75FE76DA17EA1B8
:10D420008FA198A50F94C30A18160CF4CDC02BA990
:10D430003CA94DA95EA96FA978AD89AD9AAD0F94AD
:10D440000F1118160CF0B3C0209135193091361910
:10D4500040913719509138196D817E818F8198855F
:10D460000F94AE0E6B017C01AC019B012C966CAD50
:10D470007DAD8EAD9FAD2C970F946A069B01AC01DC
:10D48000609141197091421980914319909144190A
:10D490000F94AF0E6D8B7E8B8F8B988FA7019601AB
:10D4A00062966CAD7DAD8EAD9FAD62970F946A06AE
:10D4B00020913D1930913E1940913F1950914019EA
:10D4C0000F94AF0E9B01AC01C501B4010F94AF0ED8
:10D4D00069837A838B839C832896EFAC28978E018F
:10D4E000075E1F4F9E012B5E3F4FAE014F5F5F4FA8
:10D4F000BE01635F7F4FCE0105960E94366011E04A
:10D50000411A510808F0DFCE2091BE0A3091BF0ABF
:10D510004091C00A5091C10A609135197091361935
:10D5200080913719909138190F94C30A81114DCB0E
:10D530002091C20A3091C30A4091C40A5091C50A91
:10D540006091391970913A1980913B1990913C1969
:10D550003ACD072E000C880B990B0F94CA0A20E0D5
:10D5600030E040EF52E40F946A0620E030E046E9F4
:10D5700052E40F94AE0E6B017C01C1CE072E000C5D
:10D58000880B990B0F94CA0A20E030E040EF52E478
:10D590000F946A0620E030E042E852E40F94AE0EA9
:10D5A0005B018C01C8CEC12CD12C76011DCF2091FE
:10D5B000391930913A1940913B1950913C196D85B8
:10D5C0007E858F8598894CCF8091CA0A9091CB0A2D
:10D5D000A091CC0AB091CD0A8D8B9E8BAF8BB88F6A
:10D5E0002091C60A3091C70A4091C80A5091C90AD1
:10D5F0006BCF8BA49CA4280C391C07E020163104A7
:10D6000008F0A6C0A30189A09AA04819590946307C
:10D61000510508F09DC0B101CE0109960E949B18EA
:10D620006B017C0186EC9AE00E94D819A701960153
:10D630000F946A064B015C012FEF3FEF4FE75FE766
:10D640006DA17EA18FA198A50F94441281110DC0E8
:10D650002FEF3FEF4FE75FE76DA17EA18FA198A568
:10D660000F94C30A18160CF484C02BA93CA94DA929
:10D670005EA96FA978AD89AD9AAD0F940F111816F8
:10D680000CF06AC020913519309136194091371944
:10D690005091381969897A898B899C890F94AE0ECB
:10D6A0006B017C01AC019B012C966CAD7DAD8EAD08
:10D6B0009FAD2C970F946A069B01AC0160914119B4
:10D6C0007091421980914319909144190F94AF0EB3
:10D6D0006D8B7E8B8F8B988FA701960162966CADB8
:10D6E0007DAD8EAD9FAD62970F946A0620913D1976
:10D6F00030913E1940913F19509140190F94AF0E4F
:10D700009B01AC01C501B4010F94AF0E69837A830C
:10D710008B839C832896EFAC28978E01075E1F4F62
:10D720009E012B5E3F4FAE014F5F5F4FBE01675FB3
:10D730007F4FCE0141960E94366009A51AA501507F
:10D7400011091AA709A70F3F1F4F09F0BCCDDCCE66
:10D75000C12CD12C760166CF2091391930913A191C
:10D7600040913B1950913C1969857A858B859C8540
:10D7700095CF8091CA0A9091CB0AA091CC0AB09122
:10D78000CD0A8D8B9E8BAF8BB88F2091C60A3091BE
:10D79000C70A4091C80A5091C90AB4CF20E030E0CE
:10D7A000A901C701B6010F94C30A87FFD5C18FAA8B
:10D7B00098AEA9AEBAAE1E8E1D8ED701C601B05866
:10D7C0008BAB9CABADABBEABA9A5BAA5EFA5F8A939
:10D7D000AE17BF0709F45DCB0D8D1E8D012B09F02F
:10D7E0005FCB21E030E03AA329A341E050E05CA701
:10D7F0004BA721960EAD1FAD219729A93AA9021773
:10D80000130709F456CB49A15AA1452B09F456CB6D
:10D810008FEF9FEF27969FAF8EAF27972BA93CA93D
:10D820004DA95EA96FA978AD89AD9AAD0F940F117E
:10D8300014018501181614F0160187012091411971
:10D840003091421940914319509144196091CA0A8C
:10D850007091CB0A8091CC0A9091CD0A0F94AE0EB4
:10D860006D8B7E8B8F8B988F9101A8010F94A90FE0
:10D870002C966CAF7DAF8EAF9FAF2C9720913D194A
:10D8800030913E1940913F1950914019C301B201A6
:10D890000F94AE0E9101A8010F94A90F62966CAF80
:10D8A0007DAF8EAF9FAF6297A5019401C701B6010E
:10D8B0000F94A90F25966CAF7DAF8EAF9FAF2597C4
:10D8C0009B01AC016DA17EA18FA198A50F946A0662
:10D8D0009B01AC016BAD7CAD8DAD9EAD0F94AE0EDA
:10D8E0006BAF7CAF8DAF9EAF2C960CAD1DAD2EAD4A
:10D8F0003FAD2C973F770DA31EA32FA338A78BA472
:10D900009CA4892809F064CB21962EAC3FAC2197CA
:10D91000A9A0BAA02A0C3B1C89A89AA88A0C9B1C17
:10D920009AA289A225960CAD1DAD2EAD3FAD2597CF
:10D930003F770D8F1E8F2F8F38A389A09AA0821456
:10D94000930409F41CCB2796AEACBFAC27972A0CE6
:10D950003B1C7101FF24122D163008F0B6CAF701E6
:10D96000EE0FFF1FEE0FFF1FE658FD4E85919591BC
:10D97000A591B491B82EC92EDA2E0B2F2FEF3FEFC1
:10D980004FE75FE76D8D7E8D8F8D98A10F944412C8
:10D990008111B3CA2FEF3FEF4FE75FE76D8D7E8DAB
:10D9A0008F8D98A10F94C30A18160CF0A6CA609127
:10D9B0003519709136198091371990913819698706
:10D9C0007A878B879C87812C912C540106E0201646
:10D9D000310448F4A10169A57AA5CE0109960E94F7
:10D9E0003A194B015C0186EC9AE00E94D8196BA7AA
:10D9F0007CA78DA79EA7163008F092CAF701EE0FFC
:10DA0000FF1FEE0FFF1FE658FD4E85919591A591E2
:10DA1000B4917C018D01C701D8018D839E83AF83B2
:10DA2000B8874090391950903A1960903B1970901E
:10DA30003C19A3019201B701C8010F94C30A8823BE
:10DA400009F47BCF2FEF3FEF4FE75FE76DA17EA19A
:10DA50008FA198A50F94441281110DC02FEF3FEFB5
:10DA60004FE75FE76DA17EA18FA198A50F94C30A30
:10DA700018160CF46FCA2BA93CA94DA95EA96FA971
:10DA800078AD89AD9AAD0F940F1118160CF05DCAE0
:10DA90002091351930913619409137195091381924
:10DAA00069857A858B859C850F94AE0E6B017C0110
:10DAB000AC019B012C966CAD7DAD8EAD9FAD2C97CE
:10DAC0000F946A069B01AC01609141197091421953
:10DAD00080914319909144190F94AF0E6D8B7E8BFA
:10DAE0008F8B988FA701960162966CAD7DAD8EAD40
:10DAF0009FAD62970F946A0620913D1930913E19AF
:10DB000040913F19509140190F94AF0E6B017C0169
:10DB1000A50194016BA57CA58DA59EA50F946A0611
:10DB2000A70196010F94AF0E69837A838B839C8340
:10DB30002896EFAC28978E01075E1F4F9E012B5E43
:10DB40003F4FAE014F5F5F4FBE016B5F7F4FCE0116
:10DB500009960E943660F1CEA9A5BAA5EFA5F8A94D
:10DB60008FAA98AEA9AEBAAECBAADCAAEDAAFEAA3D
:10DB70001E8E1D8E1AA219A2AE17BF0709F035CE50
:10DB80008CC9EF920F931F93CF93DF93CDB7DEB77E
:10DB900064970FB6F894DEBF0FBECDBF198A1A8AFC
:10DBA0001B8A1C8AE09014198E2D90E0FC01EE0F68
:10DBB000FF1FEE0FFF1FE25AF54F40815181628136
:10DBC0007381880F991FE1E0F0E0EC0FFD1FE80F73
:10DBD000F91F518B408B20E030E040EA51E4609126
:10DBE00041197091421980914319909144190F94F1
:10DBF000AF0E60934119709342198093431990932B
:10DC0000441980E090E0A0EAB1E48D879E87AF8759
:10DC1000B88B80913D1990913E19A0913F19B09118
:10DC200040194091391950913A1960913B197091FE
:10DC30003C190091351910913619209137193091FE
:10DC4000381909831A832B833C834D835E836F834A
:10DC5000788789879A87AB87BC87AE01475F5F4F1C
:10DC6000BE016B5F7F4FCE0101960E94432E8E0155
:10DC7000035F1F4F21E439E1AE01475F5F4FBE01F3
:10DC80006B5F7F4FCE0101960E9436600E947752F3
:10DC900020911419E22FF0E0DF01AA0FBB1FAA0F99
:10DCA000BB1FA25AB54F8D919D910D90BC91A02D97
:10DCB000EE0FFF1F41E050E04C0F5D1FE40FF51F1A
:10DCC00040895189841B950B9093F90A8093F80A37
:10DCD000E1EEFCE0211138C0E5EFFCE084918823FF
:10DCE00041F09091C80095FFFCCF8093CE00319613
:10DCF000F5CF4091F80A5091F90A052E000C660BF9
:10DD0000770B85E499E10E94853A8091C80085FFF0
:10DD1000FCCF8AE08093CE008091F80A9091F90AB6
:10DD20000A96459708F444C081E080931A07E4ED11
:10DD3000FCE08491882321F19091C80095FFFCCFED
:10DD40008093CE003196F5CF8491882341F0909155
:10DD5000C80095FFFCCF8093CE003196F5CF40915F
:10DD6000F80A5091F90A052E000C660B770B85E432
:10DD700099E10E94853A8091C80085FFFCCFC9CF08
:10DD80008091C80085FFFCCF8AE08093CE0080910F
:10DD90004D0581110E941F4164960FB6F894DEBFB5
:10DDA0000FBECDBFDF91CF911F910F91EF900895DE
:10DDB00010921A07E7ECFCE08491882341F09091DF
:10DDC000C80095FFFCCF8093CE003196F5CF8091AF
:10DDD000C80085FFFCCFD8CFCF92DF92EF920F9390
:10DDE0001F93CF93DF93CDB7DEB768970FB6F89444
:10DDF000DEBF0FBECDBFCE0101966C0188E0F601FB
:10DE000011928A95E9F7E0901419F4E0EF9EC001B1
:10DE10001124FC01E25AF54F4081518162817381E6
:10DE20008C0D9D1DFC01408351836283738320E030
:10DE300030E040EA50E460914119709142198091BC
:10DE40004319909144190F94AF0E60934119709348
:10DE50004219809343199093441980E090E0A0E028
:10DE6000B0E48D8B9E8BAF8BB88F80913D199091D4
:10DE70003E19A0913F19B091401940913919509124
:10DE80003A1960913B1970913C1900913519109124
:10DE90003619209137193091381909871A872B873D
:10DEA0003C874D875E876F87788B898B9A8BAB8B8E
:10DEB000BC8BAE014F5E5F4FBE01635F7F4FCE01F3
:10DEC00009960E94432E8E010B5E1F4F21E439E11B
:10DED000AE014F5E5F4FBE01635F7F4FCE0109967B
:10DEE0000E9436600E94775280911419F4E08F9F4F
:10DEF00090011124F901E25AF54F4081518162816C
:10DF00007381C20ED31EF601208131818A01021B6A
:10DF1000130BEFE9FCE0811130C0E3EBFCE08491EE
:10DF2000882341F09091C80095FFFCCF8093CE00EC
:10DF30003196F5CFA801012E000C660B770B85E416
:10DF400099E10E94853A8091C80085FFFCCF8AE064
:10DF50008093CE008091F60290E08017910734F50F
:10DF6000E2E9FCE084918823A1F19091C80095FF3B
:10DF7000FCCF8093CE003196F5CF8491882341F079
:10DF80009091C80095FFFCCF8093CE003196F5CFDD
:10DF9000A801012E000C660B770B85E499E10E9425
:10DFA000853A8091C80085FFFCCFD1CF91958195AE
:10DFB0009109E5E8FCE00817190794F28491882399
:10DFC00031F19091C80095FFFCCF8093CE0031963F
:10DFD000F5CF8091C80085FFFCCF8AE08093CE000A
:10DFE00081E080931A07E0911419F0E0EE5EF44F9F
:10DFF000108268960FB6F894DEBF0FBECDBFDF91DA
:10E00000CF911F910F91EF90DF90CF900895809165
:10E01000C80085FFFCCF8AE08093CE0010921A07DB
:10E02000E8CF4F925F926F927F928F929F92AF92C2
:10E03000BF92CF92DF92EF92FF920F931F93CF93F5
:10E04000DF93CDB7DEB7E0970FB6F894DEBF0FBE13
:10E05000CDBF8091AE138F7319F0833009F0EAC100
:10E060008091AE13807C81608093AE130E947752C2
:10E070008090351990903619A0903719B0903819C2
:10E0800089829A82AB82BC82C0903919D0903A19A9
:10E09000E0903B19F0903C19CD82DE82EF82F88649
:10E0A00080913D1990913E19A0913F19B09140196E
:10E0B0008DA79EA7AFA7B8AB89879A87AB87BC8788
:10E0C0004090411950904219609043197090441942
:10E0D0004D865E866F86788A8092FA0A9092FB0A55
:10E0E000A092FC0AB092FD0AC092FE0AD092FF0AEA
:10E0F000E092000BF092010B8093020B9093030BC4
:10E10000A093040BB093050B4092060B5092070BA3
:10E110006092080B7092090B8091E9029091EA02DB
:10E12000A091EB02B091EC028093B90A9093BA0AE5
:10E13000A093BB0AB093BC0A109114191093B204B7
:10E140008091220B9091230B4397029708F45BC0B8
:10E1500094E0199FF0011124E45FF64E2081318193
:10E16000428153816091F7027091F8028091F90227
:10E170009091FA020F94A90F9B01AC01C301B20167
:10E180000F94AE0E6D877E878F87988B20E030E0EE
:10E1900040E752E46091E5027091E6028091E70267
:10E1A0009091E8020F94A90F698B7A8B8B8B9C8BD3
:10E1B0008D8E9E8EAF8EB8A2C9A2DAA2EBA2FCA26F
:10E1C0008DA59EA5AFA5B8A98DA39EA3AFA3B8A703
:10E1D000AE014B5D5F4FBE016F5D7F4FCE014D962F
:10E1E0000E94432EE12E8E010F5E1F4F9E01235F82
:10E1F0003F4FAE014B5D5F4FBE016F5D7F4FCE0164
:10E200004D960E94366020E030E04AEF53E4609182
:10E210003D1970913E1980913F19909140190F94CA
:10E22000C30A87FF0EC020E030E040E251E4698578
:10E230007A858B859C850F94AF0E69877A878B874B
:10E240009C87E090141920E030E040E752E46091B0
:10E25000D8027091D9028091DA029091DB020F947A
:10E26000A90F69A77AA78BA79CA789859A85AB85F3
:10E27000BC854D815E816F81788589809A80AB8075
:10E28000BC80898A9A8AAB8ABC8A4D8B5E8B6F8BE5
:10E29000788F898F9A8FAB8FBC8FAE01475E5F4FAF
:10E2A000BE016B5E7F4FCE0141960E94432E8E01D0
:10E2B000075D1F4F9E01235F3F4FAE01475E5F4FDB
:10E2C000BE016B5E7F4FCE0141960E9436600E9478
:10E2D000775289819A81AB81BC8180933519909363
:10E2E0003619A0933719B09338198D819E81AF816B
:10E2F000B8858093391990933A19A0933B19B0933C
:10E300003C1989859A85AB85BC8580933D1990938E
:10E310003E19A0933F19B09340198D859E85AF8516
:10E32000B8898093411990934219A0934319B093EF
:10E3300044196091140B7091150B072E000C880B7B
:10E34000990B0F94CA0A60930A0B70930B0B80937E
:10E350000C0B90930D0BE090FB02F090FC02B701C8
:10E360000F2C000C880B990B0F94CA0A4B015C010F
:10E3700020E030E0A9010F94C30A87FD4AC0109243
:10E38000150B1092140B6091160B7091170B072E42
:10E39000000C880B990B0F94CA0A60930E0B7093B4
:10E3A0000F0B8093100B9093110B20E030E0A9012C
:10E3B000C501B4010F94C30A87FD30C01092170B3A
:10E3C0001092160B8091AE13807C82608093AE1306
:10E3D0001092660A1092670A1092680A1092690AEF
:10E3E000E091141994E0E99FF0011124E55EF84FE3
:10E3F0001082118212821382E6EEFBE08491882360
:10E4000091F09091C80095FFFCCF8093CE0031969B
:10E41000F5CFF092150BE092140BB5CFF092170BDD
:10E42000E092160BCFCF8091C80085FFFCCF8AE029
:10E430008093CE00E0960FB6F894DEBF0FBECDBF3E
:10E44000DF91CF911F910F91FF90EF90DF90CF90D0
:10E45000BF90AF909F908F907F906F905F904F9004
:10E460000895CF92DF92EF92FF920F931F93CF9375
:10E47000DF93CDB7DEB76C970FB6F894DEBF0FBE53
:10E48000CDBF10925A050E94891D0E94A83A0E9491
:10E490002C32E090FB02F090FC02B7010F2C000C34
:10E4A000880B990B0F94CA0A20E030E0A9010F9461
:10E4B000C30A87FD00C11092150B1092140B109225
:10E4C000170B1092160B1092B10A1092B00A10920C
:10E4D000F60A1092F50A10926B0A10926A0A80915D
:10E4E000AE13982F907C19F08F738093AE138FEF3B
:10E4F0009FEFDC0180932A0B90932B0BA0932C0BA6
:10E50000B0932D0B1092D20A1092D30A1092D40A13
:10E510001092D50A8091AE13982F9F7319F0807CCA
:10E520008093AE1381E080932B0220E030E040EA3C
:10E5300050E460913D1970913E1980913F1990917E
:10E5400040190F94AF0E6B017C01C0923D19D0921F
:10E550003E19E0923F19F092401920E030E040E788
:10E5600052E46091D8027091D9028091DA029091C0
:10E57000DB020F94A90F6D877E878F87988B809120
:10E58000391990913A19A0913B19B0913C194091D9
:10E59000351950913619609137197091381949839E
:10E5A0005A836B837C838D839E83AF83B887C986B0
:10E5B000DA86EB86FC86AE01475F5F4FBE016B5F7C
:10E5C0007F4FCE0101960E94432EE12C8E01035F06
:10E5D0001F4F21E439E1AE01475F5F4FBE016B5F22
:10E5E0007F4FCE0101960E943660C12CD12C80EA6B
:10E5F000E82E80E4F82EC0923519D0923619E092B8
:10E600003719F0923819C0923919D0923A19E0921C
:10E610003B19F0923C1920E030E040E752E4609171
:10E62000D0027091D1028091D2029091D3020F94C6
:10E63000A90F698F7A8F8B8F9C8F80913D19909154
:10E640003E19A0913F19B0914019CD86DE86EF8624
:10E65000F88AC98ADA8AEB8AFC8A8D8B9E8BAF8B0B
:10E66000B88FAE014B5E5F4FBE016F5E7F4FC8013A
:10E670000E94432EE12C045F1F4F21E439E1AE01DB
:10E680004B5E5F4FBE016F5E7F4FCE010D960E94C5
:10E6900036608091B80A81111092B80AE2E1FBE07D
:10E6A0008491882389F09091C80095FFFCCF8093D6
:10E6B000CE003196F5CFF092150BE092140BF0924C
:10E6C000170BE092160BFFCE8091C80085FFFCCFA0
:10E6D0008AE08093CE00E3E0FBE08491882341F060
:10E6E0009091C80095FFFCCF8093CE003196F5CF76
:10E6F0008091C80085FFFCCF8AE08093CE006C96A5
:10E700000FB6F894DEBF0FBECDBFDF91CF911F9142
:10E710000F91FF90EF90DF90CF9008951F93CF93CC
:10E72000DF93CAE0DAE411E08091721890917318D7
:10E730002091741830917518821B930B9370892B5C
:10E7400009F483C00E9433B08A3069F08D3059F0EB
:10E750008A3321F490910905992329F0E0915D0A0B
:10E76000E93408F48CC067E87DE08FEB94E00F9407
:10E77000790A892B29F0DF91CF911F910C94317286
:10E7800062E87DE08FEB94E00F94790A892B09F41D
:10E7900060C0E7E7FDE08491882341F09091C800D4
:10E7A00095FFFCCF8093CE003196F5CF8091C800C5
:10E7B00085FFFCCF8AE08093CE000E94A83A0E9499
:10E7C0002C32409134075091350760913607709193
:10E7D000370780E69DE00E94983A8091C80085FF47
:10E7E000FCCF8AE08093CE000E941170E2E5FDE04C
:10E7F0008491882341F09091C80095FFFCCF8093CD
:10E80000CE003196F5CF8091C80085FFFCCF8AE01D
:10E810008093CE008091AE13807C8034B1F420913F
:10E82000AF1380912A0B90912B0BA0912C0BB091E0
:10E830002D0B821B9109A109B10980932A0B90939A
:10E840002B0BA0932C0BB0932D0BDF91CF911F912D
:10E8500008956FEB74E086E49DE00E94832D809123
:10E86000C80085FFFCCFC093CE00EFEBF4E0DF01E2
:10E870008D2F1D928A95E9F710925D0A55CF8B3343
:10E8800011F4109309059091090591114DCF91E074
:10E890009E0F90935D0AF0E0E154FB4F808344CFDC
:10E8A000EF920F931F93CF93DF93CDB7DEB72C97E3
:10E8B0000FB6F894DEBF0FBECDBFE0901419E5E3AC
:10E8C000F9E180859185A285B38544815581668172
:10E8D0007781008111812281338109831A832B83FF
:10E8E0003C834D835E836F83788789879A87AB8764
:10E8F000BC87AE01475F5F4FBE016B5F7F4FCE01AC
:10E9000001960E94432E03E013E021E439E1AE01B9
:10E91000475F5F4FBE016B5F7F4FCE0101960E9444
:10E9200036602C960FB6F894DEBF0FBECDBFDF91D8
:10E93000CF911F910F91EF9008952F923F924F9298
:10E940005F926F927F928F929F92AF92BF92CF927F
:10E95000DF92EF92FF920F931F93CF93DF9300D03C
:10E960001F92CDB7DEB71C017A8369835C834B832A
:10E970004901409003035090040360900503709098
:10E98000060380916E1485FF1EC020E030E0A901CF
:10E99000EB81FC8160817181828193810F94AF0E44
:10E9A000E981FA81E080F18002811381F101208107
:10E9B0003181428153815B016C0170E060E082EF44
:10E9C00097E00E945C32F401C080D180E280F38045
:10E9D00020E030E0A901C701B6010F94C30A8111FC
:10E9E00008C0C090D802D090D902E090DA02F0902E
:10E9F000DB02EB81FC812081318142815381609176
:10EA00003D1970913E1980913F19909140190F94D2
:10EA1000C30A87FF18C0C0920303D0920403E09298
:10EA20000503F0920603EB81FC8180819181A28134
:10EA3000B38180933D1990933E19A0933F19B093F1
:10EA400040190E945074F40180809180A280B380AC
:10EA500020E030E0A901C501B4010F94C30A81117F
:10EA600008C08090FF0290900003A0900103B09036
:10EA700002038092030390920403A0920503B092D4
:10EA80000603F10180819181A281B38180933519C0
:10EA900090933619A0933719B0933819E981FA8108
:10EAA00080819181A281B3818093391990933A1921
:10EAB000A0933B19B0933C190E945074EB81FC81E8
:10EAC000208131814281538160913D1970913E19BD
:10EAD00080913F19909140190F940F111816C4F4AA
:10EAE000C0920303D0920403E0920503F092060360
:10EAF000EB81FC8180819181A281B38180933D195A
:10EB000090933E19A0933F19B09340190E945074FE
:10EB10000E947752409203035092040360920503CF
:10EB20007092060380916E1485FF14C0EAEDF7E041
:10EB30008491882341F09091C80095FFFCCF809389
:10EB4000CE003196F5CF8091C80085FFFCCF8AE0DA
:10EB50008093CE000F900F900F900F90DF91CF9188
:10EB60001F910F91FF90EF90DF90CF90BF90AF90EB
:10EB70009F908F907F906F905F904F903F902F90DD
:10EB80000895CF92DF92EF92FF921F93CF93DF937E
:10EB9000CDB7DEB72C970FB6F894DEBF0FBECDBF52
:10EBA000182F80916E1485FF13C063E278E08AE32A
:10EBB00098E00E94D6AD612F70E08AE198E00E9453
:10EBC0006F3D8091C80085FFFCCF8AE08093CE0026
:10EBD0008091AC04811709F489C080916E1485FF7F
:10EBE00016C040E050E060E271E48AE098E00E94E4
:10EBF00041328091C80085FFFCCF89E28093CE002E
:10EC00008091C80085FFFCCF8AE08093CE0080E031
:10EC100090E0A0E2B1E48D839E83AF83B887C0907B
:10EC20006A14D0906B14E0906C14F0906D1420E096
:10EC300030E0A901C701B6010F94C30A87FF0CC0D9
:10EC4000A701960160E070E080E291E40F94AE0EBF
:10EC50006D837E838F8398872D813E814F81588578
:10EC600060913D1970913E1980913F199091401922
:10EC70000F94C30A87FF10C019821A821B821C825C
:10EC80009E012F5F3F4FAE014B5F5F4F69E379E11C
:10EC900085E399E10E949D74809135199091361910
:10ECA000A0913719B091381989879A87AB87BC87AB
:10ECB0008091391990913A19A0913B19B0913C1962
:10ECC0008D839E83AF83B88719821A821B821C8230
:10ECD0009E012F5F3F4F4DE359E1BE016B5F7F4FB8
:10ECE000CE0109960E949D741093AC0480E02C968E
:10ECF0000FB6F894DEBF0FBECDBFDF91CF911F914D
:10ED0000FF90EF90DF90CF9008958F929F92AF92F7
:10ED1000BF92CF92DF92EF92FF920F931F93CF9308
:10ED2000DF93CDB7DEB7E5970FB6F894DEBF0FBE21
:10ED3000CDBFE090141984E0E89EF0011124E45F57
:10ED4000F64E20813181428153816091F7027091AA
:10ED5000F8028091F9029091FA020F94A90F9B0199
:10ED6000AC016091411970914219809143199091C1
:10ED700044190F94AE0E6093411970934219809319
:10ED800043199093441920E030E040E752E4609149
:10ED9000E5027091E6028091E7029091E8020F94FB
:10EDA000A90F69837A838B839C8380913D1990910D
:10EDB0003E19A0913F19B0914019409139195091D5
:10EDC0003A1960913B1970913C19809035199090D7
:10EDD0003619A0903719B09038198D869E86AF8667
:10EDE000B88A498B5A8B6B8B7C8B8D8B9E8BAF8BB0
:10EDF000B88FAE014B5E5F4FBE016F5E7F4FCE019D
:10EE00000D960E94432E8E010F5F1F4F21E439E1C2
:10EE1000AE014B5E5F4FBE016F5E7F4FCE010D9620
:10EE20000E943660812C80E4982E84E2A82E84E42F
:10EE3000B82E8092351990923619A0923719B09257
:10EE40003819C12CD12C9FE7E92E93E4F92EC092FA
:10EE50003919D0923A19E0923B19F0923C1910916D
:10EE6000141920E030E040E752E46091D002709144
:10EE7000D1028091D2029091D3020F94A90F69839D
:10EE80007A838B839C8380913D1990913E19A09148
:10EE90003F19B0914019898E9A8EAB8EBC8ECD8E63
:10EEA000DE8EEF8EF8A289A39AA3ABA3BCA3AE011A
:10EEB0004F5D5F4FBE01635E7F4FCE0149960E945A
:10EEC000432EE12E8E010F5F1F4F21E439E1AE0189
:10EED0004F5D5F4FBE01635E7F4FCE0149960E943A
:10EEE00036600E94775282E08DAB20E030E040E057
:10EEF00051E46091411970914219809143199091A8
:10EF000044190F94AF0E6093411970934219809386
:10EF1000431990934419E090141920E030E040E246
:10EF200051E46091E5027091E6028091E7029091D0
:10EF3000E8020F94A90F20E030E040E752E40F947C
:10EF4000A90F6DA37EA38FA398A780913D199091DF
:10EF50003E19A0913F19B091401940913919509133
:10EF60003A1960913B1970913C1980903519909035
:10EF70003619A0903719B090381989AA9AAAABAA65
:10EF8000BCAA4DA75EA76FA778AB89A79AA7ABA726
:10EF9000BCA7AE01475D5F4FBE01635D7F4FCE01F1
:10EFA000C1960E94432E8E010B5D1F4F21E439E173
:10EFB000AE01475D5F4FBE01635D7F4FCE01C196DD
:10EFC0000E94366020E030E040E450E46091411956
:10EFD0007091421980914319909144190F94AE0E8B
:10EFE0006093411970934219809343199093441987
:10EFF000E090141920E030E040E752E46091E5022F
:10F000007091E6028091E7029091E8020F94A90FB7
:10F010006DA37EA38FA398A780913D1990913E196F
:10F02000A0913F19B09140194091391950913A1966
:10F0300060913B1970913C19809035199090361968
:10F04000A0903719B090381989829A82AB82BC821D
:10F050004D835E836F83788789879A87AB87BC8768
:10F06000AE01475F5F4FBE016B5F7F4FCE010196E0
:10F070000E94432E21E439E1AE01475F5F4FBE019C
:10F080006B5F7F4FCE0101960E9436600E947752DF
:10F090008DA9813069F4E2EAF4E08491882351F08B
:10F0A0009091C80095FFFCCF8093CE003196F5CFAC
:10F0B00081E01ACF8091C80085FFFCCF8AE0809361
:10F0C000CE00E5960FB6F894DEBF0FBECDBFDF9140
:10F0D000CF911F910F91FF90EF90DF90CF90BF9055
:10F0E000AF909F908F9008958F929F92AF92BF9212
:10F0F000CF92DF92EF92FF920F931F93CF93DF9304
:10F10000CDB7DEB76C970FB6F894DEBF0FBECDBF9C
:10F1100060912E0270912F02072E000C880B990B24
:10F120000F94CA0A4B015C018092351990923619EE
:10F13000A0923719B092381960912C0270912D026B
:10F14000072E000C880B990B0F94CA0A6B017C01E7
:10F15000C0923919D0923A19E0923B19F0923C19B9
:10F160001091141920E030E040E752E46091D002A1
:10F170007091D1028091D2029091D3020F94A90F85
:10F1800069837A838B839C8380913D1990913E198A
:10F19000A0913F19B09140198D869E86AF86B88A9E
:10F1A000C98ADA8AEB8AFC8A8D8B9E8BAF8BB88FEB
:10F1B000AE014B5E5F4FBE016F5E7F4FCE010D967D
:10F1C0000E94432EE12E8E010F5F1F4F21E439E193
:10F1D000AE014B5E5F4FBE016F5E7F4FCE010D965D
:10F1E0000E943660A895E090141980E090E4A4E2B3
:10F1F000B4E4EE2021F080E090E4ABE2B4E480934C
:10F20000351990933619A0933719B093381980E0C7
:10F2100090E0AFE7B3E48093391990933A19A09343
:10F220003B19B0933C1920E030E040E752E4609194
:10F23000D0027091D1028091D2029091D3020F94AA
:10F24000A90F698F7A8F8B8F9C8F80913D19909138
:10F250003E19A0913F19B091401940913519509134
:10F260003619609137197091381949835A836B8325
:10F270007C8340E050E06FE773E44D835E836F83EF
:10F28000788789879A87AB87BC87AE01475F5F4FD6
:10F29000BE016B5F7F4FCE0101960E94432E8E010F
:10F2A000075E1F4F21E439E1AE01475F5F4FBE01AA
:10F2B0006B5F7F4FCE0101960E9436606C960FB651
:10F2C000F894DEBF0FBECDBFDF91CF911F910F919C
:10F2D000FF90EF90DF90CF90BF90AF909F908F9076
:10F2E00008952F923F924F925F926F927F928F92EA
:10F2F0009F92AF92BF92CF92DF92EF92FF920F93C5
:10F300001F93CF93DF93CDB7DEB7C854D1090FB6A3
:10F31000F894DEBF0FBECDBF0E9474786091411992
:10F3200070914219809143199091441925966CAFC0
:10F330007DAF8EAF9FAF259720E030E040E251E4F3
:10F340000F94AF0E60934119709342198093431943
:10F3500090934419E090141980E090E0A0E4B0E4A8
:10F3600089839A83AB83BC8380913D1990913E1928
:10F37000A0913F19B09140194091391950913A1913
:10F3800060913B1970913C19809035199090361915
:10F39000A0903719B09038198DA29EA2AFA2B8A63E
:10F3A00049A75AA76BA77CA78DA79EA7AFA7B8AB05
:10F3B000AE01435D5F4FBE01675D7F4FCE01859615
:10F3C0000E94432E8E010F5F1F4F21E439E1AE01F1
:10F3D000435D5F4FBE01675D7F4FCE0185960E9402
:10F3E00036600E947752CE018F5B9F4F0E94DB2DCB
:10F3F00081E9282E82E0382E812C912C9FE7A92EBE
:10F4000093E4B92E109114196091D0027091D10239
:10F410008091D2029091D3029B01AC010F94AF0E68
:10F4200020E030E040E752E40F94A90F6B017C012B
:10F4300080913D1990913E19A0913F19B0914019CA
:10F4400029968CAF9DAFAEAFBFAF29971111C2C047
:10F45000B101032C000C880B990B0F94CA0A2B01E5
:10F460003C014092351950923619609237197092CA
:10F47000381980E090E0A5EAB3E4809339199093BD
:10F480003A19A0933B19B0933C19C9AADAAAEBAA7E
:10F49000FCAA4D865E866F86788A898B9A8BAB8BA9
:10F4A000BC8B29968CAD9DADAEADBFAD29978D8B34
:10F4B0009E8BAF8BB88FAE014B5E5F4FBE016F5E10
:10F4C0007F4FCE010D960E94432EE12C8E010F5CE2
:10F4D0001F4F21E439E1AE014B5E5F4FBE016F5E0D
:10F4E0007F4FCE010D960E943660409235195092A2
:10F4F00036196092371970923819809239199092A2
:10F500003A19A0923B19B0923C19E09014196091FD
:10F51000D0027091D1028091D2029091D3029B01CE
:10F52000AC010F94AF0E20E030E040E752E40F94BE
:10F53000A90F69AB7AAB8BAB9CAB80913D199091D5
:10F540003E19A0913F19B0914019498E5A8E6B8E89
:10F550007C8E8D8E9E8EAF8EB8A289A39AA3ABA30C
:10F56000BCA3AE014F5D5F4FBE01635E7F4FCE0116
:10F5700049960E94432E21E439E1AE014F5D5F4F71
:10F58000BE01635E7F4FCE0149960E94366091E0D6
:10F59000291A3108AEE82A16A2E03A0609F032CF5D
:10F5A000C85BDF4F0FB6F894DEBF0FBECDBFDF9153
:10F5B000CF911F910F91FF90EF90DF90CF90BF9070
:10F5C000AF909F908F907F906F905F904F903F9003
:10F5D0002F900895B101645E7F4F072E000C880BB9
:10F5E000990B0F94CA0A2B013C0140923519509295
:10F5F0003619609237197092381980E090E0A5EAC8
:10F60000B3E48093391990933A19A0933B19B093BE
:10F610003C19C9AADAAAEBAAFCAA21964CAE5DAEA7
:10F620006EAE7FAE219789AF9AAFABAFBCAF2996D4
:10F630008CAD9DADAEADBFAD29978DAB9EABAFABE5
:10F64000B8AFAE014B5C5F4FBE01675C7F4FCE0130
:10F65000CD960E94432EE12E8E010F5C1F4F21E4B8
:10F6600039E1AE014B5C5F4FBE01675C7F4FCE015D
:10F67000CD960E94366040923519509236196092AC
:10F680003719709238198092391990923A19A092CC
:10F690003B19B0923C19E09014196091D00270911E
:10F6A000D1028091D2029091D3029B01AC010F94C0
:10F6B000AF0E20E030E040E752E40F94A90F69ABB1
:10F6C0007AAB8BAB9CAB80913D1990913E19A09188
:10F6D0003F19B091401949825A826B827C828D8297
:10F6E0009E82AF82B88689879A87AB87BC87AE0136
:10F6F000475F5F4FBE016B5F7F4FCE0101960E9457
:10F70000432E21E439E1AE01475F5F4FBE016B5FDD
:10F710007F4FCE01019639CF2F923F924F925F9249
:10F720006F927F928F929F92AF92BF92CF92DF9211
:10F73000EF92FF920F931F93CF93DF9300D000D0EF
:10F74000CDB7DEB75C019C01220F331F220F331FA0
:10F750003E832D832B5C364E3901F90110821182D4
:10F76000128213824DE359E169E379E185E399E17E
:10F770000E9427AD8091351990913619A0913719C3
:10F78000B09138198093BE0A9093BF0AA093C00A23
:10F79000B093C10A8091391990913A19A0913B19FF
:10F7A000B0913C198093C20A9093C30AA093C40AF3
:10F7B000B093C50A80913D1990913E19A0913F19CF
:10F7C000B09140198093C60A9093C70AA093C80AC3
:10F7D000B093C90A8091411990914219A09143199F
:10F7E000B09144198093CA0A9093CB0AA093CC0A93
:10F7F000B093CD0A80E090E8ABEBB4E48093490A83
:10F8000090934A0AA0934B0AB0934C0A8D819E8133
:10F8100089509E4D0E94763095012C503E4D4901F5
:10F82000F90114912D813E812254354F3A83298369
:10F830002AE939E949E95FE30F946A066B017C0123
:10F84000612F110F770B880B990B0F94CA0A9B013C
:10F85000AC01C701B6010F946A06E981FA816083A1
:10F860007183828393832D813E8120533D4F2901F3
:10F87000F90160817181828193816093E9027093C3
:10F88000EA028093EB029093EC0220E030E040E744
:10F8900052E40F94A90F54E1C52E59E1D52E7B01F6
:10F8A0008C012AEC3AE046EC5AE062EC7AE08EEB0E
:10F8B0009AE00E94B6520E9477522D813E812851D3
:10F8C000374E1901F90160817181828193810F9412
:10F8D000CA0A2D813E812B5D364E3C832B83F90174
:10F8E00020813181428153810F94A90FAB01BC016A
:10F8F0008DEC91E10E944132F3011082118212825B
:10F9000013824DE359E169E379E185E399E10E94CE
:10F9100027AD2D813E8128513E4D3901C9010E94FC
:10F920007630F401149120E030E040E050EC0F9488
:10F930006A066B017C01612F110F770B880B990B05
:10F940000F94CA0A9B01AC01C701B6010F946A0665
:10F95000E981FA816083718382839383F2016081FC
:10F960007181828193816093E9027093EA028093AE
:10F97000EB029093EC0210922B0220E030E040E783
:10F9800052E40F94A90FE4E1CE2EE9E1DE2E7B01D3
:10F990008C012AEC3AE046EC5AE062EC7AE08EEB1D
:10F9A0009AE00E94B6520E947752F1016081718103
:10F9B000828193810F94CA0AEB81FC81208131817D
:10F9C000428153810F94A90FAB01BC0184EC91E1FA
:10F9D0000E94413281E080932B02C3010E94763065
:10F9E0006B017C01F4016491062E000C770B880BEF
:10F9F000990B0F94CA0AA70196010F946A06E98130
:10FA0000FA81608371838283938320E030E040E455
:10FA100050E4F20160817181828193810F94A90F7A
:10FA20006093E9027093EA028093EB029093EC02F8
:10FA300020E030E040E752E40F94A90FF4E1CF2E2C
:10FA4000F9E1DF2E7B018C012AEC3AE046EC5AE02A
:10FA500062EC7AE08EEB9AE00E94B6520E947752F6
:10FA6000F10160817181828193810F94CA0AEB81D7
:10FA7000FC8120813181428153810F94A90FAB0118
:10FA8000BC0187EB91E10E9441328091C80085FF63
:10FA9000FCCF8AE08093CE00ED81FE81EB5CF64ED8
:10FAA00010821182128213824DE359E169E379E1F8
:10FAB00085E399E10E9427ADF2E0AF16B10409F0A9
:10FAC00003C110922B0280EF91E20E947630F40184
:10FAD00024916B017C01F7FAF094F7F8F094622F0F
:10FAE000220F770B880B990B0F94CA0A9B01AC016C
:10FAF000C701B6010F946A066093C60A7093C70ADD
:10FB00008093C80A9093C90A20E030E040E05FE3A8
:10FB10006091D8027091D9028091DA029091DB0253
:10FB20000F946A066093E9027093EA028093EB02F5
:10FB30009093EC0220E030E040E752E40F94A90FEC
:10FB400024E1C22E29E1D22E7B018C012AEC3AE07D
:10FB500046EC5AE062EC7AE08EEB9AE00E94B652F4
:10FB60000E9477526091F0187091F1188091F2180C
:10FB70009091F3180F94CA0A20912D1930912E19E3
:10FB800040912F19509130190F94A90FAB01BC016E
:10FB900089EA91E10E94413281E080932B0280EF5B
:10FBA00091E20E9476306B017C01F4016491062E93
:10FBB000000C770B880B990B0F94CA0AA7019601CA
:10FBC0000F946A066093C60A7093C70A8093C80AA6
:10FBD0009093C90A20E030E040E450E46091D802FC
:10FBE0007091D9028091DA029091DB020F94A90FF3
:10FBF0006093E9027093EA028093EB029093EC0227
:10FC000020E030E040E752E40F94A90F34E1C32E26
:10FC100039E1D32E7B018C012AEC3AE046EC5AE024
:10FC200062EC7AE08EEB9AE00E94B6520E94775224
:10FC30008091F0189091F118A091F218B091F318FA
:10FC4000181619061A061B060CF07FC08091F018D2
:10FC50009091F118A091F218B091F318C297A105F4
:10FC6000B1050CF080C06091F0187091F11880918E
:10FC7000F2189091F3180F94CA0A20912D1930911F
:10FC80002E1940912F19509130190F94A90FAB01E3
:10FC9000BC018EE991E10E9441328091C80085FF4C
:10FCA000FCCF8AE08093CE0010923D1910923E194D
:10FCB00010923F19109240194DE359E169E379E13F
:10FCC00085E399E10E9427AD2D813E812254354F75
:10FCD000AD81BE81AB5CB64E8D919D910D90BC9176
:10FCE000A02DF90180839183A283B3831092E9024E
:10FCF0001092EA021092EB021092EC020E947C2D0C
:10FD000080E090E8ABE3B5E48093490A90934A0A17
:10FD1000A0934B0AB0934C0A26960FB6F894DEBF18
:10FD20000FBECDBFDF91CF911F910F91FF90EF904C
:10FD3000DF90CF90BF90AF909F908F907F906F900B
:10FD40005F904F903F902F9008958091F018909180
:10FD5000F118A091F218B091F3188F3C9F4FAF4F5C
:10FD6000BF4F0CF080CF84E490E00E94963C7BCFA4
:10FD7000CF92DF92EF92FF920F931F93CF93DF9377
:10FD800080916E1485FF06C064E771E18AE891E115
:10FD90000E94D6AD80B185FB882780F99091240B15
:10FDA000891378C00E94D42D8330A0F52AE037ED66
:10FDB00043E25CE360913D1970913E1980913F19D7
:10FDC000909140190F94AE0E60933D1970933E19B7
:10FDD00080933F199093401920E030E040E752E4CF
:10FDE0006091D8027091D9028091DA029091DB0281
:10FDF0000F94A90F24E1C22E29E1D22E7B018C01A0
:10FE000021E439E14DE359E169E379E185E399E1E1
:10FE10000E94B652A895C0903D19D0903E19E0902E
:10FE20003F19F090401920E030E040EA50E4609142
:10FE30008702709188028091890290918A020F94C2
:10FE4000AE0E9B01AC01C701B6010F94C30A87FF38
:10FE5000A1CFB701A60180E691E10E9441328091D5
:10FE6000C80085FFFCCF8AE08093CE00E7E4F1E193
:10FE70008491882341F09091C80095FFFCCF809336
:10FE8000CE003196F5CF8091C80085FFFCCF8AE087
:10FE90008093CE0064E170E080E090E00E9468B45E
:10FEA000D0B1D5FBDD27D0F9E2E3F1E184918823DD
:10FEB00041F09091C80095FFFCCF8093CE00319621
:10FEC000F5CF4D2F50E070E060E085E499E10E94AD
:10FED000853A64E170E080E090E00E9468B4C0B1CF
:10FEE000C5FBCC27C0F9EDE1F1E18491882341F015
:10FEF0009091C80095FFFCCF8093CE003196F5CF4E
:10FF00004C2F50E070E060E085E499E10E94853A72
:10FF10008091C80085FFFCCF8AE08093CE0080915D
:10FF2000240BC827D81301C0C0E00E94EB3B0E94FD
:10FF30007C2D0E94FCAC0E94573180916E1485FF8D
:10FF400006C063EF70E189E091E10E94D6AD81E0E7
:10FF50008C27DF91CF911F910F91FF90EF90DF9051
:10FF6000CF9008958F929F92AF92BF92DF92EF92BF
:10FF7000FF920F931F93CF93DF93CDB7DEB7E49734
:10FF80000FB6F894DEBF0FBECDBF97FD08C0D12CD1
:10FF900082309105C4F0DD24D3940497A4F0EEE6FA
:10FFA000F0E1D490DD2041F08091C80085FFFCCFC6
:10FFB000D092CE003196F5CF8091C80085FFFCCF5E
:10FFC0008AE08093CE00812C912C60E2A62E61E421
:10FFD000B62E8092351990923619A0923719B092A8
:10FFE00038198092391990923A19A0923B19B0921F
:10FFF0003C19E090141920E030E040E752E46091B1
:020000021000EC
:10000000D0027091D1028091D2029091D3020F94CC
:10001000A90F6D877E878F87988B80913D1990916E
:100020003E19A0913F19B091401989829A82AB8202
:10003000BC828D829E82AF82B88689879A87AB8781
:10004000BC87AE01475F5F4FBE016B5F7F4FCE0144
:1000500001960E94432E8E01035F1F4F21E439E178
:10006000AE01475F5F4FBE016B5F7F4FCE010196D0
:100070000E94366080E090E8A2E2B5E480934119E6
:1000800090934219A0934319B093441981E499E1E4
:100090000E94DB2DEEE3F0E18491882341F0909102
:1000A000C80095FFFCCF8093CE003196F5CF8091AC
:1000B000C80085FFFCCF8AE08093CE0024E0D29E6A
:1000C00050011124C501845F964E4C01FC01208132
:1000D0003181428153816DEC7CEC8CEC9DE30F947B
:1000E000A90F9B01AC016091411970914219809157
:1000F0004319909144190F94AE0E60934119709377
:100100004219809343199093441980E090E0A0E74E
:10011000B2E48093E9029093EA02A093EB02B093D9
:10012000EC0280E090E0A0E8BFE3809303039093AB
:100130000403A0930503B0930603898F9A8FAB8FB6
:10014000BC8F80913D1990913E19A0913F19B091BB
:1001500040194091391950913A1960913B197091A9
:100160003C190091351910913619209137193091A9
:1001700038190D871E872F87388B498B5A8B6B8BCD
:100180007C8B8D8B9E8BAF8BB88FAE014B5E5F4FA0
:10019000BE016F5E7F4FCE010D960E94432EED2C67
:1001A0008E01075E1F4F21E439E1AE014B5E5F4FC8
:1001B000BE016F5E7F4FCE010D960E943660F40146
:1001C000208131814281538160E070E088EC91E4CC
:1001D0000F94A90F9B01AC016091411970914219D4
:1001E00080914319909144190F94AE0E6093411978
:1001F00070934219809343199093441980E090E0E2
:10020000A6E1B4E48093E9029093EA02A093EB02A2
:10021000B093EC0280E090E0A0E2B1E48DA39EA355
:10022000AFA3B8A780913D1990913E19A0913F19B5
:10023000B09140194091391950913A1960913B1988
:1002400070913C1900913519109136192091371988
:1002500030913819098F1A8F2B8F3C8F4D8F5E8FFD
:100260006F8F78A389A39AA3ABA3BCA3AE014F5D04
:100270005F4FBE01635E7F4FCE0149960E94432EC1
:100280008E010B5D1F4F21E439E1AE014F5D5F4FE1
:10029000BE01635E7F4FCE0149960E9436600E9488
:1002A000775280E090E0AAE7B5E48093E90290936A
:1002B000EA02A093EB02B093EC0281E0D110A0C05F
:1002C0000E94774653E0969587955A95E1F7F82F67
:1002D000F170FF2EC501845F964E5C01F110E4C001
:1002E0000E94D42D81116FC0F5012081318142819E
:1002F000538160E070E080EA90E40F94A90F9B01C5
:10030000AC0160914119709142198091431990910B
:1003100044190F94AE0E6093411970934219809363
:1003200043199093441920E030E040E752E4609193
:10033000E9027091EA028091EB029091EC020F9435
:10034000A90F6DA37EA38FA398A780913D199091CB
:100350003E19A0913F19B09140194091391950911F
:100360003A1960913B1970913C190091351910911F
:100370003619209137193091381909AB1AAB2BABCC
:100380003CAB4DA75EA76FA778AB89A79AA7ABA791
:10039000BCA7AE01475D5F4FBE01635D7F4FCE01DD
:1003A000C1960E94432EED2C8E010B5D1F4F21E460
:1003B00039E1AE01475D5F4FBE01635D7F4FCE0106
:1003C000C1960E94366020E030E0A9016091411999
:1003D0007091421980914319909144190F94C30A66
:1003E00018160CF43DC0EDE1F0E18491882399F0FA
:1003F0009091C80095FFFCCF8093CE003196F5CF49
:100400000E94774645E0969587954A95E1F7282F13
:100410002170F22E5FCF8091C80085FFFCCF8AE06B
:100420008093CE0080911419811117C082E390E06F
:100430000E94963C8F2DE4960FB6F894DEBF0FBE57
:10044000CDBFDF91CF911F910F91FF90EF90DF9083
:10045000BF90AF909F908F90089583E390E0E8CF96
:1004600081E0D11019C00E94774633E096958795B8
:100470003A95E1F7182F11700E94BE4C0E94D4519A
:100480000E94A92E0E941F410E948E738091AE137C
:10049000807C81F2F12E22CF0E94774625E096954E
:1004A00087952A95E1F7E6CF0E94775220E030E069
:1004B0004AE754E4609141197091421980914319BF
:1004C000909144190F940F1187FDB4CFE5EFFFE031
:1004D0008491882341F09091C80095FFFCCF8093D0
:1004E000CE003196F5CF8091C80085FFFCCF8AE021
:1004F0008093CE0080911419811106C080E490E0B1
:100500000E94963CF12C96CF81E490E0F9CFE9E986
:10051000FDE08491882341F09091C80095FFFCCFC5
:100520008093CE003196F5CF8091C80085FFFCCF37
:100530008AE08093CE0065E070E080E090E00E9469
:1005400068B40E94BE4C0E94D4510E9455B0E0E9AC
:10055000FDE08491882341F09091C80095FFFCCF85
:100560008093CE003196F5CF40912A0B50912B0B02
:1005700060912C0B70912D0B4F5F5F4F6F4F7F4F32
:1005800085E499E10E94853A8091C80085FFFCCFFF
:100590008AE08093CE000E942F30ECE8FDE0849149
:1005A000882341F09091C80095FFFCCF8093CE0046
:1005B0003196F5CF8091C80085FFFCCF8AE080930B
:1005C000CE0008956F927F928F929F92AF92BF92CA
:1005D000CF92DF92EF92FF920F931F93CF93DF930F
:1005E000CAE4DAE078EE872E73E0972EA12CB12CC6
:1005F00077247394809172189091731820917418D5
:1006000030917518821B930B9370892BD9F08091D0
:10061000AF138830B8F40E9433B0E0915D0A8A309D
:1006200069F08D3059F08C3249F08A3321F4909181
:100630000905992319F0E93408F42AC4E11111C01D
:1006400010920905DF91CF911F910F91FF90EF90CC
:10065000DF90CF90BF90AF909F908F907F906F90E2
:1006600008950091AB04C09F900111242751384F89
:10067000E20FF32FF11D108280910905811105C44D
:100680000C9F8001112498012751384F79016EE4A5
:1006900070E0C9010F947C12009709F4DEC29093B8
:1006A000DB0A8093DA0A8E199F09800F911F4AE0B6
:1006B00050E070E060E08651984F0F942A096093F3
:1006C000DE0A7093DF0A8093E00A9093E10A6115D5
:1006D00071058105910511F4109226072091AE1342
:1006E000203409F095C2C090AB040C2D10E0CC9ED4
:1006F00060011124D601A751B84F7D0120912A0B2A
:1007000030912B0B40912C0B50912D0B62177307DE
:100710008407950749F40E942F30F7011192CA957A
:10072000E9F710925D0A8ECF2F5F3F4F4F4F5F4F1B
:10073000621773078407950759F067E877E0CD01E2
:100740000F94790A892B21F48091B80A8823D9F073
:100750006AE270E0C7010F947C12892B09F07FC018
:10076000E0ECF7E284918111DBC1EEEAF6E08491DE
:10077000882309F4DDC19091C80095FFFCCF8093D8
:10078000CE003196F4CF0E948782E0ECF7E28491AC
:1007900081110DC0E4E5F7E08491882381F0909108
:1007A000C80095FFFCCF8093CE003196F5CF909195
:1007B000C80095FFFCCF8093CE003196E8CF4091E2
:1007C0002A0B50912B0B60912C0B70912D0B85E413
:1007D00099E10E94853A8091C80085FFFCCF8AE0AC
:1007E0008093CE004091DE0A5091DF0A6091E00ACA
:1007F0007091E10A8FE397E00E94983A8091C800D7
:1008000085FFFCCF8AE08093CE0040912A0B509167
:100810002B0B60912C0B70912D0B8091DE0A909127
:10082000DF0AA091E00AB091E10A841B950BA60BA8
:10083000B70B853F9140A105B1050CF472CF14169A
:100840001506160617062CF083E690E00E94B133D9
:1008500068CF809126078F5F8093260762CF8091B3
:10086000330781118BC040E0612CC09F9001C19F74
:10087000300D11242751384F842F90E0F901E80FF3
:10088000F91F50815A3219F04F5F6526F5CFE80EF7
:10089000F91EF092DB0AE092DA0A8C0D9D1D70E0E1
:1008A00060E08651984F0F94CC070F941B1066168A
:1008B000170609F44EC1E0ECF7E2849181110DC0F6
:1008C000E0E2F7E08491882381F09091C80095FFE1
:1008D000FCCF8093CE003196F5CF9091C80095FF64
:1008E000FCCF8093CE003196E8CF40912A0B5091F7
:1008F0002B0B60912C0B70912D0B85E499E10E94DC
:10090000853A8091C80085FFFCCF8AE08093CE00B5
:10091000E091AB042AE4E29FF0011124E751F84F83
:100920008191882339F09091C80095FFFCCF809386
:10093000CE00F6CF8091C80085FFFCCF8AE080937F
:10094000CE00E6E1F7E08491882341F09091C80061
:1009500095FFFCCF8093CE003196F5CF662D70E0E9
:1009600090E080E00E94EC1A8091C80085FFFCCFE7
:100970008AE08093CE000E948782D3CE20E0C09F81
:10098000A001C19F500D11244751584F822F90E074
:10099000FA01E80FF91F30813A3211F02F5FF6CFDC
:1009A00040915D0A9C012A5F3F4F4217130609F0F0
:1009B0000CF444C0E0ECF7E2849181110DC0E7EF44
:1009C000F6E08491882381F09091C80095FFFCCFD8
:1009D0008093CE003196F5CF9091C80095FFFCCF63
:1009E0008093CE003196E8CF40912A0B50912B0B8B
:1009F00060912C0B70912D0B85E499E10E94853A52
:100A00008091C80085FFFCCF8AE08093CE00E09102
:100A1000AB043AE4E39FF0011124E751F84F8191D0
:100A2000882339F09091C80095FFFCCF8093CE00C9
:100A3000F6CF8091C80085FFFCCF9ACFF7010FEF6A
:100A40001FEF9F012E193F0928173907B8F421918C
:100A5000022E000C330B0227132728E030E0A801F8
:100A60004170552716950795452B21F041E0042745
:100A700040EA14272150310991F7E3CF8C0D9D1DD9
:100A800070E060E08651984F0F94CC070F941B10D4
:100A90000617170709F45DC0E0ECF7E284918111B5
:100AA0000DC0E8EDF6E08491882381F09091C800B4
:100AB00095FFFCCF8093CE003196F5CF9091C80082
:100AC00095FFFCCF8093CE003196E8CF40912A0B62
:100AD00050912B0B60912C0B70912D0B85E499E1BB
:100AE0000E94853A8091C80085FFFCCF8AE0809300
:100AF000CE00E091AB048AE4E89FF0011124E751B5
:100B0000F84F8191882339F09091C80095FFFCCF70
:100B10008093CE00F6CF8091C80085FFFCCF28CF10
:100B20009091C80095FFFCCF8093CE0031961ACEED
:100B300040912A0B50912B0B60912C0B70912D0B37
:100B400085E499E10E94853A8091C80085FFFCCF39
:100B50000FCF8091DE0A9091DF0AA091E00AB09158
:100B6000E10A80932A0B90932B0BA0932C0BB0934C
:100B70002D0B0091AB040C9F80011124C8018751FB
:100B8000984F7C0167E470E00F947C12009709F4A1
:100B90003DC19093DB0A8093DA0A8E199F09800F7A
:100BA000911F70E060E08651984F0F94CC070F942E
:100BB0001B106430710508F029C18091D60A90910C
:100BC000D70A009741F420914D05211104C02091CE
:100BD000EE0A2111A7C02091EE0AE7E7F6E02223F2
:100BE00009F4FBC0892B09F0DBC080914D058823F7
:100BF00009F40CC1EAE5F6E08491882309F4F8C011
:100C00009091C80095FFFCCF8093CE003196F4CF31
:100C1000207C09F0AECF00912A0B10912B0B209174
:100C20002C0B30912D0B601B710B820B930B653FCE
:100C30007140810591050CF49CCF10161106120627
:100C400013062CF083E690E00E94B13392CF80919E
:100C500026078F5F809326078CCF6AE270E0C7017A
:100C60000F947C12892B09F484CFE0ECF7E2849195
:100C700081110DC0E4E8F6E08491882381F0909121
:100C8000C80095FFFCCF8093CE003196F5CF9091B0
:100C9000C80095FFFCCF8093CE003196E8CF4091FD
:100CA0002A0B50912B0B60912C0B70912D0B85E42E
:100CB00099E10E94853A8091C80085FFFCCF8AE0C7
:100CC0008093CE00E091AB04BAE4EB9FF0011124D5
:100CD000E751F84F8191882339F09091C80095FF32
:100CE000FCCF8093CE00F6CF8091C80085FFFCCF6B
:100CF0008AE08093CE00E091AB048AE4E89FF001A3
:100D00001124E751F84FDF011D928A95E9F7E2E7D8
:100D1000F4E180E094E0DF019C011D92215030401D
:100D2000E1F729CE8091AE13807CECE7F6E08034C9
:100D300009F043C0E1E8F6E08491882341F0909106
:100D4000C80095FFFCCF8093CE003196F5CF60911F
:100D5000DE0A7091DF0A8091E00A9091E10AA50114
:100D600094010F943D0EAB01BC018FE796E00E9409
:100D7000983A8091C80085FFFCCFD093CE000E94A6
:100D80009AB46093CE0A7093CF0A8093D00A90935E
:100D9000D10A8091D60A9091D70A892B09F436C0DE
:100DA000E4EEF5E08491882359F19091C80095FF15
:100DB000FCCF8093CE003196F5CF8491882341F00B
:100DC0009091C80095FFFCCF8093CE003196F5CF6F
:100DD0008091C80085FFFCCFD0CF84918823C9F2D1
:100DE0009091C80095FFFCCF8093CE003196F5CF4F
:100DF0008091C80085FFFCCF8AE08093CE0022CC92
:100E00008091C80085FFFCCFD093CE000091AB0449
:100E10000C9F80011124D801A751B84F7D016DE4CA
:100E200070E0CD010F947C129093DB0A8093DA0A74
:100E30008E199F09800F911F4AE050E070E060E03A
:100E40008651984F0F942A096936710581059105DD
:100E500011F00E949AB48091AB0490E0E0915D0A99
:100E6000C89F9001C99F300D11242751384FE20FC0
:100E7000F32FF11D10820196877099278093AB04A0
:100E80008091AF138F5F8093AF1310925D0AB2CB46
:100E9000E1110DC0A091AB04AC9FD00111249D01C4
:100EA0002751384FD901FC2F1D92FA95E9F78B3362
:100EB00011F4709209059091090591119BCB209135
:100EC000AB0491E09E0F90935D0AC29F90011124A4
:100ED0002751384FE20FF32FF11D80838BCB5F92A8
:100EE0006F927F928F929F92AF92BF92CF92DF923A
:100EF000EF92FF920F931F93CF93DF93CDB7DEB79F
:100F000064970FB6F894DEBF0FBECDBF8093BD0AC5
:100F1000823008F44AC0E3ECFDE2849181110DC0F7
:100F2000E4EBF7E08491882381F09091C80095FF6D
:100F3000FCCF8093CE003196F5CF9091C80095FFFD
:100F4000FCCF8093CE003196E8CF6091BD0A70E06F
:100F500090E080E00E94EC1AEBEEF3E081918823B0
:100F600039F09091C80095FFFCCF8093CE00F6CF6A
:100F70008091C80085FFFCCF8AE08093CE00649604
:100F80000FB6F894DEBF0FBECDBFDF91CF911F919A
:100F90000F91FF90EF90DF90CF90BF90AF909F9018
:100FA0008F907F906F905F90089586E40E94B73095
:100FB000882399F00E94D9306B017C0120E030E059
:100FC000A9010F940F11181644F4C092E902D092AF
:100FD000EA02E092EB02F092EC029091BD0A80915D
:100FE0001419981709F46EC21092300280E1E5E3FB
:100FF000F9E1DE01119601900D928A95E1F7C0901A
:101000003D19D0903E19E0903F19F090401920E032
:1010100030E04AEF53E4C701B6010F94C30A812CB4
:10102000912C540118169CF120E030E040E050E48F
:10103000C701B6010F94AF0E60933D1970933E192E
:1010400080933F199093401920E030E040E752E44C
:101050006091D8027091D9028091DA029091DB02FE
:101060000F94A90FB4E1CB2EB9E1DB2E7B018C01EB
:1010700021E439E14DE359E169E379E185E399E15F
:101080000E94B652812C912CA12C10E4B12E80919B
:10109000BD0A8130C9F520E030E0A9016091351921
:1010A0007091361980913719909138190F94C30AAD
:1010B00087FF2AC0109235191092361910923719ED
:1010C000109238196091D0027091D1028091D202B1
:1010D0009091D3029B01AC010F94AF0E20E030E061
:1010E00040E752E40F94A90FA4E1CA2EA9E1DA2E39
:1010F0007B018C0121E439E14DE359E169E379E1B8
:1011000085E399E10E94B6528091BD0A811157C0D2
:10111000C0903519D0903619E0903719F0903819F1
:1011200020E030E045E254E4C701B6010F940F110E
:1011300018160CF044C0E091141984E0E89FF00107
:101140001124E159FD4F2081318142815381C70132
:10115000B6010F94AF0E20916F0230917002409152
:101160007102509172020F94AE0E60933519709314
:10117000361980933719909338196091D002709185
:10118000D1028091D2029091D3029B01AC010F94C5
:10119000AF0E20E030E040E752E40F94A90FF4E1F5
:1011A000CF2EF9E1DF2E7B018C0121E439E14DE303
:1011B00059E169E379E185E399E10E94B652009132
:1011C000141910E05090BD0AE52CF12C6801CC0CEC
:1011D000DD1CCC0CDD1CF601E159FD4F2081318175
:1011E0004281538160913519709136198091371978
:1011F000909138190F94AE0E3701660C771C660C6F
:10120000771CF301E159FD4F2081318142815381E7
:101210000F94AF0E60933519709336198093371978
:1012200090933819F601E958FD4F208131814281B0
:1012300053816091391970913A1980913B199091BD
:101240003C190F94AE0EF301E958FD4F2081318116
:10125000428153810F94AF0E6093391970933A19FC
:1012600080933B1990933C19F601E959FD4F208179
:1012700031814281538160913D1970913E19809175
:101280003F19909140190F94AE0EF301E959FD4FAB
:1012900020813181428153810F94AF0E60933D19BB
:1012A00070933E1980933F199093401981E0581232
:1012B00015C16091D0027091D1028091D2029091BB
:1012C000D3029B01AC010F94AF0E20E030E040E769
:1012D00052E40F94A90F44E1C42E49E1D42E7B01BE
:1012E0008C0121E439E14DE359E169E379E185E3DA
:1012F00099E10E94B6520E947752E7EAF7E08491A2
:10130000882341F09091C80095FFFCCF8093CE00D8
:101310003196F5CF8091C80085FFFCCF8AE080939D
:10132000CE0010E000E04E9B17C00E94D42D833009
:1013300048F43799CBC065E47DE081E00E9430231A
:101340000B5B124F0E94BE4C0E94D4510E94A92EEA
:101350000D3E8FE018073CF3B801110F880B990B75
:101360000F94CA0A26E636EE47E053E40F94A90F1D
:10137000AB01BC0180EA97E00E9441328091C80035
:1013800085FFFCCF8AE08093CE0068E870E081E0C2
:101390000E94302380914602909147020E94A1470B
:1013A00080E090E0AEE2B4E48093390290933A0298
:1013B000A0933B02B0933C0280E1FE013196A5E38D
:1013C000B9E101900D928A95E1F78091BD0A8111F2
:1013D00034C0C0903519D0903619E0903719F0908C
:1013E000381920E030E045E254E4C701B6010F941B
:1013F0000F11181614F5E091141984E0E89FF0011C
:101400001124E159FD4F2081318142815381C7016F
:10141000B6010F94AF0E20916F023091700240918F
:101420007102509172020F94AE0E60933519709351
:1014300036198093371990933819A501940160915A
:101440003D1970913E1980913F19909140190F9468
:10145000AF0E698B7A8B8B8B9C8BAE014F5E5F4F8F
:1014600069E379E185E399E10E9427AD8091BD0AA6
:101470008093141980E090E0A4E3B3E48093E90240
:101480009093EA02A093EB02B093EC0280E090E02C
:10149000A0E4B0E48093030390930403A0930503B6
:1014A000B093060324E1C22E29E1D22E7C018D01E6
:1014B00021E439E14DE359E169E379E185E399E11B
:1014C0000E94B65281E08093300259CD68E070E00E
:1014D00081E00E943023085F1F4F34CF0E94775273
:1014E000E3E9F7E08491882341F09091C80095FFEB
:1014F000FCCF8093CE003196F5CF8091C80085FF58
:10150000FCCF8AE08093CE0010E000E0379B13C050
:101510004E995EC065E47DE080E00E9430230B5B65
:10152000124F0E94BE4C0E94D4510E94A92E0D3E23
:101530008FE018075CF368E870E080E00E943023D9
:10154000B801110F880B990B0F94CA0A26E636EEE4
:1015500047E053E40F94A90FAB01BC018CE897E07E
:101560000E9441328091C80085FFFCCF8AE08093C1
:10157000CE006091D0027091D1028091D202909100
:10158000D3029B01AC010F94AF0E20E030E040E7A6
:1015900052E40F94A90F34E1C32E39E1D32E7B011D
:1015A0008C0121E439E14DE359E169E379E185E317
:1015B00099E10E94B6520E94775280912307909140
:1015C00024070E940D4880E090E0A5E2B4E4ECCE50
:1015D00068E070E080E00E943023085F1F4FA1CFD9
:1015E0008F929F92AF92BF92CF92DF92EF92FF9233
:1015F0000F931F93CF93DF93CDB7DEB7CA54D109B2
:101600000FB6F894DEBF0FBECDBF0091FB02109164
:10161000FC02B801012E000C880B990B0F94CA0A2A
:101620004B015C01C0900A0BD0900B0BE0900C0BAF
:10163000F0900D0BA70196010F94C30A87FDADC072
:1016400020E030E0A901C701B6010F94C30A87FD6D
:101650009FC0C701B6010F941B107093150B6093C8
:10166000140BC0900E0BD0900F0BE090100BF0906D
:10167000110BA5019401C701B6010F940F111816A3
:101680000CF090C01093170B0093160B8091AE13C3
:10169000807C83608093AE1383E08093DC0A80912A
:1016A000B2049091141989130E946F87FF24F39458
:1016B0008091AE138F73833009F01CC1009114190F
:1016C00010E0F801EE0FFF1FEC5EF44F60817181B6
:1016D000072E000C880B990B0F94CA0A000F111FDC
:1016E000000F111FF801E85EF44F20813181428123
:1016F00053810F94AE0E20E030E040EA50E40F94A6
:101700000F1118160CF0F6C00E941F410E94BE4C2B
:101710000E94D4510E94A92E809172189091731842
:101720002091741830917518821B930B9370892B3C
:1017300009F4BECF0E9433B08A3069F08D3059F081
:101740008A3321F490910905992329F0E0915D0AEB
:10175000E93408F4BAC060E87CE0CE0101960F9449
:10176000790A892BB1F1C65BDF4F0FB6F894DEBF63
:101770000FBECDBFDF91CF911F910F91FF90EF90E2
:10178000DF90CF90BF90AF909F908F900C9431726C
:101790001092150B1092140B64CF1093150B00933D
:1017A000140B5FCF20E030E0A901C701B6010F9410
:1017B000C30A87FF05C01092170B1092160B66CF55
:1017C000C701B6010F941B107093170B6093160B93
:1017D0005DCF6BE77CE0CE0101960F94790A892BEF
:1017E00009F470C0E0E7FCE08491882341F0909117
:1017F000C80095FFFCCF8093CE003196F5CF809145
:10180000C80085FFFCCF8AE08093CE000E94A83AF2
:101810000E942C3240913407509135076091360771
:101820007091370789E59CE00E94983A8091C80042
:1018300085FFFCCF8AE08093CE000E941170EBE41C
:10184000FCE08491882341F09091C80095FFFCCF83
:101850008093CE003196F5CF8091C80085FFFCCFF4
:101860008AE08093CE008091AE13807C8034B1F406
:101870002091AF1380912A0B90912B0BA0912C0BF0
:10188000B0912D0B821B9109A109B10980932A0BFC
:1018900090932B0BA0932C0BB0932D0BC65BDF4FBB
:1018A0000FB6F894DEBF0FBECDBFDF91CF911F9171
:1018B0000F91FF90EF90DF90CF90BF90AF909F90EF
:1018C0008F90089510925D0A27CF8B3311F4F09218
:1018D00009059091090591111FCF91E09E0F9093FA
:1018E0005D0A21E030E02C0F3D1F2E0F311DF90164
:1018F000808312CF0E94717920E030E040EA50E40A
:101900006091020B7091030B8091040B9091050B79
:101910000F94AF0E60933D1970933E1980933F1959
:10192000909340196091D8027091D9028091DA02A7
:101930009091DB029B01AC010F94AF0E20E030E0F0
:1019400040E752E40F94A90F34E1C32E39E1D32EBE
:101950007B018C0121E439E14DE359E169E379E14F
:1019600085E399E10E94B6528091FD06882309F42F
:1019700047C1409134075091350760913607709107
:10198000370740932A0B50932B0B60932C0B7093CB
:101990002D0B8091BF059091C005A091C105B0911C
:1019A000C2058093411990934219A0934319B093B3
:1019B000441981E39CE00E94983A8091C80085FF19
:1019C000FCCF8AE08093CE0070E060E086E19CE08E
:1019D0000E946F3D8091C80085FFFCCF8AE0809314
:1019E000CE006091FB0670E082E09CE00E946F3DBB
:1019F0008091C80085FFFCCF8AE08093CE001092D2
:101A0000FD0680912A0B90912B0BA0912C0BB0918D
:101A10002D0B8F3F9F4FAF4FBF4F5CF48FEF9FEF6A
:101A2000DC0180932A0B90932B0BA0932C0BB0938B
:101A30002D0B81E499E10E94DB2D20E030E040E7AE
:101A400052E46091E5027091E6028091E702909184
:101A5000E8020F94A90F24E1C22E29E1D22E7B01C6
:101A60008C0121E439E14DE359E169E379E185E352
:101A700099E10E94B6526091D0027091D10280919A
:101A8000D2029091D3029B01AC010F94AF0E20E0E3
:101A900030E040E752E40F94A90F7B018C0121E470
:101AA00039E14DE359E16EEF7AE08AEF9AE00E9466
:101AB000B6526091D8027091D9028091DA02909169
:101AC000DB029B01AC010F94AF0E20E030E040E759
:101AD00052E40F94A90F7B018C0121E439E142E02B
:101AE0005BE06EEF7AE08AEF9AE00E94B6520E94C5
:101AF00077528091FA0A9091FB0AA091FC0AB0916A
:101B0000FD0A8093351990933619A0933719B09335
:101B100038198091FE0A9091FF0AA091000BB091B4
:101B2000010B8093391990933A19A0933B19B09304
:101B30003C198091FD06882309F486C01092FD06A9
:101B40008091C3059091C405A091C505B091C605CB
:101B500080933D1990933E19A0933F19B09340197B
:101B60006091D0027091D1028091D2029091D30203
:101B70009B01AC010F94AF0E20E030E040E752E44F
:101B80000F94A90F7B018C0121E439E14DE359E168
:101B900069E379E185E399E10E94B6526091B90A5F
:101BA0007091BA0A8091BB0A9091BC0A6093E902D5
:101BB0007093EA028093EB029093EC0220E030E015
:101BC00040E752E40F94A90F60930303709304035A
:101BD00080930503909306031092DC0A8091AE1364
:101BE000807C8093AE13E4EFFBE084918823E9F1DD
:101BF0009091C80095FFFCCF8093CE003196F5CF31
:101C000080912A0B90912B0BA0912C0BB0912D0B56
